:020000040000FA
:040000006FD00400B9
:101000006F00907E00000000000000009020002093
:10101000AA220020A9BDF9F56C23002000000000E1
:10102000000000006C230020902000200000000041
:101030000000000090200020000000009020002010
:101040000000000090200020902000209020002030
:101050009020002090200020582F00209424002071
:101060000000000090200020902000201E2400207E
:1010700090200020D22300209020002090200020EB
:101080009020002090200020902000209020002020
:101090009020002001A04111B7170040985F3AC688
:1010A000945F3247E39CE6FE3245410182800111A4
:1010B00013078008F337078093F787083EC20100C3
:1010C0000100B7170040930570052380B70413068D
:1010D00080FA2380C7040100010083C6B70493F699
:1010E000F60DA385D704238007049246F3A6068055
:1010F0000100010093760502D5CEF336078093F602
:10110000860836C4010001002380B7042380C70489
:1011100001000100B70614007D89558D88C70100C4
:1011200001000100010023800704A246F3A6068007
:101130000100010073370780137787083AC6010062
:1011400001002380B7042380C704010001000100CF
:1011500001003727004093061005A303D7802380A2
:101160000704B247F3A70780010001009307800836
:10117000F3B7078093F787083ECE01000100B71749
:101180000040130770052380E704130780FA2380CB
:10119000E7040100010003C7B70413670708A3852C
:1011A000E70423800704F247F3A70780010001004A
:1011B0000561828093760504BDC6F336078093F6F9
:1011C000860836C8010001002380B7042380C704C5
:1011D00001000100B7061400938606047D89558D31
:1011E00088C7010001000100010023800704C246F6
:1011F000F3A6068001000100733707801377870884
:101200003ACA010001002380B7042380C70401000B
:1012100001003727004093062005A303D7802380D1
:101220000704D24781B773370780137787083ACC12
:10123000010001002380B7042380C70401000100DE
:1012400098471367070C98C723800704E24719BF24
:101250000111814601468145114506CE97000000E7
:10126000E780605893078008F3B7078093F78708F3
:101270003EC601000100B717004013077005238028
:10128000E704130780FA2380E7040100010003C785
:101290006704136717002383E70423800704B2471A
:1012A000F3A7078001000100F2400561828041112F
:1012B000814601468145114597000000E780A05214
:1012C00013078008F337078093F787083EC40100AF
:1012D0000100B7170040130670052380C70493066A
:1012E00080FA2380D70401000100FD552396B70240
:1012F00023800704A245F3A5058001000100733790
:101300000780137787083AC6010001002380C704CD
:101310002380D7040100010003C767041367170087
:101320002383E70423800704B247F3A70780010063
:10133000010001A0BD473305F50201007D1575FDD3
:101340008280411122C426C206C6AA8401446317C2
:101350009400B24022449244410182800504130566
:10136000803E420497000000E78000FD4180C5B741
:101370009305000273A04580824573901534924016
:101380002242B2424243D2436244F2440255925551
:101390002256B2564257D2576258F25806499649D9
:1013A000264AB64A464BD64B664CF64C065D965DD1
:1013B000265EB65E465FD65F09617300203041113C
:1013C000B7170040985F3AC6945F3247E39CE6FE49
:1013D000324541018280B71700401307000323887C
:1013E000E702854717170000232EF74673002030C9
:1013F000411122C42D6426C24AC006C637190040D6
:101400001304A4AAB704002023208900977000E0E9
:10141000E780C02E9C408297977000E0E780002E06
:10142000E5B737370040834747009146BD8B639E41
:10143000D702B73600401306F00F973500009385AA
:10144000E5219737000083D7673103C7A6001377DC
:10145000F70F1DE3B7E70400BC4F09468945171590
:1014600000000345A5F7829731A099466394D70001
:10147000834757007300203003C786001377F70FA8
:10148000E365F6FC13851700AE97173800002317A5
:10149000A82C2380E70075B7B787004003C7670013
:1014A000098B6309071003C77700930600031377BE
:1014B0000703630DD708174800000348F880173664
:1014C00000001306667D0547B30606012380E6008B
:1014D00083C57700173700001307077E429793F5FF
:1014E000F50F2300B70003C58700973500009385EB
:1014F000A57BC2951375F50F2380A5000347070050
:1015000089451377F703630CB70C63E7E50A6306B5
:10151000071A8545630CB7129737000083C7D77A3F
:101520003307F600034707001377F70F19CB85073A
:1015300093F7F70F3D476363F71A17370000A305CA
:10154000F778B787004009472383E700B787004053
:1015500083C77700E207E18763DE0704973700005F
:1015600083C7977617370000130707733E978546A2
:101570002300D70017370000130707743E97930620
:1015800000032300D700173700001307E7713E97C9
:10159000A14685072300D70093F7F70F3D47636403
:1015A000F71417370000A301F772B7870040094707
:1015B0002383E70073002030930610026300D70EE8
:1015C000930620026305D70693060002E316D7F4BC
:1015D00003C727021377C70F13672700D5A803C7D0
:1015E00067001377070465CB03C7A702173800000D
:1015F0001308084C17350000130545431347070827
:101600002385E70203C7A7021377370F1367870005
:101610002385E702814713070004B305F5008C41D9
:10162000B306F80091078CC2E399E7FEF5B503C74E
:10163000A702134707042385E70203C7A70213770E
:10164000C70F136727002385E702F9B503C76700B3
:101650001377070449C303C767021738000013084C
:10166000E838173500001305253013470708238392
:10167000E70203C767021377370F136787002383D7
:10168000E702814713070004B305F5008C41B30658
:10169000F80091078CC2E399E7FEBDBD03C767025E
:1016A000134707042383E70203C767021377C70FB3
:1016B000136727002383E70285B503C76700137705
:1016C000070411CB03C727021377370F136787006F
:1016D0002381E70291B5238006003DBD97370000C6
:1016E000A384075EB9BD97370000A38F075C75BD63
:1016F0002303048015472303E48001002302A48010
:10170000828083076480E3CE07FE23030480828007
:1017100083076480E3CE07FE03454480828083070D
:101720006480E3CE07FE2302A4808280411126C498
:101730004AC24EC006C61377F50BAD47AA892E895B
:101740009544630CF700194597000000E78080FA84
:1017500097000000E78020FB8D444E859700000035
:10176000E78040F9FD59FD1463983401B240A2446A
:101770001249824941018280135509011375F50F01
:1017800097000000E780E0F92209F1BF011126CCA3
:1017900006CEB704080097000000E780C0F61545A4
:1017A00097000000E78000F597000000E78080F6D2
:1017B00097000000E78000F62AC697000000E78047
:1017C00080F432459377150089EB13651500137586
:1017D000F50FF240E24405618280FD14E9F0014515
:1017E000CDBF397126DC4ADA4ED852D656D45AD2F9
:1017F0005ED006DE62CE66CCB7E700E07D5783AAF6
:10180000070022C603AA470023A0E71823A2E7186F
:10181000B7170040130770052380E704130780FA09
:101820002380E70483C74704930B75FFB684E20760
:1018300093FBFB0F8546AA892E8B32893724004003
:10184000E187015763FA76016308D50089461307DB
:1018500000026313D5000157D98F93F7F70FB71C18
:1018600000402382FC0411472303E4801305F00F9A
:1018700097000000E78000E8094C97000000E7802F
:1018800080E863657C15B7050700DA9537870700A0
:10189000795563FEE504B3879500636AF704370B57
:1018A0000800A94733EB65016395F90881E8814495
:1018B00097000000E78020E5268515A8DA85094510
:1018C00097000000E780C0E605090345F9FFFD1415
:1018D000050B97000000E780C0E481C49377FB0FFD
:1018E000E5F797000000E780A0EA69F17D55B7179A
:1018F0000040130770052380E704130780FA238054
:10190000E70403C74704418B2382E704F250B7E79B
:1019100000E023A0571123A24711E2543244525948
:10192000C259325AA25A125B825B724CE24C21615C
:101930008280A547639BF90685691309F00FB306FA
:101940009900B3742B01B6941349F9FFB37499004D
:10195000856B33796901416B9387F9FFB3F72701F1
:1019600099E363FC340193D94900C147E3E637FFAB
:101970003DBF0569C1697D19D9B71305800D63881D
:101980006901130500026384790113051008CA85F3
:1019900097000000E780C0D997000000E78040DF93
:1019A00031D54E99B38434416DBFDA852D4597000A
:1019B0000000E780E0D7CA94E30B99EE0509970091
:1019C0000000E78020D5A30FA9FEFDB79387F9FF9C
:1019D00093F7F70F636DFC0C83C71C0413073008E3
:1019E0006315F706370708006361EB06B3079B0032
:1019F000B706100063FBD704334BEB0089476399AC
:101A0000F9068980D549E38404EADA850945970017
:101A10000000E780E0D111090327C9FF9147232087
:101A2000E48003076480E34E07FE23033481FD173F
:101A3000EDFBFD14110B81C49377FB0FE9FF9700B9
:101A40000000E780E0D461F155B5B717004003C747
:101A50005704B70708001377070219E3B787070091
:101A60007955E376FBE833079B00E3F9E7F841B5E6
:101A70008547E380F9F0DA852D4597000000E7807F
:101A800020CB9389F4FFE38404E297000000E78011
:101A900060C893F7390091EB83260480032709007F
:101AA00093074900E396E6E03E89CE84D9BFB54767
:101AB0006399F9001305900B97000000E78080C33D
:101AC000FDB3B1471305B00AE388F9FE9947639760
:101AD000F904B7050800B365BB002D459700000069
:101AE000E78000C581448D4BA14997000000E78045
:101AF00060C263967401832704802320F900850463
:101B0000E39534FF8327048013172B0163550700E7
:101B10002312F90069BB2322F90051BB9D47639F43
:101B2000F90281451305B00497000000E78040C02A
:101B3000BD442320090023220900FD59970000001D
:101B4000E78040BD93F77400CA9703C70700FD14F0
:101B5000398D2380A700E39334FF91BBA14763979E
:101B6000F90697000000E780A0C28144630D0B00D6
:101B70008D479304C0036308FB00930400056304CE
:101B80008B01930440041375C507E30295D21945F0
:101B900097000000E78000B697000000E780A0B63D
:101BA000054597000000E780E0B426859700000017
:101BB000E78020B7094597000000E78080B69700CE
:101BC0000000E780E0BCE31405CE0DB39147639FAE
:101BD000F9001305600697000000E780A0B19700A8
:101BE0000000E78040B213059009F9B5E38109CC04
:101BF000F1547DB9BD66014717360000130606395A
:101C0000938606A685458347060093F7F70F91C391
:101C100082800507E3F9E6FE973700002388B73690
:101C2000DDB77D166206618693178601E18763D46E
:101C3000070001458280931726003307F500AE9711
:101C400018439C4363E7E7007D16E37FF7FC7D556F
:101C5000828005458280FD15E205E18513978501A7
:101C6000618793F7F50F63480700FD15139725006B
:101C70002A97584365D713851700620561858280CE
:101C80003308B5021C4283A80600B335B502C297DB
:101C900033B50701AE98469585486367B5006394F0
:101CA000A50063E3070181480C43C6950CC388C2B5
:101CB0001CC2828081471397870161876343B70005
:101CC0008280139727002A97232007008507E5B70E
:101CD0008147014793968701E18663C5B6001335B6
:101CE0001700828093962700AA9694428507558F05
:101CF000D5B793D755408A07AA979C430545331516
:101D0000B5007D8D828017F3FFDFE702833D2A84D3
:101D100097000000E78060F405C5931725003E9406
:101D20000327C4FF814711EB7D1516053E9542053B
:101D3000418517F3FFDF6700033D05838507E5B79E
:101D40000145C5BF81471397870161876343C7007A
:101D5000828013972700B386E50094422A9785076F
:101D600014C3D5B77D1662066186014793178601B5
:101D7000E18763D50700133517008280931726008B
:101D8000B306F500AE9794429C437D16B58F5D8FE8
:101D9000F1BF8A05AA9501476363B500828083A6D7
:101DA000C5FFF11593D71600D98F9CC11397F60183
:101DB000E5B72A830148014701456343D700828084
:101DC000B387050183A80700B30706019C43C697A4
:101DD000AA976384F80033B517010507B308030118
:101DE000620723A0F80061871108C1BF2A83014759
:101DF0008147014563C3D70082803388E50083288B
:101E00000800330EE600032E0E003388A840330886
:101E1000C8416384080133B508018507B308E300AE
:101E2000E20723A00801E1871107E9B717F3FFDFF5
:101E3000E702232B0111B286B2842E86AA850A8579
:101E400097000000E780C0FA2A84A6850A859700DB
:101E50000000E78020E833348000060413351500C5
:101E6000018D056117F3FFDF6700E32917F3FFDF3B
:101E7000E702A3244111AA89AE8A328BB68402C23A
:101E800002C402C60144131C8401135C8C416349E3
:101E90009C02939B1400FD1B0549138CF4FFF15C1D
:101EA00033048901620461846340740792478E049D
:101EB000CE9423AEF4FE410117F3FFDF67006323E6
:101EC00013192400B30B2B01014A93172A00D6974C
:101ED00083A50B0088437800340050009700000071
:101EE000E78040DA050A93178A01E187F11BE35E78
:101EF000FCFC92474E9905042320F900A2473EC2FC
:101F0000B24702C63EC441B7131A8901135A8A4127
:101F1000131D240093178A01E18763CF970092472E
:101F20000A044E941CC0A24705091379F90F3EC25A
:101F3000B24702C63EC4ADB7B3079A0313152A00D1
:101F400056950841780034005000050AEA97DA9760
:101F50008C4397000000E780E0D26DBF197106C284
:101F600012C416C61AC81ECA22CC26CE2AD02ED219
:101F700032D436D63AD83EDA42DC46DECAC0CEC2C9
:101F8000D2C4D6C6DAC8DECAE2CCE6CEEAD0EED2F9
:101F9000F2D4F6D6FAD8FEDA971500009385058CB0
:101FA0008841E700050092402242B2424243D243B8
:101FB0006244F244025592552256B2564257D257C5
:101FC0006258F25806499649264AB64A464BD64BBD
:101FD000664CF64C065D965D265EB65E465FD65F45
:101FE0000961730020300000972100209381810156
:101FF000175100201301018117F5FFFF1305C500DC
:102000009705002093850500171600201306C6FDCE
:1020100063FAC5008322050023A055001105910530
:10202000E3EAC5FE171502001305C5219715002028
:102030009385C5FB171600201306C66563FAC50015
:102040008322050023A0550011059105E3EAC5FE92
:102050001715002013050564974500209385053F5B
:102060006377B500232005001105E36DB5FEFD4241
:10207000739002BC8D4273904280B722000093821D
:10208000828873900230970200209382A2F793E235
:1020900032007390523097520000938202BD7390C9
:1020A00012346FB0F47573002030397101436EC67D
:1020B00019A0397141536AC866CA62CC5ECE19A0B4
:1020C000397101535AD056D252D44ED64AD826DA54
:1020D00022DC06DE33016140828241114AC026C201
:1020E00022C406C68282B24D4101024D924C224C5E
:1020F000B24B4101024B924A224AB2494101024984
:1021000092442244B240410182803D432A87637356
:10211000C3029377F700BDEFADE5937606FF3D8AE6
:10212000BA960CC34CC30CC74CC74107E36BD7FE30
:1021300011E28280B306C3408A0697020000969699
:102140006780A6002307B700A306B7002306B700E1
:10215000A305B7002305B700A304B7002304B70005
:10216000A303B7002303B700A302B7002302B700FD
:10217000A301B7002301B700A300B7002300B700F5
:10218000828093F5F50F93968500D58D9396050182
:10219000D58D61B7939627009702000096968682A8
:1021A000E78086FA9680C1171D8F3E96E374C3F8C8
:1021B000A5B73367B500FD530D8B79E7B7877F7FF0
:1021C0009387F7F710419441B372F6003363F6003A
:1021D000BE92B3E262006397720C6318D606504158
:1021E000D441B372F6003363F600BE92B3E26200EC
:1021F0006398720A631BD60410459445B372F600C7
:102200003363F600BE92B3E262006391720A631E0A
:10221000D6025045D445B372F6003363F600BE9241
:10222000B3E26200639A72086311D60210499449BE
:10223000B372F6003363F600BE92B3E262006393BA
:1022400072085105D105E30FD6F6131706019397CF
:102250000601631CF7001357060193D706013305E7
:10226000F7409375F50F91E982804183C18333056F
:10227000F7409375F50F91E182801377F70F93F78D
:10228000F70F3305F74082800346050083C605003B
:10229000050585056313D60065FA3305D6408280AF
:1022A00011059105E312D6FE014582802105A105A5
:1022B000E31CD6FC014582803105B105E316D6FC4E
:1022C000014582804105C105E310D6FC01458280AD
:1022D000B717004003C777051377E70FA38BE70411
:1022E000130700F8A38DE7043D47238CE704130789
:1022F0005003A38CE70403C7A7051377D70F238DDB
:10230000E7048280B717004003C7E7020D89411137
:102310001377C70F498F93068008F3B6068093F6AC
:10232000860836C601000100930670052380D70495
:10233000930680FA2380D704010001002387E70277
:1023400023800704B247F3A7078001000100410181
:10235000828041112A83014E930E407E130F001993
:10236000930F400663E56E129308001913034006AD
:10237000B3781503854E0D4FA14F337365020D8958
:102380001335150063EFBE121308F6FF79467298F5
:102390004208135808013307C70213D61700BE07B7
:1023A00032976146B3F6C60213068070B386C60242
:1023B0003697A166F58F42075D8FB716004083C739
:1023C000F60293F70708A303F1000346710083C7E1
:1023D000F60293F70708E394C7FE83477100B71628
:1023E000004093F7F70F6388071293078008F3B74D
:1023F000078093F787083EC401000100B71700402B
:10240000930670052380D704930680FA2380D704AF
:102410000100010023AA070383C6170393E60608F9
:10242000A388D70223800704A247F3A707800100EF
:1024300001001166B71700407D16D45BC85F938515
:102440004703A98EF18EF5FA93068008F3B606804D
:1024500093F6860836C601000100930670052380B6
:10246000D704930680FA2380D7040100010098C1A5
:1024700003C7170313670704A388E7022380070431
:10248000B247F3A7078001000100410182807D135C
:102490003368E3039308E016630E08003368F30320
:1024A0009308D016630808009378330093B8180097
:1024B0009388D81633081E01131E0801135E0E01FF
:1024C00055B56393E5030548638608000148630337
:1024D00003002A8871087298FD15131E0801C205B1
:1024E000135E0E01C18179BD13F8150063F4BF00BE
:1024F0007908D5B713381800E5BF83C7F60293F7FC
:102500000708A303F1000346710083C7F60293F79F
:102510000708E394C7FE8347710093F7F70FF1DFD5
:10252000E9B531714AD966CB06DF22DD26DB4ED70D
:1025300052D556D35AD15ECF62CD6AC96EC7AA8C26
:1025400002D897100000E78020B12A8993078008FD
:10255000F3B7078093F787083EDA01000100B71749
:102560000040130770052380E704130780FA2380D7
:10257000E7040100010003C7F7021377770FA38771
:10258000E70203C7F70213678700A387E7022380E8
:102590000704D257F3A70780010001000545970003
:1025A0000000E78060D6130780C13347E902116A53
:1025B00093070AE893065002BD69930BA004814A71
:1025C000014B13048008930470057D1AB347F90288
:1025D0003307D7023EC0FD873ECC938709A69309F7
:1025E000803E3347F7023AC27D873AC43347390306
:1025F0008549B399990193D93940B306D702B30BF2
:102600007703B3C6F602B3CBFB0236C6FD8636C8E7
:1026100093D6FB4136CEB7460F0093860624334946
:10262000D9028566938606FAB3969601B389E902C4
:10263000130760553309D90293060010B389E902E4
:102640003349D902B3C9F9029316390036CA37198A
:102650000040FD8636D0930D090493D7F9413ED250
:10266000F336048093F6860836DC010001009307F8
:1026700070052380FD00930680FA2380DD000100B1
:1026800001008346390593F6860FA309D9048346D2
:10269000390593E61600A309D90423800D00E256FC
:1026A000F3A6068001000100130C80FA116DF336C9
:1026B000048093F6860836DE01000100930770055A
:1026C0002380FD0023808D01010001008346390530
:1026D000216693E60602A309D90483560905B3E6E9
:1026E000A6012318D90483560905D18E2318D904CD
:1026F00023800D00F256F3A60680010001008346F8
:10270000390593F606026381061A03463905218AC4
:102710006DDE081897100000E7800098733604807B
:1027200013768608B2C20100010023809D00238039
:102730008D0101000100B717004003C6370513766D
:10274000F60DA389C70403C6370513660602A389DD
:10275000C704835609052166B3E6A6012318D904E8
:1027600083560905D18E2318D90423800D0096467F
:10277000F3A60680010001008346390593F60602A0
:10278000638B061483463905A18AEDFE970000206D
:10279000E7806090AA8636D497000020E780A08F5B
:1027A000A256E30AD5FE835609054255B3E6A601B3
:1027B0002318D90497100000E780C08F834639059D
:1027C000A18AEDDE03560905834629058247337643
:1027D000CA00B306DA0293D5F641B296B388F64042
:1027E000E24733B8C6002E983308F840A247B3B684
:1027F00016013308D84063C70701631DF8009247EC
:1028000063FA1701C247634FF80E63950701B24799
:1028100063EAF80E894663E9660FF24693151800DD
:1028200013D3F8015E8613951800B365B30042D642
:1028300046D497D00100E780E0CE3258050B137BD9
:10284000FB0F63470001631A0838A25863870838F2
:1028500013081500B336A800B69513D6F5013298C3
:10286000B336C800AE9613581800FE06B3E606014C
:102870007336048013768608B2C6010001002380F7
:102880009D0023808D01010001000356C902B2960C
:10289000C206C1822316D90223800D00B646F3A6D4
:1028A00006800100010021B5F336048093F6860806
:1028B000B6C00100010023809D0023808D0101002E
:1028C00001008346390593E60602A309D904238053
:1028D0000D0086460DB5F336048093F68608B6C41F
:1028E0000100010023809D0023808D010100010073
:1028F0008346390593E60602A309D90423800D0017
:10290000A646BDB5E30B0BF0F336048093F68608BC
:10291000B6C801000100930680FA23809D00238041
:10292000DD00010001008346390593F5FC0F93F6A5
:10293000860FA309D90483463905CD8EA309D9048E
:1029400023800D00C646F3A6068001000100130592
:1029500080FA03463905930639051D8A631C9629BA
:102960007336048013768608B2CC0100010013068A
:1029700080FA23809D002380CD000100010003C662
:1029800006001376F60D2380C60003C60600136604
:1029900006022380C600835609051166D18E2318CE
:1029A000D904835609052166D18E2318D9042380C2
:1029B0000D00E646F3A6068001000100130680FA2A
:1029C0008346390593F60602638006268346390559
:1029D000130C3905A18AFDDA081897000000E7807A
:1029E000A06BF336048093F68608B6D00100010090
:1029F000930680FA23809D002380DD000100010002
:102A000083460C00116693F6F60D2300DC00834626
:102A10000C0093E606022300DC0083560905D18EE4
:102A20002318D904835609052166D18E2318D904A9
:102A300023800D008656F3A60680010001001306D0
:102A400080FA8346390593F60602638A0620834698
:102A50003905A18AEDFE97F0FF1FE780C0632A8C3D
:102A600097F0FF1FE7802063E30C85FF835609057D
:102A700011664255D18E2318D90497000000E780D3
:102A800060638346390513063905A18AFDDAF336FA
:102A9000048093F68608B6D401000100930680FAFC
:102AA00023809D002380DD00010001008346060095
:102AB00093F6F60D2300D60023800D00A656F3A64C
:102AC0000680010001008356090503462905D24707
:102AD000B376DA003306CA021305800C9355F6412B
:102AE0003696330DF6408257333CD6002E9C333653
:102AF000A601330CFC40330CCC40330885039256BE
:102B00004E86B335A5033305A503C29597D00100C2
:102B1000E78040A163468001631E0C16630C0D160E
:102B2000130615003335A6002E959356F5013696FB
:102B3000B335D600AA959396F50105828585D18E89
:102B40006346B000639D051A638B061A0356C902DB
:102B500015823305D6003336C500B2956348B00000
:102B6000639105241306F00F637DA622894663F363
:102B7000561593078008F3B7078093F78708BED6EA
:102B80000100010037170040930770052300F70488
:102B9000930780FA2300F704010001008356C7025F
:102BA00089678117D58FC207C1832316F7022300D7
:102BB0000704B657F3A7078001000100FA506A54D2
:102BC000DA544A59BA592A5A9A5A0A5BFA4B6A4C49
:102BD000DA4C4A4DBA4D296182801308F5FF33352E
:102BE000A800FD152E951356F5013298B336C8008E
:102BF000AA9695B9F336048093F68608B6CA010002
:102C0000010023809D002380AD0001000100834668
:102C10003905CD8EA309D90423800D00D646F3A62D
:102C200006800100010035B3F336048093F6860870
:102C3000B6CE0100010023809D002380CD0001005D
:102C400001008346390593E60602A309D9042380CF
:102C50000D00F646F3A606800100010095B3F33699
:102C6000048093F68608B6D20100010023809D00FF
:102C70002380CD00010001008346390593E606025A
:102C8000A309D90423800D009656F3A606800100FF
:102C9000010045BB9306F5FF33B5A600FD152E9543
:102CA0009355F501AE96B3B5B600AA951396F50106
:102CB000858269B5F336048093F68608B6D801009C
:102CC0000100930680FA23809D002380DD0001002F
:102CD00001008356C9020566011693F6F60FD18EE0
:102CE000C206C1822316D90223800D00C656F3A660
:102CF000068001000100850A93FAFA0F95B233E6C7
:102D0000B60045C20356C9023305D0403338A0008F
:102D1000B305B040B385054115826345B000D1E1EC
:102D20006371A608894663F0560593078008F3B7D8
:102D3000078093F78708BEDA01000100B71700404B
:102D4000130770052380E704130780FA2380E70444
:102D50000100010003D7C7027D8B2396E702238081
:102D60000704D65781BDF336048093F68608B6DC97
:102D700001000100930680FA23809D002380DD007E
:102D8000010001008356C9020566011693F6F60F8D
:102D9000D18EC206C1822316D90223800D00E656C9
:102DA000B9B793078008F3B7078093F78708BEDEAB
:102DB0000100010037170040930770052300F70456
:102DC000930780FA2300F704010001000356C702AD
:102DD00093975600B297C207C1832316F7022300C8
:102DE0000704F657C1BB914763EEB70217E701002E
:102DF000130747118A05BA959C41BA978287B7177E
:102E0000004003A7470B1345F5FF698F23AAE70A84
:102E100003A7070B698F23A8E70A03A7070A798D81
:102E200023A0A70A8280B717004083A6470B134749
:102E3000F5FFF98E23AAD70A83A6070B558D23A881
:102E4000A70A83A6070A758F23A0E70A8280B7170F
:102E5000004003A7470B498F23AAE70A03A7070BE4
:102E60001345F5FF45BFB717004083A6470B13472F
:102E7000F5FF758F23AAE70A03A7070A598D4DB7F7
:102E8000B717004003A7470B498FEDB7914763EE93
:102E9000B70217E70100130727088A05BA959C4176
:102EA000BA978287B717004003A7470D1345F5FF70
:102EB000698F23AAE70C03A7070D698F23A8E70CE6
:102EC00003A7070C798D23A0A70C8280B7170040B9
:102ED00083A6470D1347F5FFF98E23AAD70C83A6C7
:102EE000070D558D23A8A70C83A6070C758F23A06B
:102EF000E70C8280B717004003A7470D498F23AA2C
:102F0000E70C03A7070D1345F5FF45BFB7170040B2
:102F100083A6470D1347F5FF758F23AAE70C03A778
:102F2000070C598D4DB7B717004003A7470D498FC0
:102F3000EDB7797122D43714004026D24AD0035914
:102F400024028354040206D64209C2044ECE52CC57
:102F500056CA13590901C1802DE11379F9F793F489
:102F6000F49F4209C20413590901C18093078008E4
:102F7000F3B7078093F787083EC401000100930769
:102F800070052300F404930780FA2300F404010081
:102F90000100231124032310940223000404A247F8
:102FA000F3A7078001000100B25022549254025945
:102FB000F249624AD24A45618280B7F507008146EC
:102FC0003000B105194597000020E7808081A247B5
:102FD00013972701E34A07FC1369090893E40440A7
:102FE00093098008F3B7098093F787083EC0010072
:102FF0000100930A700523005405130A80FA230088
:10300000440501000100231124032310940223002E
:1030100004048247F3A7078001000100294597F0C7
:10302000FF1FE7802031F3B9098093F989084EC268
:1030300001000100230054052300440501000100A4
:103040008357040293E707202310F40223000404AB
:103050009247B9B7B7170040884742054181937737
:10306000050491EB9377F5013755E80113050580C9
:103070003345F50282809377050C130700046397AC
:10308000E7009377F50137459C1CCDB72165130503
:1030900005D0828037E700E01C435443A183E20659
:1030A000D58F1CC1FD572320F7182322F7188280E3
:1030B00013178500B7E700E023A0E710618123A282
:1030C000A7108280B7F700E08847CC47828081470D
:1030D00037370040A14663C4C7003285828003456C
:1030E000B740E38EA6FE3385F5000345050085074E
:1030F0002304A740CDB797070020938727EF9C4371
:1031000017370020130787343E95636EE5001737A5
:1031100000201307273F6368A70017070020232715
:10312000A7EC3E858280FD57EDBF8280411122C40D
:1031300006C62A8497000000E78000F22947B307FB
:10314000E502B2408D83B3D7870222449507B3D7F7
:10315000E70237370040C207C1832316F700410159
:103160008280411137150E0006C697000000E780E7
:1031700020FCB7370040130770F82381E7000D47A4
:10318000A381E70013070004A380E7000547238716
:10319000E700B24041018280373700408347270073
:1031A0001A0593F7F703C98F93F7F70F2301F70079
:1031B0008280B737004003C7170019C9D98DA38093
:1031C000B70003C70700136787002380E7008280EA
:1031D00093C5F5FFF98DA380B7008280AE872A875B
:1031E000B736004021463738004089E71703000012
:1031F0006700E3F383C8B600E30916FF05078348B9
:10320000F7FFFD17C20723041801C183F9BF41115D
:1032100022C406C62A8497000000E780E0E329471D
:10322000B307E502B2408D83B3D7870222449507E6
:10323000B3D7E70237370040C207C1832316F740F0
:1032400041018280716541111305052006C6970072
:103250000000E78000FCB7370040130770F82381B7
:10326000E7400D47A381E74013070004A380E74030
:1032700005472387E740B24041018280CC4141119C
:1032800006C6328503C6150083C5050022064D8E8D
:1032900042068D654186138875A2630C0611634B47
:1032A000C804138845A26300060D634AC8009385CD
:1032B00035A26301B6082390060029464DA0138865
:1032C00055A26305060D938565A2E316B6FE8D45EE
:1032D0001D4663E6E5081146198E63F3C7003E8676
:1032E000B7E704002390C600FC4797E501009385EB
:1032F000E5C49DA0138895A263030611634E060DD5
:103300001388A5A263000613938505A5E315B6FAF5
:1033100099451D4663E5E504198E63F3C7003E86B3
:10332000B7E704002390C600FC479705002093856B
:1033300025D61DA09D451D4663E3E5022146198E55
:1033400063F3C7003E86B7E70400FC472390C6003E
:103350009705002093858534BA9582970146B2403F
:10336000328541018280AD451D46E3EAE5FE3146E6
:10337000198E63F3C7003E86B7E704002390C600AA
:10338000FC4797E501009385E5BDF9B7B1451D46BA
:10339000E3E7E5FC3546198E63F3C7003E86B7E7E1
:1033A00004002390C600FC4797E50100938585BC87
:1033B00065B78D451D46E3E4E5FA1146198E63F3C2
:1033C000C7003E86B7E704002390C600FC4797E598
:1033D0000100938565B749B78D451D46E3E1E5F8E2
:1033E0001146198E63F3C7003E86B7E704002390A9
:1033F000C600FC4797E50100938585B9B1BFA54597
:103400001D46E3EEE5F42946198E63F3C7003E86B8
:10341000B7E704002390C600FC4797E501009385B9
:1034200065B31DBFB5451D46E3EBE5F23946198E80
:1034300063F3C7003E86B7E704002390C600FC474D
:1034400097E50100938585AE01BFB7E7040003A3AC
:103450000713970600209386A6C24146A545170587
:1034600000201305E5B802832D455DE703C505007F
:103470000947631FE50803A84500411106C6034735
:10348000180032850346080022074168518F9308CF
:1034900028FE6307170563E9E800051863030703BF
:1034A00023900600294591A8130648FE630AC70425
:1034B0001518E31707FF15463E87637BF60015478F
:1034C00001A8130600023E876374F600130700028A
:1034D000B7E704002390E600FC471316070111A884
:1034E0003E8691C30546B7E70400FC472390C6001B
:1034F0004206CC45418282970145B240410182801B
:10350000130600083E87E375F6FC13070008C9B7E9
:103510002390060005458280828041677917630405
:10352000E504411122C406C685472A84639FF5003D
:10353000B7E7040022852244B24003A3871397050E
:1035400000209385E52F4101028389476399F500A7
:10355000B7E7040083A7070B8545829771D9B2406E
:103560002244410182808280797126D252CCAE847D
:103570002A8A97E501009385A5A317E501001305A5
:10358000A5A506D63AC622D44AD0368432894ECE74
:1035900097C00100E7804044A28517E501001305AC
:1035A000A5A497C00100E7802043294597C00100EA
:1035B000E780604783C7840093F70702F9E383C974
:1035C00004008947054532476396F908D44083C70C
:1035D000160083C60600A207D58FC166138616FEA5
:1035E000638CC7028D16638FD7068D6693862690EF
:1035F00029456391D706B7E70400A286225403A3A6
:103600004714B250F2494A86A6850259925452850F
:10361000624A8547456102832D450DEF93070002FD
:10362000354563E98702B7E70400FC47C844130641
:103630000002CA8582978149970700209387072156
:103640009C43014581CB9C4391C74E852286CA8508
:1036500082970145B250225492540259F249624A6B
:10366000456182802D457DF79307700F3545E3E373
:1036700087FEB7E70400FC47C8442286CA858297C4
:1036800065BF2145C1BF411122C437E4040083272F
:10369000841326C2AA84416506C697050020938537
:1036A000251A7D1582978327C40A17050000130584
:1036B00005E78588829795C0032304132244B2400E
:1036C000924497060020938626AE4146C5451705CD
:1036D00000201305659C41010283B24022449244BC
:1036E00001454101828019C59707002023A0A71634
:1036F00001458280454582801147636AA70A97E6A3
:1037000001009386A6890A0536951841411106C61F
:103710003697AE87B2850287130700026145639D25
:10372000E700B7E70400FC47130600021705002076
:10373000130545F782970145B24041018280054754
:103740006145E39BE7FEB7E70400FC470546170524
:103750000020130525F7F9BF1307700F6145E39D9E
:10376000E7FCB7E70400FC471306700F17050020BD
:10377000130585F5C1B7130700086145E39EE7FA15
:10378000B7E70400FC4713060008170500201305DF
:1037900025034DB715476145E390E7FAB7E7040005
:1037A000FC471546170500201305C50961B70945F3
:1037B0008280411126C2B7E4040083A7C41322C447
:1037C0004AC006C62E8497050020938565072A897E
:1037D0008297058905C5970700209387E78B83D7D4
:1037E000A70BA28503A3440D2310F4002244B2408A
:1037F00092444A850249014641010283B240224473
:103800009244024949454101828097070020238163
:1038100007049707002023AF0702B717004003A74C
:10382000070CB706C0FFFD16758F23A0E70C03A792
:10383000070DB7064000558F23A8E70C03A7070C18
:103840003D9B23A0E70C03A7070D1367070123A8DF
:10385000E70C8280B717004003A5470C83A7470CED
:10386000598113451500C18B058999E3136525001E
:103870009707002083C7C7FD6380A7029707002032
:103880002388A7FC11C9970700209387A7FC03A3EF
:1038900007006303030002838280114517F3FFFFD3
:1038A000670063C8011122CC06CE3714004026CA37
:1038B0004AC84EC652C483447405034AB4058349BA
:1038C00084050349940597F0FFFFE780A0A0834794
:1038D000A40593F4F40F137AFA0F93E71700230D5E
:1038E000F40493F9F90F1379F90FB717004003C7E0
:1038F000A705058B6DFF03D5C705A38D4705238C51
:103900003705A38C2705A38B9704F2406244D24469
:103910004249B249224A05618280411193970501CB
:1039200022C406C626C2C1872E8463DC0700B7E422
:103930000400FC54829719C1BC5482972165218DE3
:1039400015A893F7150013C515008DE793F725000B
:103950009DC797000000E78020F0B7E70400BC4F48
:103960001306000A894517050020034525EF8297B5
:1039700013452400B240224492444101828093972F
:10398000250163D80702B7E4040083A7C41E829709
:1039900097000000E780A0F0BC4C375607001306E4
:1039A0000630896517050020034545EB82970965B8
:1039B00079B7939715010145E3DE07FA17D50100A2
:1039C0001305856A97C00100E780E018B7E7040097
:1039D000BC4F13060064916517050020034505E8F8
:1039E00082971165A9BF1D71A2CC37E404005C5C0D
:1039F000485886CE494697D50100938565628297DF
:103A000011E917D501001305E56297C00100E780B1
:103A1000801401A0B7F600E0795798CAFD57DCCAB8
:103A20000567B7E700E023A0E7101306F00290C295
:103A300023A0E718010001003707002018471306EC
:103A4000000481459706002023A8E6E04157A38A99
:103A5000E7403C4408088297970700209387877FB8
:103A60003EC8856713870740938757D1231AE10023
:103A70002312F1021307B00F97F7FFFF9387C76474
:103A80002310E1023ED81547970700009387C7E14E
:103A9000B7F50700A30FE1003EDC054797070000DC
:103AA0009387E7DF81463000E10519452301E102F4
:103AB0003EDE97F0FF1FE780C0D218088147994685
:103AC00030003E960346060085070507A30BC70096
:103AD000E398D7FEC24791C70357410185676373D7
:103AE000F70001A0B7E7040083A7470A08088297F8
:103AF000AA8511C917D501001305055597C0010006
:103B0000E78080ED01A0F640664425618280411186
:103B100026C2B7E4040083A7040806C622C417051A
:103B200000001305C5DF829717040020130404D397
:103B30002300A40097000000E780800297000000A7
:103B4000E780E0CC03450400224403A38405B2408F
:103B5000924413060032896541010283797106D6C9
:103B600022D413078008F337078093F787083EC2F3
:103B700001000100B7170040930570052380B704CA
:103B8000130680FA2380C7040100010083C6F702F0
:103B900093F6A60FA387D702238007049246F3A6C5
:103BA00006800100010073370780137787083AC445
:103BB000010001002380B7042380C7040100010035
:103BC00003C7F70213672700A387E70223800704D0
:103BD000A247F3A7078001000100054597E0FFFF1A
:103BE000E780807297000000E78060CB0147814644
:103BF0008147054685451305407E97E0FFFFE78036
:103C0000807537E404003C44680051468145829742
:103C1000B707C0A83EC8B787E803938707D03ECA56
:103C200097E7FF1F9387A7793EC67C586800829765
:103C3000B250225445618280411197E5010093857D
:103C4000A5A617D501001305253906C697C00100A2
:103C5000E78080D817E501001305C5BC97C00100B7
:103C6000E78080D7B2402945410117C301006700B2
:103C700083DB411197E50100938545A417D5010029
:103C80001305853506C697C00100E780E0D417E527
:103C900001001305E5B797C00100E780E0D3B2400B
:103CA0002945410117C301006700E3D7411122C430
:103CB00006C6834705002A849DC797E501009385C2
:103CC000A5A517D501001305253197C00100E78090
:103CD000A0D04C4017E501001305C5C997C00100ED
:103CE000E78080CF3DA058410DEF97E50100938517
:103CF000A5A217D501001305252E97C00100E78066
:103D0000A0CD17E50100130565C897C00100E78045
:103D1000A0CC2244B2402945410117C301006700ED
:103D200083D0A1679386D7036313D70297E5010079
:103D30009385859E17D501001305052A97C00100BC
:103D4000E78080C917E50100130545C57DBFED0774
:103D500097E501009385459C17D501001305C527FC
:103D6000631BF70097C00100E78000C717E501005B
:103D7000130505C459BF97C00100E780E0C54C405A
:103D800017E501001305C5C491BF411197E5010076
:103D90009385059417D501001305052406C697C021
:103DA0000100E78060C3B2402945410117C301000B
:103DB000670063C7397122DC26DA4AD82E842A8943
:103DC0008145B2844808714636C606DE97E0FFFF9B
:103DD000E780E03397F7FF1F9387075EDC4783D7C1
:103DE0000700231C2101231BF10097600000E780DE
:103DF00000DA9307800CB2463ECE03576101FD57AF
:103E00002302F102C167230DA100A30DD100FD170C
:103E10007D556309F7002686A28548089760000053
:103E2000E780C0D9F2506254D25442592161828055
:103E3000854617030000670023F8411197270020EB
:103E4000239D0790972700202386078006C6170723
:103E500000200347A7309307F00A6315F702930782
:103E6000F0F88945170500201305452F1707002096
:103E70002306F72E97070020A382072E97700000D5
:103E8000E780209297700000E780E0BE9770000006
:103E9000E78020C08145370504009707002023A54F
:103EA000072A97070020238F0728970700202393CE
:103EB000071E970700202391071C97070020239EC9
:103EC0000724970700202393072897400000E780E6
:103ED000E023014597700000E780A095D1471707C0
:103EE00000202310F726B7E70400BC4F1306001488
:103EF0008945170500200345E596829797D501006F
:103F00009385857F17D501001305050D97C0010026
:103F1000E78080AC9705002083D5A52217E5010036
:103F2000130545B197C00100E78000ABB2402945B9
:103F3000410117C30100670003AF4111814617F625
:103F4000FF1F1306A644854517050020035585125B
:103F500006C697D00000E780E01915C997D5010083
:103F60009385457A17D501001305050797C0010011
:103F7000E78080A617E501001305C59B97C00100E7
:103F8000E78080A5294597C00100E780C0A997D5A3
:103F900001009385257717D501001305E50397C028
:103FA0000100E78060A317E501001305E59997C0BC
:103FB0000100E78060A2294597C00100E780A0A624
:103FC00097F7FF1F9387473FDC47054797D50100C9
:103FD000938545732390E70017D501001305C5FFAE
:103FE00097C00100E780409F17E501001305059782
:103FF00097C00100E780409EB2402945410117C3A8
:104000000100670043A2411122C497D501009385A6
:10401000E5712A8417D50100130505FC06C697C073
:104020000100E780609B4C4017E501001305058EF9
:1040300097C00100E780409A294597C00100E780BA
:10404000809E034704009307F00F631FF70297D584
:1040500001009385A56D17D501001305E5F797C0FD
:104060000100E78060974C4017E501001305058BC0
:1040700097C00100E78040962244B24029454101A3
:1040800017C301006700239AB24022444101828095
:10409000411122C426C22A84AE8417D5010013051B
:1040A000A5F397D501009385256406C697C0010046
:1040B000E780809217E501001305459697C001003F
:1040C000E7808091294597C00100E780C09597D58A
:1040D00001009385656197070020239D87F817D518
:1040E0000100130565EF054497070020239297F818
:1040F00097070020239F87F697170020239F976438
:1041000097C00100E780408D9715002083D5E564B6
:1041100017E501001305059197C00100E780C08BEA
:10412000294597C00100E78000909717002023835E
:10413000875297F7FF1F93872728DC4717F5FF1F44
:104140000345457203D70700C167FD17631EF700DB
:10415000B7E7040003A387051306000A8545224438
:10416000B240924441010283B7E7040003A38705EC
:104170001306001493050010DDB7B1C1411122C42C
:1041800017D50100130545E52E8497D501009385C9
:10419000E55406C697C00100E7800084A28517E5B4
:1041A00001001305E58697C00100E780E082224404
:1041B000B2402945410117C301006700C3868280D0
:1041C000011122CC06CE26CA4AC84EC693F7150066
:1041D0002E84B5CB97000000E78060D6930710F8D7
:1041E00017070020230CF7F69707002083D747E82E
:1041F00017070020A304F7F69145A18317050020B7
:104200001305C5F517070020230BF7F497070020C7
:10421000A38707F497600000E780A058B7E7040081
:10422000BC4F130600149305001017F5FF1F03453C
:104230006563829713451400F2406244D2444249B8
:10424000B2490561828093F7052081CB9707002052
:10425000238607EC13C50520C5B793F705408DC726
:104260009705002083D5C5ED89CD170500201305DE
:1042700025EB97F0FFFFE780A0F69707002023913A
:1042800007EC134504404DBF93F70510B1C3054536
:1042900097600000E780E059171500200355E54BB3
:1042A00097600000E780602597200000E7802044A9
:1042B0009707002083C7D7F989E797600000E78058
:1042C000807B97600000E780C07C13450410ADB789
:1042D00093F72500E9CF17070020035787E669C742
:1042E000AD64B71900409384A4AA23A0990097064F
:1042F0000020938666E5944297D70100938747751F
:1043000017060020034606E4814517D50100130572
:10431000257597800000E780A0F923A0990097F702
:10432000FF1F239FA7F82A8941C197D501009385D4
:10433000254417D50100130525CA97B00100E78071
:10434000A069CA8517D50100130585E297B0010061
:10435000E7808068294597B00100E780C06C970727
:104360000020239007DE930710F81707002023078B
:10437000F7DE9707002083D7A7CF17070020A30FEA
:10438000F7DCA18317070020230BF7DC91458D474D
:1043900017050020130585DC17070020A301F7DCB3
:1043A00097600000E780E03F1345240071B593F764
:1043B0004500D1C397D501009385853B17D50100F2
:1043C000130585C197B00100E780006117D5010092
:1043D0001305C5DB97B00100E7800060294597B061
:1043E0000100E7804064930720F8170700202307A7
:1043F000F7D69707002083D7E7C917070020A30F38
:10440000F7D4A18317070020230BF7D4854717079C
:104410000020A306F7D497600000E780408E1705C0
:1044200000201305A5D3914597600000E780603711
:104430001345440011B593F78500A9C797D501002E
:104440009385053317D50100130505B997B0010011
:10445000E780805817D50100130585D497B0010077
:10446000E7808057294597B00100E780C05B970738
:104470000020239807CC97800000E78040F3134585
:1044800084005DBB93F70501D1C385451705002066
:10449000035545C097700100E78000A997D501003A
:1044A0009385052D17D50100130505B397B00100BD
:1044B000E780805217D501001305C5CF97B00100E2
:1044C000E7808051294597B00100E780C0559307E8
:1044D00030F8170700202303F7C89707002083D779
:1044E00067BB17070020A30BF7C6170500201305AD
:1044F000E5C6A1838D45170700202302F7C6976004
:104500000000E780002A134504013DB393F705023C
:10451000D1C797D501009385A52517D501001305AF
:10452000A5AB97B00100E780204B17D5010013051C
:10453000A5CA97B00100E780204A294597B001003D
:10454000E780604E930740F8170700202308F7C064
:104550009707002083D747B217070020A300F7C0B2
:10456000A18317070020230CF7BE854717070020FB
:10457000A307F7BE97070020239007B097500000CD
:10458000E780E07717050020130545BD914597604A
:104590000000E78000211345040279B993F7050470
:1045A000FDC397D501009385A51C17D50100130500
:1045B000A5A297B00100E780204217D5010013059E
:1045C00025C397B00100E7802041294597B001003D
:1045D000E78060459707002083C747B81307700A34
:1045E0006386E7061307800A638CE7081307600AEF
:1045F0006393E704930760F8170700202300F7B6DA
:104600009707002083D767B117070020A308F7B4E6
:10461000A183170700202304F7B48547170700205C
:10462000A303F7B4B14517050020130525B3976020
:104630000000E780001797500000E780406C1345AA
:10464000040497070020239A07ACFDB6930770F87F
:10465000170700202304F7B09707002083D7E7ABA4
:1046600017070020A30CF7AEA1831707002023082B
:10467000F7AE854717070020A304F7AE994565B745
:10468000930780F8F1B793F705080145E38607BA69
:1046900097D501009385C50D17D501001305C59366
:1046A00097B00100E780403317D501001305C5B569
:1046B00097B00100E7804032294597B00100E780BC
:1046C00080369307A0F8170700202309F7A897075B
:1046D000002083D7A7A717070020A301F7A8A1836D
:1046E00017070020230DF7A6854717070020A3080A
:1046F000F7A697070020239B07A497500000E780A8
:10470000006017050020130565A59145976000001E
:10471000E78020091345040805B6011122CC37E4CF
:1047200004005C5C06CE26CA354697D50100938509
:10473000A51017E501001305A516829711E917D5F5
:1047400001001305258F97B00100E780C04001A04C
:1047500097F7FF1F9387C7113EC4B7F5070085671A
:1047600093870780814617F6FF1F1306E60FE105C2
:1047700019453EC697E0FF1FE780A0067C44194616
:1047800097F5FF1F9385450E170500201305C5906B
:104790008297340017F6FF1F1306060D97D5010008
:1047A0009385455417D501001305455597800000A2
:1047B000E7800085AA8421C197D50100938545FA39
:1047C00017D501001305458197B00100E780C0208F
:1047D000A68517D501001305250797B00100E780CE
:1047E000A01F294597B00100E780E023F240624412
:1047F000D2440561828097F00000E780E0EA17D597
:104800000100130565FB97600000E780207997B0F1
:104810000000E780203F97700100E780A0A317F514
:10482000FF1F1305E5B597700100E780408C17D591
:104830000100130565F997700100E78020A4AA84A0
:1048400097700000E78060DF97100100E780807BB1
:1048500097900100E780A01497800000E780403B1C
:1048600097700000E780605597400100E780E03CCA
:1048700097D501009385C5EE17C501001305C575D1
:1048800099C897B00100E7802015A68517D50100CB
:104890001305C5FD99B797B00100E780E01317D560
:1048A00001001305E5FE97B00100E780E0122945FD
:1048B00097B00100E780201797400100E780C018FB
:1048C00097000100E78080376DC5854537050400F6
:1048D00097400000E780808397D50100938545E8E5
:1048E00017C501001305456F97B00100E780C00EA2
:1048F00017D50100130545FB97B00100E780C00DF7
:10490000294597B00100E780001297F7FF1F9387B2
:10491000279A83D70700171700202310F7E485474D
:10492000171700202308F7D297F7FF1F9387C7A810
:10493000DC4703D70700C167FD176316F70097F040
:10494000FFFFE780C05F97800000E78080B6856743
:10495000938707E33E9597800000E78040B6972055
:104960000000E780C0D817150020035505DF9760C9
:104970000000E78080B8054597600000E78060EBA5
:1049800097600000E780E01097D50100938545DD32
:1049900017C501001305456497B00100E780C00307
:1049A00017D50100130545F597B00100E780C00257
:1049B0000DBDD14797D50100938585DA17C5010054
:1049C0001305856117F7FF1F231DF77697B00100C8
:1049D000E780800017D601001306865097F5FF1F69
:1049E00083D5257617D50100130545EE97B0010054
:1049F000E78080FE294597B00100E780C0023C4C6B
:104A00001306000A894517F5FF1F0345A5E58297A0
:104A1000014597600000E780C0E1BDB7411122C4A5
:104A200037E404008327041A06C6829797600000C3
:104A3000E78060B08327040817F5FFFF130585782A
:104A4000829797F7FF1F238FA7E017F5FF1F130526
:104A5000A59697500000E78040612244B240410192
:104A6000170300006700A3CBB7E70400FC471171F0
:104A7000A2DDCAD986DFA6DBCED72E8432892E8668
:104A8000AA8517F5FF1F1305656D829717F7FF1F9E
:104A90001307C76C834707009306F0029387E70765
:104AA00093F7F70FE3ECF610BA898A0717C70100EE
:104AB0001307C75BBA979C43BA9782878D4797D5F0
:104AC0000100938525CC17C501001305E550630F40
:104AD000F40097B00100E78020F017D5010013051E
:104AE000258997B00100E78020EFBDA497B00100B1
:104AF000E78080EE17D501001305058997B0010006
:104B0000E78080ED294597B00100E780C0F1930769
:104B100020F8114697F5FF1F938545644A8517F7DE
:104B2000FF1F230DF76297F7FF1FA38A076297F015
:104B3000FFFFE78020302A841DC997D501009385A7
:104B400065C417C501001305254997B00100E7802A
:104B5000A0E8A28517D501001305C58697B001000E
:104B6000E78080E7294597B00100E780C0EB97D543
:104B70000100938525C117C501001305E54597B0D0
:104B80000100E78060E517D501001305E58497B0C3
:104B90000100E78060E4294597B00100E780A0E8C4
:104BA0004165930730FA054697F5FF1F9385055B2E
:104BB0007D1517F7FF1F2303F75A97F0FFFFE780D4
:104BC00060272A841DC997D501009385A5BB17C509
:104BD00001001305654097B00100E780E0DFA28582
:104BE00017C501001305057E97B00100E780C0DE00
:104BF000294597B00100E78000E3B7E70400BC4F08
:104C00000566130606C8A14517F5FF1F034585C5B0
:104C10008297FE506E54DE544E59BE591161828007
:104C200091476303F40297D501009385A5B517C595
:104C300001001305653A97B00100E780E0D917C578
:104C400001001305A57C71BDB7E70400FC4F914539
:104C500017F5FF1F034505C1829797D5010093857E
:104C600065B217C501001305253797B00100E7802D
:104C7000A0D617C501001305257B97B00100E7807A
:104C8000A0D5294597B00100E780E0D997500000F2
:104C9000E780E006914535A485476303F40297D584
:104CA0000100938525AE17C501001305E53297B0C5
:104CB0000100E78060D217C501001305657815B5BE
:104CC00097F7FF1F2398273DB7E704000566BC4F01
:104CD000130606C8C1450DBF8D476303F40297D57F
:104CE0000100938525AA17C501001305E52E97B08D
:104CF0000100E78060CE17C5010013052576D5B306
:104D0000930740F8114697F5FF1F938525454A857F
:104D100017F7FF1F2304F74497F7FF1FA3810744EA
:104D200097F0FFFFE78000112A84E30405EE97D592
:104D30000100938525A517C501001305E52997B046
:104D40000100E78060C9A28517C5010013058567CA
:104D500097B00100E78040C8294597B00100E7807F
:104D600080CC45BD9147E31CF4F6B7E70400FC4F47
:104D70009305000217F5FF1F0345C5AE829797D52F
:104D80000100938525A017C501001305E52497B000
:104D90000100E78060C417C501001305A56DF1BDD2
:104DA000894763E3870297D501009385A59D17C5C1
:104DB00001001305652297B00100E780E0C117C527
:104DC00001001305656C31BB97F4FF1F83C42439C0
:104DD00097F7FF1F83C7973897D501009385859A6A
:104DE000A20417C501001305251FDD8C97B0010033
:104DF000E78080BEA28517C501001305256A97B01C
:104E00000100E78060BDC204294597B00100E7803A
:104E100080C1C1849305D4FF93960401C1824A8660
:104E200093F5F50F17F5FF1F130575339730000045
:104E3000E7808031E35F90DC930750F817F7FF1F9E
:104E4000230EF73083C73900228697F5FF1F93851D
:104E5000E53085074A8517F7FF1FA302F73097F063
:104E6000FFFFE78020FD2A84E30505DA97D50100DE
:104E70009385459117C501001305051697B00100EC
:104E8000E78080B5A28517D50100130565B7C9B5C0
:104E9000894763E3870297D501009385A58E17C5DF
:104EA00001001305651397B00100E780E0B217C554
:104EB00001001305656035B197500000E78020E4DC
:104EC000A28517F5FF1F1305652997600000E7808D
:104ED000408D81B38D476303F40297D5010093851C
:104EE000658A17C501001305250F97B00100E780FB
:104EF000A0AE17C501001305E55DE5B6B766020073
:104F00000146B7750200054597E0FF1FE780608DF9
:104F1000930760F817F7FF1F2302F72497F7FF1F87
:104F2000A38F07229307000617F7FF1F230AF72214
:104F3000894717F7FF1FA305F72297F7FF1F238263
:104F4000072297F7FF1FA38E0720C14717F7FF1F00
:104F5000230AF720930720F917F7FF1FA304F72070
:104F6000314697F7FF1FA380A72097F5FF1F938572
:104F7000E51E4A8597F7FF1F2387071E97F0FFFF5F
:104F8000E78040EB2A84E30605C897C501009385B6
:104F9000657F17C501001305250497B00100E78060
:104FA000A0A3A28517C501001305455455B3B14709
:104FB0006303F40297C501009385C57C17C5010002
:104FC0001305850197B00100E78000A117C5010016
:104FD0001305855339B6B7E70400FC4F9305000469
:104FE00017F5FF1F03450588829797500000E7805B
:104FF00000D1B145F9B5914763E3870297C5010038
:105000009385457817C50100130505FD97B001008C
:10501000E780809C17C501001305C550D9B497F4EB
:10502000FF1F83C4E41397F7FF1F83C75713A2041E
:10503000DD8C8E04B77702006D14BE942286A6859F
:1050400017C501001305454F97B00100E780C098D0
:10505000B7E70400FC47228697F5FF1F938555109C
:105060002800829793160401C1823000A685094565
:1050700097D0FF1FE780E0762A8409C917C5010091
:105080001305454D97B00100E780E0AC930770F839
:10509000194697F5FF1F9385650C4A8517F7FF1F83
:1050A000230EF70A97F7FF1FA38C870A97F0FFFFDD
:1050B000E78040D82A84E30E05B497C501009385A4
:1050C000656C17C50100130525F197B00100E78055
:1050D000A090A28517C501001305C54895B9994749
:1050E000630BF41297C501009385C56917C50100CC
:1050F000130585EE97B00100E780008E17C501000B
:105100001305C547F9BA914763E3870297C50100C4
:105110009385456717C50100130505EC97B001009D
:10512000E780808B17C501001305C5465DBA97F46B
:10513000FF1F83C4E40297F7FF1F83C75702A2042F
:10514000DD8C8E04B77702006D14BE942286A6858E
:1051500017C501001305454597B00100E780C087DA
:10516000B7E70400FC47228697F5FF1F938555FF9C
:105170002800829793160401C1823000A6850D4550
:1051800097D0FF1FE780E0652A8409C917C5010091
:105190001305454397B00100E780E09B930780F833
:1051A000194697F5FF1F938565FB4A8517F7FF1F83
:1051B0002306F7FA97F7FF1FA38487FA97F0FFFFFC
:1051C000E78040C72A84E30605A497C501009385BC
:1051D000655B17C50100130525E097A00100E78076
:1051E000A07FA28517C501001305053F95B6994715
:1051F0006303F40297C501009385C55817C50100E4
:10520000130585DD97A00100E780007D17C501002B
:105210001305053EF9B0B7E70400FC4F9305000401
:1052200017E5FF1F03450564829797500000E7804C
:1052300000AD994579B18D476303F40297C501002C
:105240009385455417C50100130505D997A00100A2
:10525000E780807817C501001305053B59B017C5D5
:1052600001001305653B97B00100E780C08E130570
:10527000C01297D0FF1FE780C00C014597E0FFFFE9
:10528000E78080E10D4597100000E78000C12945C7
:1052900097D0FF1FE780E00A97D0FF1FE78040FB11
:1052A0008DBA99476303F40297C501009385854D34
:1052B00017C50100130545D297A00100E780C07112
:1052C00017C501001305053629B817F7FF1F034757
:1052D00037E997F7FF1F83C7A7E822075D8F91661D
:1052E000BA96C2061166C1821306F6EF8D47636552
:1052F000D60297E7FF1F9387270C9C4B17F6FF1FDB
:105300000346F6E59386C7002DC203D6070069CA97
:105310008907E39CD7FE89471307A0F8114697F544
:10532000FF1F9385A5E34A8597F6FF1F2388E6E2D2
:1053300017F7FF1FA305F7E297F0FFFFE78080AFA5
:105340002A84E308058C97C501009385A54317C5FA
:105350000100130565C897A00100E780E067A285FA
:1053600017C501001305452DE5B203D60700630EEE
:10537000E60A8907E39BF6FE8D4779BF91476304F0
:10538000F40297C501009385E53F17C50100130599
:10539000A5C497A00100E780206417C5010013058C
:1053A000252B6FF00FF4B7E70400FC4F93050008BE
:1053B00017E5FF1F0345054B8297C9B897C5010044
:1053C0009385453C17C50100130505C197A0010051
:1053D000E780806017C50100130505296FF06FF0A5
:1053E0002390E70017E5FF1F130505FD9740010017
:1053F000E780008B97C501009385C53817C501006C
:10540000130585BD97A00100E780005D17C5010069
:105410001305852697A00100E780005C294597A029
:105420000100E78040608147C5BD2390070017E574
:10543000FF1F130565F897400100E780608697C558
:1054400001009385253417C501001305E5B897A021
:105450000100E780605817C50100130565235DBF93
:1054600041114AC006C622C426C2834705002A89C4
:1054700085CB97C501009385A52C17C501001305A1
:10548000A5B597A00100E78020558325490017C5E1
:1054900001001305E55D97A00100E780E0539DA49E
:1054A0005841B707CF009387777D631BF72083545C
:1054B000C500054700450359E5008147637897001B
:1054C0008347040003471400A207D98F17F7FF1F73
:1054D000035767BE050797F6FF1F239EE6BC17F725
:1054E000FF1F231727BD17F7FF1F231197BC014785
:1054F00099C00347040097F6FF1F238AE6BA316775
:105500001307C755639BE70297F7FF1F83D767BA57
:10551000850717F7FF1F231EF7B897F7FF1F23967E
:1055200097B8034604008546A6854A859720000063
:10553000E780A069A6852285DDA0034604009307C5
:10554000100B6317F60E854763FB97128946130607
:10555000100BA6854A8597200000E7800067B947B1
:1055600063F9970A83471400130730056393E70A2A
:105570008346240013075004639DE60883463400E5
:10558000130710046397E608034744006313F70802
:10559000034754009307B004631DF70603476400F4
:1055A000930790056317F7068347740013070002FB
:1055B0006391E7060347840093063004631BD70416
:1055C00003469400930640046315D6048346A40062
:1055D0006391E6040347B400631DF7020347C40068
:1055E000930780046317F7020347D4009307F0047E
:1055F0006311F7020347E40093070005631BF700FC
:1056000097F7FF1F83D707AB850717F7FF1F2313F4
:10561000F7AA9385F4FFC205C18113051400224443
:10562000B2409244024941011723000067006370B1
:10563000954763F69704930730056314F604034710
:10564000140093075004631EF702034724009307D6
:1056500010046318F702834734006394C7020347BA
:1056600044009307B004631EF700034754009307F8
:1056700090056318F7008D461306300575B591E067
:1056800001469146A6854A8597200000E780E053B1
:105690009707002083D7670C63882701A68522859A
:1056A00097E0FFFFE780C0B322852244B2404A86DC
:1056B000A68502499244410117F3FFFF6700033BAF
:1056C000B707CC009387777D6318F70497C501006F
:1056D0009385050717C501001305059097A00100E4
:1056E000E780802F832789008356E9008355C9000E
:1056F00003C6070017C501001305053997A001006F
:10570000E780802D2244B24092440249294541015C
:1057100017A3010067002331B707CE009387777D79
:105720006305F70297C501009385850117C5010040
:105730001305858A97A00100E780002A8325490088
:1057400017C501001305C528B9B3B24022449244DD
:10575000024941018280B7E70400FC4741112E86CF
:1057600006C622C426C24AC02E842A89AA8517F5F5
:10577000FF1F1305A59E829797C5010093854502DB
:1057800017C501001305458597A00100E780C024D7
:1057900097F5FF1F83C5859C17C50100130545A814
:1057A00097A00100E7804023294597A00100E780EA
:1057B000802797F4FF1F9384649A83C704004147AE
:1057C0009387070693F7F70F6369F75A17C7010026
:1057D0001307C7958A07BA979C43BA9782879D4754
:1057E0006307F40297C50100938585FB17B5010097
:1057F0001305857E97A00100E780001E17C50100F4
:10580000130585A297A00100E780001DA1AC97F7C2
:10581000FF1F83C7B794DDCB17F7FF1F03473794EC
:1058200097F7FF1F83C7A79322075D8F97F7FF1F87
:1058300083C70793C2075D8F97F7FF1F83C75792F0
:10584000E207D98F17F7FF1F2320F79083C7640063
:1058500097C501009385C5F417B501001305C577F9
:1058600017F7FF1F2300F78E97A00100E780C016EF
:1058700097F7FF1F9387478D8C4317F6FF1F03464B
:10588000668C17C501001305E59B97A00100E78012
:10589000A014294597A00100E780E01897F7FF1FA3
:1058A000A38E078A2244B24092440249930700F82B
:1058B00017F7FF1F2304F78A9D4517F5FF1F1305F0
:1058C000E5894101175300006700A3ED97700000C0
:1058D000E78060BD97F7FF1F2383A7889357850054
:1058E00017F7FF1FA30DF786935705012A8417F7B3
:1058F000FF1F2307F78693578501014517F7FF1F01
:10590000A300F78697700000E78040BE97F7FF1F5F
:105910002389A78497C50100938585E817B5010001
:105920001305856B97A00100E780000B17F6FF1F9A
:1059300003462683A28517C5010013052592B1B73A
:10594000CD476303F40297C50100938565E517B55C
:1059500001001305656897A00100E780E00717C5FF
:1059600001001305259179BD97F7FF1F83C7278095
:10597000A20717E7FF1F0347777FD98FC207C187A9
:105980006357F00217E7FF1F231DF77AB7E70400FC
:1059900003A387051306000A89452244B2409244B6
:1059A000024917E5FF1F0345E5EB41010283D1479B
:1059B000D1BF8D476303F40297C50100938545DE8F
:1059C00017B501001305456197A00100E780C000ED
:1059D00017C501001305C59935B517E4FF1F03442A
:1059E000047897E7FF1F83C7777797C501009385F2
:1059F00025DB220417B501001305055E5D8C97A019
:105A00000100E78060FDA28517C501001305058828
:105A100097A00100E78040FC294597A00100E7809E
:105A200080000D4697E5FF1F93854573228597E01B
:105A3000FFFFE7802040AA8421C197C5010093851C
:105A400025D617B501001305255997A00100E78059
:105A5000A0F8A68517C501001305858497A001004D
:105A6000E78080F72244B24092440249294541012F
:105A700017A30100670023FB97E7FF1F239C8760A4
:105A8000B7E70400116603A38705130606E89145EE
:105A900029B78D476303F40297C50100938545D06C
:105AA00017B501001305455397A00100E780C0F228
:105AB00017C501001305859AB1B317E4FF1F03440E
:105AC000046A97E7FF1F83C7776997C5010093852D
:105AD00025CD220417B50100130505505D8C97A054
:105AE0000100E78060EFA28517B501001305857CF2
:105AF00097A00100E78040EE294597A00100E780CC
:105B000080F20D4697E5FF1F93854565228597E056
:105B1000FFFFE7802032AA841DC197C5010093854D
:105B200025C817B501001305254B97A00100E78094
:105B3000A0EAA68517B501001305057905B797E713
:105B4000FF1F239B8752B7E70400116603A3870555
:105B5000130606E89305000289B5894763E38702C7
:105B600097C501009385C5C317B501001305C54648
:105B700097A00100E78040E617C501001305C59016
:105B800051B197E4FF1F83C4845D97E7FF1F83C76C
:105B9000F75C97C501009385A5C0A20417B5010065
:105BA00013058543DD8C97A00100E780E0E2A68520
:105BB00017B501001305C57297A00100E780C0E189
:105BC000294597A00100E78000E6228697E5FF1FA0
:105BD0009385C558268597E0FFFFE780A0252A8496
:105BE000630E051A97C50100938585BB17B50100A3
:105BF0001305853E97A00100E78000DEA28517B55A
:105C000001001305256F99BD854763F98718834502
:105C100019002244B24092440249B335B00097E7DC
:105C2000FF1F2383B74817B501001305E56D410138
:105C300017A30100670043DAA2852244B2409244D0
:105C40004A8502494101170300006700432B994729
:105C50006303F40297C50100938585B417B501006D
:105C60001305853797A00100E78000D717C501000D
:105C70001305459B41BE17E4FF1F0344444E97E7BD
:105C8000FF1F83C7B74D97C50100938565B12204F7
:105C900017B50100130545345D8C97A00100E7801E
:105CA000A0D3A28517B501001305856797A0010051
:105CB000E78080D2294597A00100E780C0D6194629
:105CC00097E5FF1F93858549228597E0FFFFE780D1
:105CD0006016AA841DC197C50100938565AC17B5F0
:105CE00001001305652F97A00100E780E0CEA6858F
:105CF00017B501001305C56395B397E7FF1F2397F9
:105D00008744B7E70400116603A38705130606E876
:105D10009305000859B1854797C50100938545A8AB
:105D200017B501001305452B630BF40097A0010084
:105D3000E78080CA17B501001305C560E1B497A0DC
:105D40000100E78060C917B501001305256197A020
:105D50000100E78060C8294597A00100E780A0CC3A
:105D60002244B2409244024997E7FF1F239B073C1D
:105D70004101176300006700836397C501009385A5
:105D800025A217B501001305252597A00100E7807E
:105D9000A0C417C501001305258DADB4B24022443F
:105DA0009244024941018280411106C622C426C2A2
:105DB00039C12A8497F00000E78040E8AA8411EDF9
:105DC000B7E70400BC474146814522858297B2402F
:105DD0002244268592444101828041657D1597F0D9
:105DE0000000E78080E6B7E7040001E9BC474146D0
:105DF0008145228582978144D9BF0347E501FC474D
:105E00009305900819E393050003AA95414622855E
:105E1000829785446DBFB5CD7971930710FB23023E
:105E2000F10006D68147F1463387F50003070700E6
:105E300013960701418209C78507639DD7026D4606
:105E400005064206914641824C0097E0FFFFE7803D
:105E5000A0F615C597E7FF1F83D70726850717E725
:105E6000FF1F231BF72497E7FF1F2398A724B25097
:105E70004561828050003E962300E60075B797E7A3
:105E8000FF1F83D7A723850717E7FF1F2318F722D4
:105E9000F9BF7D558280411122C491462A8417E6BC
:105EA000FF1F1306A6399D652D4506C697D0FF1F17
:105EB000E7802093B7F7070003C70701A5476313DF
:105EC000F70001A09306001001469D65254597D077
:105ED000FF1FE780009197E7FF1F23818736224449
:105EE000B240914617E6FF1F130646359D652945CA
:105EF000410117D3FF1F6700C38E1171CED7B7E9D9
:105F0000040083A7C904CAD917E9FF1F130909258B
:105F1000A2DD2E8686DFA6DB2E84AA854A8582979F
:105F200097E7FF1F83C787231307700A6385E7106E
:105F3000636DF7001307600A6385E704FE506E5433
:105F4000DE544E59BE59116182801307800A638561
:105F5000E7161307900AE393E7FE8D476306F41CE8
:105F600097C501009385C5BD17B501001305C5068A
:105F700097A00100E78040A617C50100130585B969
:105F800025A08D47630CF40297C50100938545BB9E
:105F900017B501001305450497A00100E780C0A3D1
:105FA00017C50100130545B097A00100E780C0A206
:105FB000294597A00100E78000A749B7854717C585
:105FC0000100130525B017E7FF1F230FF70C97A05B
:105FD0000100E78040B8B7750200B76602000146CD
:105FE000054597C0FF1FE780C07F930760F817E75C
:105FF000FF1F2305F71697E7FF1FA38207169307D6
:10600000002617E7FF1F232DF714E5779387072155
:1060100017E7FF1F2318F714B14597E7FF1F2384E5
:10602000071497E7FF1FA380A7144A859700000075
:10603000E780E01621B7914763E3870297C5010027
:10604000938505B017B50100130505F997A0010068
:10605000E780809817C501001305C5A8B1B797E47C
:10606000FF1F83C4E40F97E7FF1F83C7570FA204E6
:10607000DD8C83A7C9046D14228697E5FF1F9385E5
:10608000350E280082978E0493160401B77502001E
:10609000C1823000A695094597C0FF1FE780607454
:1060A000930770F817E7FF1F230AF70A994597E748
:1060B000FF1FA387A70A95BF914763E3870297C590
:1060C00001009385E5A717B501001305E5F097A03A
:1060D0000100E780609017C50100130525A2E9B50E
:1060E00097E4FF1F83C4C40797E7FF1F83C73707E1
:1060F000A204DD8C83A7C9046D14228697E5FF1FD7
:1061000093851506280082978E0493160401B775AF
:106110000200C1823000A6950D4597C0FF1FE780A1
:10612000406C930780F8BDBF17C501001305C59FDC
:1061300097A00100E78020A2930790F82304F100C4
:10614000834719008D452800A304F10083472900E7
:106150002305F10097000000E78060041305C012DA
:1061600097C0FF1FE780E01D014597D0FFFFE78044
:10617000A0F20D4597000000E78020D2294597C086
:10618000FF1FE780001C97C0FF1FE780600C7DB3F6
:1061900097E7FF1F23ACA70A828097E7FF1F93872B
:1061A000E70A03A307006303030002831743000009
:1061B0006700235F41114AC097F6FF1F83D6E65957
:1061C000328917D6FF1F0356462122C426C206C6AF
:1061D0002A84AE8497000000E780A06629C921C800
:1061E000994763F697048347140003470400A20706
:1061F000D98F13978700A183D98FC2073167C183D5
:106200001307C7556395E70297D7FF1F83D7E71C8E
:10621000A301F400A1832302F40097F7FF1F83D7A3
:10622000C75391C7A302F400A1832303F400630DB5
:10623000090297F7FF1F83C7E7419DE797E7FF1F15
:1062400083C7070195C38DC097E7FF1F83C7C7E5C5
:1062500081EF22852244B2400249A6859244410141
:10626000174300006700E353B240224492440249BE
:1062700041018280834755008345450017C50100D1
:106280001305C58EA207DD8D179301006700C37447
:1062900017C501001305858C17A301006700A38BA8
:1062A0008D4763F6B708011126CA06CE22CC0344F7
:1062B000350097E4FF1F83C4B4F997C501009385A7
:1062C000258CB337800017E7FF1FA303F7F809C435
:1062D00097C501009385858B17C501001305858B34
:1062E00097900100E780406F97E7FF1F83C757F63D
:1062F0006386970097000000E78080439740000086
:10630000E78020799967938757EE2316F10068009C
:1063100085479145A30781002307F10097000000FE
:10632000E780E0E7F2406244D244056182808280E7
:10633000894763F7B708011122CC06CE26CA8344E9
:10634000250085472A84639DF404914763F5B704CB
:10635000034545008347340022055D8D97D7FF1F15
:10636000239DA70697000000E780805699679387D2
:1063700067EE2314F1008347340023059100A30541
:10638000F10083474400954528002306F10097005B
:106390000000E780C0E0F2406244D24405618280A0
:1063A000FDF89967938767EE2314F10097D7FF1FD5
:1063B00083D7A702A305F10023050100A183E1B75C
:1063C00082800111996722CCD51717F4FF1F13049F
:1063D00064282314F1008347040026CA97F4FF1FA2
:1063E0009384A4372305F10083D704002800954542
:1063F000A305F100A18306CE2306F100970000005B
:10640000E780E0D903D604008345040017B50100F6
:106410001305457997900100E780005CF2406244E3
:10642000D244056182809D677971D9172316F100E6
:1064300097F7FF1F9387072283C707001305F10013
:1064400006D62307F10097000000E780209609E9AF
:10645000B7E70400BC47414681451305F100829728
:106460006800CD4597000000E78060D397F5FF1FD7
:1064700083C5451E17B501001305C575979001002A
:10648000E7808055B25045618280630C051601118A
:1064900026CA06CE22CC4AC84EC697E7FF1F83C73E
:1064A00037DB97F4FF1F83C4E41A99C393E42400F5
:1064B0002A8497100000E780A07093E9C40119E1D5
:1064C00093E9C40037E90400832789042285130671
:1064D000200381458297930750FA2300F400930725
:1064E000A005A300F4008D472301F4009147A30108
:1064F000F40093071005A302F40097F7FF1F83D75A
:10650000C7252304F400A183A304F40097D7FF1F39
:1065100083D7A7EC2305F4009304C400A1832302CE
:10652000040023033401A305F4002685970000002E
:10653000E780C08719E58327890441468145268580
:10654000829797D7FF1F83D7E7E6230EF400A18336
:10655000A30EF40093070002230FF400930710FA30
:10656000A30FF4009D472300F402A3000402B7E741
:106570000400FC4713052402194697D5FF1F938595
:10658000A52E829797E7FF1F83D747B32304F40212
:10659000A183A304F40297E7FF1F83D7E7B1230584
:1065A000F402A183A305F40297E7FF1F9387E7B0E6
:1065B000839707002285930500032306F402C20790
:1065C000C183A183A306F40297D7FF1F938747CF08
:1065D000839707002307F402C207C183A183A3079F
:1065E000F40297000000E780C0212308A402218163
:1065F000A308A402F2406244D2444249B249056170
:10660000828082805D71E17793C777FF1305E10097
:1066100086C62316F10097000000E78040E7680077
:106620009305400397000000E78060B7B6406161C2
:1066300082805DC9411122C426C206C6930750FA62
:106640002300F5009307A005A300F5008947230167
:10665000F5009147A301F50093071005A302F5008B
:1066600097F7FF1F938707FF83C707009304C500B1
:106670002A842303F50097E7FF1F938777BD83C71D
:10668000070023020500A303F50097F7FF1F83D738
:10669000C70C2304F500A183A304F50097D7FF1FBF
:1066A00083D7A7D32305F500A183A305F50026858D
:1066B00097F0FFFFE780806F01E9B7E70400BC4770
:1066C00041468145268582972285F1459700000045
:1066D000E7802013230EA4002181A30EA400B24062
:1066E000224492444101828082805D710A8586C67F
:1066F000A2C497000000E78000F437E404007C4463
:106700008A850810794682973C441305E1030946BF
:1067100081458297101093050002014597D0FFFF35
:10672000E780C0FDB6402644616182800111B7C791
:10673000A55A22CC9387C73317E4FF1F130454B123
:106740003EC483470400856601469965254506CE0B
:106750003EC697C0FF1FE780C0083000A14699657C
:10676000294597C0FF1FE780C0078345040017B580
:1067700001001305A55097900100E780E025F24045
:106780006244056182800111A146300099652D4562
:1067900022CC06CE97C0FF1FE780A004A24737C4D3
:1067A000A55A1304C43363958702B24517B5010097
:1067B00013058544B335B00097E7FF1FA38AB7A838
:1067C00097900100E7804021F24062440561828099
:1067D0009165A1463000938505F02D4597C0FF1FB8
:1067E000E7802000A247E38287FC97E7FF1FA38191
:1067F00007A6814517B5010013054542D1B7C1670A
:1068000069768146FD170506139706014183636487
:10681000B7003E8582803307D50003470700B98F54
:10682000214713F81700858363050800B18FC2075D
:10683000C1837D171377F70F6DF78506F1B741C553
:10684000A547054763F2B7088347150003470500CE
:106850003168A207D98F13978700A183D98FC20708
:10686000C1831308C855054763900707411106C641
:1068700022C426C203442500914763F0870493078E
:10688000540063ECF502A301C50021822302C50078
:106890009304340091C6A302D500A1822303D5003E
:1068A0002A84A68597000000E780A0F5269423009F
:1068B000A4002181A300A4000147B24022449244D5
:1068C0003A854101828005473A8582800111B7C728
:1068D000A55A22CC9387E7342A842AC685660146C6
:1068E0009565254506CE3EC497C0FF1FE78060EF43
:1068F0003000A1469565294597C0FF1FE78060EEEF
:10690000A28517B501001305653997900100E7804E
:10691000A00C97000000E78080DDF2406244056132
:1069200082800111A146300095652D4522CC06CE0E
:1069300097C0FF1FE780E0EAA24737C4A55A1304B7
:10694000E43463958702B24517B501001305052F9E
:1069500097D7FF1F2393B7A8C205C1819790010065
:10696000E7808007F2406244056182809165A1461C
:106970003000938505EE2D4597C0FF1FE78060E648
:10698000A247E38287FCD14717D7FF1F2317F7A43D
:10699000D14517B501001305652CC9B721C14111B7
:1069A00026C206C622C4AE848DC52A849710000074
:1069B000E780203897E7FF1F83C7878999CB228517
:1069C0002244B240A685924441011743000067006B
:1069D00043DDB24022449244410182808280011111
:1069E0004EC606CE22CC26CA4AC893F71500AE89F9
:1069F0009DCBAD67371700409387A7AA1CC3B7E7A5
:106A00000400BC4F13060019854517D5FF1F034529
:106A1000A59C829713C51900F2406244D2444249B2
:106A2000B2490561828093F725000145F5D717F734
:106A3000FF1F035767D2954763F9E70C014417F628
:106A4000FF1F130666C19306300513055004130893
:106A500010049308B0041303900593076400637453
:106A6000F7043A847D5997F4FF1F83C4E4BE97F777
:106A7000FF1F83C777BEA204DD8CAD679387B75530
:106A8000638BF41463E3970AA9679387A755638E12
:106A9000F414A28517F5FF1F130505BC970000002D
:106AA000E78000F0E9A0B307860083C50700639A7A
:106AB000D50483C517006396A50483C52700639298
:106AC000050583C53700639ED50283C54700639AD9
:106AD000150383C757006396670222890DE897F56F
:106AE000FF1F83D565C7B3852541C20517F5FF1F75
:106AF000130585B6C1814A9597000000E78040EAFA
:106B0000E1A005044204418089BF3A847D5985474C
:106B1000E3EB87F45DC4854517F5FF1F1305C5B387
:106B200097000000E780C0E769A8B1679387C75561
:106B30006389F404B5679387D755E39CF4F4A28581
:106B400017F5FF1F130545B197400000E78060C5AA
:106B50008947630EF4009305E4FFC205C18117F570
:106B6000FF1F130585AF97100000E780801CA685E6
:106B700017B501001305451497900100E780C0E5A3
:106B800089A097300000E78020B797100000E780C9
:106B9000200311C9A28517F5FF1F1305E5AB971058
:106BA0000000E78000190546A28517F5FF1F1305B1
:106BB000A5AA97F0FFFFE780206097300000E780EC
:106BC000A0B3FD57E31DF9F097F7FF1F239607B811
:106BD00013C5290091B5A28517F5FF1F1305C5A799
:106BE00097F0FFFFE780406959B7A28517F5FF1FAF
:106BF000130585A697F0FFFFE780C0698DBF41119F
:106C000022C437E404005C5C06C6354697B5010033
:106C1000938585C217C50100130585C8829711E9C0
:106C200017B501001305850A97900100E780A0F2CF
:106C300001A08327041C82972A84054597D0000071
:106C4000E780E0A597700100E780002B97700100B6
:106C5000E780000097C00000E78060B72285B2405F
:106C60002244410182804111054506C622C426C244
:106C700097C0FFFFE780202C1305A00497B0FF1FEB
:106C8000E780E042757585457D1597C0FFFFE78079
:106C9000C0157D7585451305F53697C0FFFFE78064
:106CA000201F371400408327840A8D4513050020D8
:106CB00093E707202324F40A97C0FFFFE780E01240
:106CC000B7E4040097C0FFFFE7800058C8589790CA
:106CD0000100E78040E817C50100130565BC9790E7
:106CE0000100E78040E78327840C8545414593E711
:106CF00007082324F40C97C0FFFFE78060198D4537
:106D00001305000897C0FFFFE780801897C0FFFFBA
:106D1000E780604537A507001305051297C0FFFF00
:106D2000E7800041014597C0FFFFE7802047954578
:106D30000545894717F7FF1F2302F7A297C0FFFFFA
:106D4000E7806047B7E700E013070006238DE740C0
:106D50003707000423A0E71097D0FFFFE780E0C8C3
:106D600097D0FFFFE780E0DA97000000E78060E956
:106D700097000000E78060A197000000E780A0BABC
:106D800097E0FFFFE780C0C997100000E780A0FBF5
:106D900097000000E780801083A704081705000013
:106DA000130525C4829797C7FF1F2387A762BC4C92
:106DB000130600648545829797B0FF1FE780406304
:106DC00001458280AD67371700409387A7AA1CC38F
:106DD000B7E700E03707400023A0E71801000100F3
:106DE000B7F7070003C70701A5476316F700939796
:106DF000450191C301A04111AE860146AA852545F2
:106E000006C697C0FF1FE780C09DB240B7E700E00D
:106E10003707400023A0E710410182804111B2866C
:106E20002E86AA852D4506C697C0FF1FE780609B6A
:106E3000B2400145410182809307000463ECC7041E
:106E40001D71A2CC2A840808A6CACAC886CE32C63A
:106E500097900100E780E0ACAD673717004093875B
:106E6000A7AA1CC3B7E400E03709400023A02419F7
:106E700001000100B2461008A285294597C0FF1FF6
:106E8000E7802096F640664423A02411D644464964
:106E9000256182803955828041110D658D4506C678
:106EA00097C0FFFFE78060F4B71700408D6623A608
:106EB000D70A17F5FF1F1305A58A1387C70A9387FB
:106EC000870A1CC15CC5856689675CC958C114C541
:106ED00018C9B7E70400B24003A3871E410102832B
:106EE0008145B307B5008387070089E717330000A2
:106EF000670023878505C205C181E5B797B7010003
:106F00009387C7351357C5003E9703470700011104
:106F100006CE2304E100135785003D8B3E970347BF
:106F2000070023060100A304E100135745003D8B31
:106F30003D893E97AA970347070083C707002800AB
:106F40002305E100A305F10097000000E78080F928
:106F5000F24005618280011106CE2307010001ED98
:106F600017B501001305452F97000000E78080F753
:106F7000F240056182805800A947BA852946254814
:106F8000B376C502FD1793F7F70F93860603A304A4
:106F9000D700B356C5026375A8007D173685EDF39B
:106FA0003385F500D1B797B701009387272B135787
:106FB00045003D893E97AA970347070083C707000E
:106FC0000111680006CE2306E100A306F1002307A5
:106FD000010097000000E780E0F0F2400561828048
:106FE00081473307F600030707000DE363E4F5026A
:106FF0004111B2853E8606C697900100E780009059
:10700000B240133715003A85410182808507C207D7
:10701000C183C1BF3A858280011117B501001305F4
:10702000651906CE22CC26CA4AC897000000E78020
:1070300060EB17E5FF1F0355457297000000E780DE
:1070400020EC97E7FF1F83C7E76017B50100130522
:10705000651189C717B50100130545109700000099
:10706000E78040E817B501001305051597000000FB
:10707000E78040E717B5010013058514970000006D
:10708000E78040E6114597000000E78000ED17B566
:1070900001001305E57497000000E780A0E40145B6
:1070A00097000000E78060EB17B5010013054573FA
:1070B00097000000E78000E313051005970000002B
:1070C000E780A0E997D7FF1F83C7971817B501007E
:1070D0001305C50989E717B501001305A509970030
:1070E0000000E78020E017B501001305E50D9700CB
:1070F0000000E78020DF37A5070013050512970081
:107100000000E78080E517B501001305650C9700C6
:107110000000E78020DD97E7FF1F83C7276617B5CC
:1071200001001305A50589E717B5010013058505BD
:1071300097000000E78000DB17B501001305050A82
:1071400097000000E78000DA17B5010013058509F4
:1071500097000000E78000D917B501001305050965
:1071600097000000E78000D817C5FF1F035585244E
:1071700097000000E780C0D817B501001305450748
:1071800097000000E78000D617C5FF1F0355E524D0
:1071900097000000E780C0D617B501001305C505AC
:1071A00097000000E78000D417D5FF1F035505F1B5
:1071B00097000000E780C0D417B50100130545040F
:1071C00097000000E78000D217D5FF1F0355C5EEDA
:1071D00097000000E780C0D217B501001305C50273
:1071E00097000000E78000D017D5FF1F0355E5EC9E
:1071F00097000000E780C0D017B501001305050116
:1072000097000000E78000CE17C5FF1F0355450B10
:1072100097000000E780C0CE17B50100130585FF79
:1072200097000000E78000CC17D5FF1F0355A5E8A5
:1072300097000000E780C0CC17B50100130505FEDC
:1072400097000000E78000CA17D5FF1F035565E6C9
:1072500097000000E780C0CA17B50100130585FC40
:1072600097000000E78000C817D5FF1F035585E48D
:1072700097000000E780C0C817B50100130505FBA3
:1072800097000000E78000C617D5FF1F0355E5E112
:1072900097000000E78060CC17B50100130585F961
:1072A00097000000E78000C417D5FF1F035545E095
:1072B00097000000E780C0C417B50100130505F86A
:1072C00097000000E78000C217D5FF1F035505DEB9
:1072D00097000000E780C0C217B50100130585F6CE
:1072E00097000000E78000C017D5FF1F034525DC8D
:1072F00097000000E78060CB97E7FF1F83C7674DCB
:1073000017B50100130585E889E717B501001305D6
:10731000A5E897000000E780E0BC97E7FF1F83C760
:10732000E75917B501001305E5E789E717B501002F
:107330001305C5E797000000E780C0BA17B5010044
:107340001305C5F097000000E780C0B9014417C9D4
:10735000FF1F130969519944B307240103C50700AE
:10736000050497000000E78040C4E31794FE17B5BA
:107370000100130525EE97000000E780A0B60A85FE
:1073800097F0FFFFE78080A20A8404088347040087
:10739000034514000904A2075D8D97000000E780F3
:1073A00020B6E39584FEF2406244D244424905612E
:1073B0008280411126C2E97797E4FF1F93844450ED
:1073C00022C49387A7552E842381B4002E86AA85D4
:1073D00017E5FF1F1305054F06C62390F400A38190
:1073E000040097800100E780C05393052400C20584
:1073F000C18117E5FF1F1305C54C97F0FFFFE7801C
:107400004040B38784002382A7002181A382A70084
:10741000930564002244B24026859244C205C1818E
:107420004101172300006700C33309C99307000413
:1074300063E6B700170300006700E3F78280930656
:10744000F0030307060019E79307F00363F0B702A0
:107450002E85828093871500C207C183E3E6F6FE7E
:10746000AA952380E5000506BE85E1BF2E95230081
:107470000500F9BF5971B7064000A6D286D6A2D43E
:10748000CAD0CECE17E7FF1F1307872F8144594676
:10749000A5066383A472834707003A89D91793F737
:1074A000F70F6367F600B3D7F600858B050785EF06
:1074B000B3049540C204C180BD4763EA9702014707
:1074C0006397F4063D4697B501009385A59C4A85D0
:1074D00097800100E7808042014731E917B501003C
:1074E0001305459C25A08504C204C1805DB74146B3
:1074F00097B50100938585974A8597800100E780BD
:10750000E03F69F117B5010013058597970000006A
:10751000E780409D97000000E78040B017A501007C
:107520001305050A97000000E780C09BADAAB706C7
:1075300040005946A506B307E90083C707001315A5
:1075400007014181D91793F7F70F636FF600B3D79F
:10755000F600858B91CB05070505931707014205BA
:10756000C1834181E3E997FCB389A440C20993D95F
:107570000901A14763F237153304A900254697B5E1
:10758000010093856593228597800100E78000378D
:1075900063140512A547638EF900834794003547AD
:1075A0006389E70029476386E70093F7F70D639542
:1075B000071017B601001306E690814508089700EA
:1075C0000000E78000E8AA8517B601001306C69000
:1075D000080897000000E780C0E6AA8517B60100FA
:1075E00013064690080897000000E78080E593079F
:1075F0004003AA851306D1000808A306F10023075B
:10760000010097000000E780C0E3AA8517B60100DB
:107610001306061D080897000000E78080E2AA858F
:1076200017B60100130646C3080897000000E7805C
:1076300040E1AA8517B601001306861A08089700CC
:107640000000E78000E0AA852307010058002946D2
:107650009307100529482545B3F607037D161376D1
:10766000F60F93860603A304D700B3D6070363750A
:10767000F5007D17B6876DF25C003E96080897000E
:107680000000E78000DCAA8517A60100130646F378
:10769000080897000000E780C0DAAA85080897204C
:1076A0000000E780000C05442285B650265496540D
:1076B0000659F6496561828017B6010013060683F4
:1076C000A6854A8597000000E780C09131C5938761
:1076D00024FFC207C1830D47637BF7021304E9004F
:1076E000114697A501009385657622859780010054
:1076F000E780C0203DC1114697A501009385057321
:10770000228597800100E780601F630F051417A58D
:1077100001001305A57E39B517B601001306468092
:10772000A6854A8597000000E780C08B11ED17A65B
:1077300001001306E67FA6854A8597000000E780D2
:10774000608A2A846309053897A901009389C96C66
:1077500097A501009385856C09A897A901009389D5
:10776000E96E97A501009385E56E81471308100423
:1077700013054004930820051303D0031387570013
:1077800093160701C18263E1D414B306F90003C65E
:1077900006001376F60D631E061303C61600137655
:1077A000F60D6318A61203C626001376F60D6312B3
:1077B000A61203C636001376F60D631C161183C697
:1077C0004600639866109D8CC204C1809387B4FF05
:1077D000C2073A99C18305476375F70283460900DA
:1077E00013070003639FE600034719009306800513
:1077F0001377F70D6317D700E51493970401090970
:10780000C1838146014491482543154513970601DC
:10781000418313F8F60F6307F70A6390160793176F
:107820000401C1876352F00A97E7FF1F83C787E20D
:10783000CDE717A501001305657397F0FFFFE780FB
:10784000606A228597F0FFFFE780806B17A5010033
:107850001305057497F0FFFFE780C0684E8597F029
:10786000FFFFE78020685DB997A901009389095C53
:1078700097A501009385055CCDBD3307D90003476B
:107880000700130607FD137EF60F6368C301120499
:10789000518C42044180850695BF1306F7FB137691
:1078A000F60F6367C5001204130797FC598CD5B710
:1078B0001306F7F91376F60F6366C5001204130773
:1078C00097FAEDB7E31D08F417A5010013058567C6
:1078D00091B98507C207C18355B597E7FF1F83D7C5
:1078E000C7E76397870017A501001305E56AB1B7DD
:1078F000C16717C7FF1F0357E7ABFD178144631428
:10790000F70417A501001305656B97F0FFFFE780EB
:10791000605D228597F0FFFFE780805E17A501007C
:107920001305056797F0FFFFE780C05B4E8597F072
:10793000FFFFE780205B17A501001305A56ADDB6F0
:107940008504C204C180B387950083870700EDFBDF
:10795000228597E0FFFFE780404C2A8959C917A587
:1079600001001305E56897F0FFFFE780A057228527
:1079700097F0FFFFE780C05817A501001305456188
:1079800097F0FFFFE78000564E8597F0FFFFE780F6
:10799000605517B501001305258797F0FFFFE780B5
:1079A000605413150901418197F0FFFFE7804055AE
:1079B00017B501001305458497F0FFFFE78080525B
:1079C00017C5FF1F0355856F97F0FFFFE7804053F2
:1079D00017B501001305C58297F0FFFFE7808050BF
:1079E00017C5FF1F0355456D97F0FFFFE780405116
:1079F00035B617A501001305E56197F0FFFFE78095
:107A0000604E228597F0FFFFE780804F17A50100A9
:107A10001305055897F0FFFFE780C04C4E8597F09F
:107A2000FFFFE780204C17A501001305256097F0A4
:107A3000FFFFE780204B1385140097F0FFFFE780DE
:107A4000C05117A501001305255F97F0FFFFE780E0
:107A5000604917A501001305657997F0FFFFE780DE
:107A6000604817C5FF1F0355E59497F0FFFFE780B7
:107A7000204917A501001305257897F0FFFFE7803F
:107A8000604617C5FF1F0355656397F0FFFFE7804A
:107A9000204717A501001305A57697F0FFFFE780A3
:107AA000604417C5FF1F0355256197F0FFFFE7806E
:107AB000204517A501001305A5B097F0FFFFE7804B
:107AC000604217A501001305A55797F0FFFFE78057
:107AD0006041228511BFC54763FE9704454697A5BF
:107AE00001009385A5574A8597800100E78000E152
:107AF00021E58347190113071003639CE7008547BD
:107B000017E7FF1F2307F7CC17A5010013054556FC
:107B100011BC1307000317A5010013056558E39373
:107B2000E7A097E7FF1F238607CA17A501001305E3
:107B3000A555CDBA639EF404414697A501009385EF
:107B4000A5584A8597800100E78040DB29E58347F7
:107B5000090113071003639CE700854717E7FF1F20
:107B6000230EF7C017A501001305455765BA130783
:107B7000000317A5010013056559E395E79A97E7F8
:107B8000FF1F238D07BE17A501001305A55659BA7F
:107B9000A547E3FB97B0294697A501009385455972
:107BA0004A8597800100E78060D5E31F05AE17A5E1
:107BB00001001305A558BDB20144FDB417E5FF1F30
:107BC0000345C5BB8280011152C406CE22CC26CA11
:107BD0004AC84EC617EAFF1F034A4ACE631E0A0A66
:107BE00085473684B289AE842A896394F60C97E778
:107BF000FF1F83D787B8638EB70697E7FF1F239EC3
:107C0000B7B697E7FF1F238907B6054A17A50100F6
:107C10001305851297F0FFFFE780C02C4A8597F087
:107C2000FFFFE780E02D17A501001305651297F00F
:107C3000FFFFE780202B268597F0FFFFE780E031EC
:107C4000630A0A0017A501001305051197F0FFFF4D
:107C5000E78040296244F240D2444249B249224A74
:107C600017A501001305C595056117F3FFFF670010
:107C7000632797E7FF1F83C7C7B599CF97E7FF1F14
:107C800083C787AF850793F7F70F6147636EF700E8
:107C900017E7FF1F2302F7AEF2406244D244424985
:107CA000B249224A0561828097E7FF1F238607AC0D
:107CB000B1BF91476397F60097E7FF1F83C767B18E
:107CC000E1DF17A501001305A50997F0FFFFE78085
:107CD00060214A8597F0FFFFE780802217A5010009
:107CE0001305050797F0FFFFE780C01F268597F073
:107CF000FFFFE780802617A501001305A50797F071
:107D0000FFFFE780201E4E8597F0FFFFE780E02908
:107D1000894717A5010013056506E309F4F28D47AD
:107D200017A5010013050506E316F4F205B797E75A
:107D3000FF1F83C7A7B889E717230000670063A266
:107D4000828097E7FF1F83C707BC99EF411106C6E2
:107D500097200000E780C098B240854717E7FF1FD3
:107D60002303F7BA410182808280630E0538638C59
:107D700005381D71CAC8CEC686CEA2CCA6CAD2C44A
:107D8000D6C2DAC05EDE62DC66DA6AD86ED6B94781
:107D9000AA892E8963FFB708394697A50100938504
:107DA00025FF97800100E78060B541E583C7E900C2
:107DB000130710036396E704854717E7FF1F230F98
:107DC000F7AE17A501001305A5FD97E7FF1F239642
:107DD00007AE97E7FF1F239D079E97F0FFFFE78001
:107DE0006010F6406644D6444649B649264A964A4B
:107DF000064BF25B625CD25C425DB25D25618280C3
:107E00001307000317A50100130585FCE397E7FCA2
:107E100097E7FF1F238407AA97E7FF1F239F07A861
:107E200097E7FF1F2396079A17A501001305C5F8CA
:107E30006DB797E7FF1F83C767A8638C072A95472D
:107E400063F52703194697A501009385A5FA4E858A
:107E500097800100E78080AA09E917A501001305B2
:107E6000E5F997F0FFFFE780E007BD6A396C014A4A
:107E700017EBFF1F130B0B96938BFA55938CFA6637
:107E8000130DEC5593170A01C183E3FC27F5B38763
:107E9000490183C6070097E7FF1F83D707A285E341
:107EA0009307A005639BF600854717E7FF1F23167E
:107EB000F7A097E7FF1F238FD790050AE1B7854DFD
:107EC000639BB7039307500A639EF600894717E741
:107ED000FF1F2314F79E930750FA17E7FF1FA30B0A
:107EE000F78EE1BF9307A005E389F6FC97E7FF1F34
:107EF0002395079CD9B7138717004207DA97418368
:107F00002380D70017E6FF1F2319E69A8D47E3F673
:107F1000E7FA17E4FF1F0344148C97E7FF1F83C79A
:107F2000878B22045D8C9307F4FFC207C1839306FD
:107F3000F00DE3EDF6FA93076400C207C183E31E78
:107F4000F7F693052400C205C18117E5FF1F13054D
:107F5000858897F0FFFFE780C08A33078B0083474F
:107F6000570003474700A207D98F17E7FF1F2316C3
:107F700007946311F5108144630CB40197E4FF1F6B
:107F800083C48485A20497E7FF1F83C7F784DD8C31
:107F900017F5FFFF1305A54997E0FFFFE780801F56
:107FA0006385740963EF9B026388A4059307EC65FE
:107FB0006383F40697E7FF1F83C707820547638043
:107FC000E70881CB1387A7051377F70F8D4663F971
:107FD000E6081307F0072300E100A300F10089453C
:107FE00095A8638994059387FA77E395F4FC97E065
:107FF000FFFFE780606111A8A28517D5FF1F130559
:10800000A57D97E0FFFFE780E029014597E0FFFFAE
:10801000E78040185DB5A28517D5FF1F1305C57B06
:1080200097E0FFFFE7800031CDB797E0FFFFE780E3
:108030008039E1BF97E0FFFFE780203FF9B7930762
:1080400010F8130511002300F10097E0FFFFE7800F
:10805000805EFD450A8597F0FFFFE780C03575B764
:10806000A28517D5FF1F1305257797E0FFFFE7804F
:1080700000E961BF9307F00789450A852310F100E5
:1080800097F0FFFFE78020330DBDB387890083C7DA
:10809000070063849700639C47010DC597F0FFFFBD
:1080A000E780803D97D7FF1F2394077221A8E3EB59
:1080B000AAFE130715005A9597D6FF1F239AE6705C
:1080C0002300F500050493170401C18317D5FF1F92
:1080D00003550570E3EB27FBE30505D097F0FFFFA1
:1080E000E7808039E30F05CE97D7FF1F2392076EF5
:1080F000CDB90144B544294A930AE00417DBFF1FB8
:10810000130B0B68C9B78280411126C2AE848D451E
:1081100022C406C62A8497B0FFFFE78060D7B7174E
:10812000004099C803A5C70C418D23A6A70CB240F7
:10813000224492444101828003A5870C418D23A4EF
:10814000A70CF5B78347050003471500A207D98F91
:10815000C2076177C18713072720639AE700834529
:1081600025003705040017030000670023FA82800A
:1081700017D6FF1F130686798147B2861303F00FC7
:10818000A9483308F6000348080013F7F70F630700
:10819000A80C630668008507E39517FF2947B38796
:1081A000E6002380A70097D7FF1F9387E7765DA897
:1081B000411113D765001347170006C693F6350023
:1081C000058B954791CA054699476387C6000946BE
:1081D0009D476383C600A14713F645003336C000B0
:1081E00093F68503050685C2A145638BB604E14578
:1081F000638AB604930580026388B60493058003FE
:108200006393B600914697E5FF1F238CF59697E59B
:10821000FF1F2387C59697E5FF1FA383D596BE85CD
:1082200017A501001305850797700100E780C07A44
:10823000B240854717E7FF1FA305F79441018280ED
:108240008546D1B78946C1B78D4675BF17A50100D0
:1082500013054507177301006700037817D7FF1F41
:108260001307876BBA972380B700E147E302F5F461
:1082700093077002E30CF5FC82802A8723800500B7
:10828000814717D5FF1F130565681308F00F2946AE
:10829000B306F50083C606006396E60297D6FF1F75
:1082A00093868667B69783C7070005452380F50048
:1082B0009947636EF7029D4763FDE700E147630D51
:1082C000F7008280638506018507E393C7FC0145BB
:1082D000C5B7238005008280B737004003C7370049
:1082E00083C7050093F70704D98F2380F5008280A8
:1082F0005D7152DC56DA5ED6716A97EBFF1F938B85
:108300006B998D6AA6C24EDE62D486C6A2C4CAC06C
:108310005AD866D26AD06ECEC1495E8C97D4FF1F00
:1083200093844460130A0A20938A7ADC17E9FF1FBA
:1083300003494999B3872B0183C7070093F7F70FC8
:10834000C9EFB787004003C76700058BE310077CC0
:1083500003C76700118BE30D077E83C75700918B1E
:1083600099E36F10200317E7FF1F0347C795854761
:108370006304F7006F10400197E7FF1FA383E780B6
:1083800097D7FF1F2380076697D7FF1F238E07709D
:1083900097D7FF1F238C077C97D7FF1F2389077C64
:1083A00097D7FF1FA380076497D7FF1FA38E076E81
:1083B00097D7FF1FA38C077A97D7FF1FA389077A48
:1083C00097D7FF1FA380077C97E7FF1FA38D078E1A
:1083D000B787004011476F0070779307190093F734
:1083E000F70F3D476364F70617E7FF1F230CF78C71
:1083F00097E7FF1F9387078CCA9783C70700130768
:10840000100293F7F703638EE71E6366F7040544D3
:108410006385871CE38C07620947638EE7101307A7
:108420000002E384E74EB7E700E03707400023A0EF
:10843000E71801000100629923000900FD1923A03B
:10844000E71093F9F90FE39309EEE5BD97E7FF1FF6
:10845000238A078671BF130730026388E70C63E83D
:10846000E71613074002638CE70A13070003E39C37
:10847000E7FA97E7FF1F9387E782CA9703C70700CA
:10848000A1471377F70FE31BF71483C7640097D650
:10849000FF1F238FF66C97D7FF1F83C7174991C71C
:1084A000FD5797D6FF1F2385F66C97D5FF1F83C511
:1084B000754797D7FF1FA38DB76A97D7FF1F83C74D
:1084C000674613FB07089306000493F70706639FAC
:1084D000D74C9307A009638DF51663EAB71293078B
:1084E000F0056386F54A930750096384F52A014431
:1084F00097D7FF1F83C7D7671547E392E736B7E7DC
:1085000000E03707400023A0E71801000100B7860C
:10851000004023808602130680FC6F00500EFD573A
:1085200017D7FF1F2305F764FDBDFD5717D7FF1FA2
:10853000230EF762CDBD17A50100130525EA97703C
:108540000100E780406197D7FF1F9387A775CA97FF
:1085500003C40700014B97DCFF1F938C2C55137449
:10856000F40F17AD0100130DEDE763478B042945A8
:1085700097700100E780204B854717D7FF1FA305A1
:10858000F75217D7FF1F2302875217D7FF1F230B5E
:10859000F75E37E700E0B70640002320D718010058
:1085A0000100378600408347A60293F7370F230563
:1085B000F6022320D71085BDB3876C0183C5070061
:1085C0006A85050B97700100E780004179BF8547F8
:1085D00017D7FF1F230AF74CB9B517D7FF1F13078B
:1085E000676C4A970347070097D6FF1FA38CF63E98
:1085F00097D6FF1F2389E63E17D7FF1F2304F7589E
:108600001DB5854717D7FF1F230EF73C29BD9307DC
:10861000400A6389F5349307200B6384F53693078A
:10862000100AE396F5EC838724000144E3D207ECBB
:1086300097D7FF1F83C7372F93F63700638A061A31
:108640000546638AC62209466395C61A1D4755A288
:1086500017D5FF1F0345252DC94797DCFF1F83CC86
:108660009C2C97D5FF1F83C5252C17D4FF1F0344CF
:10867000B42B6315F510CD476392FC109307700877
:10868000639CF5021307300FB7170E006308E40070
:108690001307900DB7B704006314E40817D7FF1F42
:1086A000232EF74CBE8517A50100130525D497701E
:1086B0000100E780603225BD93078008639DF500C7
:1086C000B307804013F4F70FB7774600938787CD41
:1086D000B3D78702E1B793079008639AF500B30711
:1086E000804013F4F70F91679387C766D5B7930758
:1086F000A008639BF500B307804013F4F70FB7178A
:108700003D0093870790E9B79307B008639AF50097
:10871000B307804013F4F70F9167938797D04DBF4D
:1087200093F5F5078D47639BF500B307804013F47D
:10873000F70FB7975B00938707D859BF8947639BAB
:10874000F500B307804013F4F70FB7770B0093875A
:10875000071BBDBF8547639AF500B307804013F43C
:10876000F70FDD67938767E3A5B7D28785F9B3076E
:10877000804093F7F70FB3D7FA020DB797000000C8
:10878000E780409FA285668597000000E780809E75
:10879000B9BB9305610017D5FF1F0345C51817D452
:1087A000FF1F0344541897000000E78040AD930575
:1087B0007100228597000000E78060AC3C0017D76D
:1087C000FF1F2327F74C834761002304F1008347F1
:1087D0007100A304F100894717D7FF1F230AF73858
:1087E0008357810017D7FF1F231EF712094409B3CF
:1087F000154793F64700B336D00093F787038506F5
:1088000085C32146638BC7066146638AC706130684
:1088100080026388C706130680036393C7009147ED
:1088200017D6FF1F230ED63497D6FF1FA38AF63420
:1088300097D7FF1F2387E73417D7FF1F0347C70EBC
:108840009376070497D7FF1F83C7170E8DEE137714
:10885000770C93067008630CD7021377F7078D46E1
:108860006312D70CB307F040B7955B0093F7F70F8F
:10887000938505D849A81947ADBF854755B789479E
:1088800045B78D4771BF930670086311D702130770
:10889000300FB7150E006389E7021307900DB7B5C7
:1088A00004006383E7021307700845BF9306800C3A
:1088B0006311D702B307F040B775460013F7F70FFF
:1088C000938785CDB3D5E70297D7FF1F23A8B72A93
:1088D000D9BB9306900C631CD700B307F04093F507
:1088E000F70F91679387C766B3D5B702F1BF9306B9
:1088F000A00C631DD700B307F040B7153D0093F7F8
:10890000F70F93850590B3D5F5027DBF9306B00CA4
:10891000E315D7F4B307F04093F5F70F916793870A
:1089200097D0D9B78946631BD700B307F040B77516
:108930000B0093F7F70F9385051BF1B78546631A74
:10894000D700B307F040DD6593F7F70F938565E334
:108950005DBFD28535FBB305F04093F5F50FB3D578
:10896000BA029DB783C72400C18B99C7854717D723
:10897000FF1F2302F720A5BE97D7FF1F238D071ED9
:10898000BDB6854717D7FF1FA30DF71E8DB63C0058
:1089900017D7FF1F232EF72E094793070003231431
:1089A000F10097D6FF1F2385E61C2DBD6394075663
:1089B000A94763E5B74217A701001307678B8A052C
:1089C000BA959C41BA97828717D4FF1F0344B4F528
:1089D000894C6306940D63E68C0685476303F408AF
:1089E0009307F00F17D7FF1F0347871863F6E700B9
:1089F00017D7FF1F230EF71697DCFF1F83CC4C17EA
:108A00009307000413F4FC0F63F4970113040004AC
:108A100097D7FF1F9387C72703AD070022862685B8
:108A2000EA85B38C8C40229D97700100E78060EF4F
:108A300097D7FF1F238E971397D7FF1F23AAA7252A
:108A400045BC8D47630CF40A9947E31BF4F897A7DC
:108A500001009387678817D7FF1F232BF722A947A9
:108A600051B717D7FF1F0347072697D7FF1F9387D5
:108A70002712494697A501009385058F6306870055
:108A800097A501009385458A3E8597700100E78090
:108A900040E917D7FF1F232DA71EC947A1B797D6B7
:108AA000FF1F83C64622054797D7FF1F9387470EB0
:108AB0006394E6023E851306700297A50100938534
:108AC000258897700100E780C0E517D7FF1F232195
:108AD000A71C9307700239B73E851306300497A58B
:108AE00001009385258097700100E78080E317D708
:108AF000FF1F232FA71893073004EDB597D5FF1F4D
:108B000083C565E217A501001305858F97700100E5
:108B1000E78080EC054D97DDFF1F83CDCD1A97D5FB
:108B2000FF1F83C545E017A501001305658D6398F8
:108B3000AD0B97700100E78020EA97D7FF1F83C72E
:108B400087DEB5CBE36EF4E817A4010013040486B6
:108B5000638CB70117A401001304C48563869701D1
:108B600017A4010013048486228597700100E78012
:108B7000C0FF1375F50F93071500860717D7FF1F62
:108B80002308F7008D4717D7FF1FA303F70097D7D8
:108B9000FF1F9387E7FF0147BE861376F70F89070C
:108BA0006365A60297D7FF1F23A4D70E97D7FF1F91
:108BB00083C707FE05BD979701009387277817D7CE
:108BC000FF1F2327F70C914731BD3306E40003460E
:108BD0000600A380070005072380C7007DBF9770AC
:108BE0000100E78060DF97D7FF1F83C7C7D3E1D7B6
:108BF000E368F4DE1794010013044478638CA70142
:108C000017940100130404786386970117940100F8
:108C10001304C478228597700100E78000F513756E
:108C2000F50F93071500860717D7FF1F2302F7F6E6
:108C30008D4717D7FF1FA30DF7F497D7FF1F938713
:108C400027F50147BE861376F70F8907E37CA6F464
:108C50003306E40003460600A380070005072380CF
:108C6000C700D5B797D5FF1F83C5E5CB1795010082
:108C70001305C57997700100E78000D697D7FF1FCD
:108C800083C7D7F093E7470017D7FF1FA300F7F07C
:108C900083C7240017D7FF1FA308F7EE89B81795DD
:108CA00001001305E57797700100E780C0EA97D7C8
:108CB000FF1F938767ED83C7070017D7FF1F2303A5
:108CC000F7C617D4FF1F0344A4EA333480000DB065
:108CD000179501001305057697700100E780A0E75E
:108CE00097D7FF1F83C797EA93E7070117D7FF1F9F
:108CF000A30EF7E883C7240017D7FF1F2306F7E862
:108D00006FF0EFFE179501001305057497700100D1
:108D1000E78060E403C704007D8B51EFB787004014
:108D200003C767021377C70B136727002383E70284
:108D300003C7A7021377C70B136727002385E70232
:108D400003C7E7021377C70B136727002387E702E0
:108D500003C727031377C70B136727002389E7028D
:108D6000854717D7FF1F230FF7C617D7FF1F230D00
:108D7000F7D217D7FF1F230BF7DE17D7FF1F2308E4
:108D8000F7DE97D7FF1FA38F07C497D7FF1FA38DC9
:108D900007D097D7FF1FA38B07DC97D7FF1FA388A8
:108DA00007DC97D7FF1FA38F07DC97D7FF1FA38C84
:108DB00007F06FF0CFF389476312F70297D7FF1FD1
:108DC00083C787B69146638CD70863E0F604638E49
:108DD000E70C6369F70A05476380E70EFD5717D76D
:108DE000FF1FA307F7D837074000B7E700E023A02D
:108DF000E71801000100B78600401306F0FC23814C
:108E0000C60223A0E7106FF00FE213072008638269
:108E1000E7086362F70213071008E391E7FC37875E
:108E200000408347670293F7C70B93E727002303AC
:108E3000F7026FF0CFEB130730086389E7021307DF
:108E40004008E39DE7F8378700408347270393F7FF
:108E5000C70B93E727002309F7026FF04FE9378725
:108E600000408347270393F73707F5B7378700405C
:108E70008347E70293F7C70B93E727002307F7021F
:108E80006FF0EFE6378700408347E70293F7370735
:108E9000F5B7378700408347A70293F7C70B93E7DF
:108EA00027002305F7026FF08FE4378700408347E0
:108EB000A70293F73707F5B7378700408347670264
:108EC00093F73707ADB7179501001305E55897706D
:108ED0000100E78040C897D7FF1F238507A4D5B3BB
:108EE000179501001305455897700100E780A0C64B
:108EF00097D7FF1F239807A297D7FF1F938747C7CE
:108F000003C40700894763F3870009441374F40F0F
:108F10006FF00FDE13070002E392E7EC631B0B0A0E
:108F2000638FF500930720026383F508179501000E
:108F30001305055797700100E78000AA45B51795FE
:108F400001001305255397700100E780C0C001445C
:108F5000179D0100130D4D53A14CB387840083C5A9
:108F600007006A85050497700100E780E0A6E31614
:108F700094FF178501001305A56A97700100E7802B
:108F800080BD17D4FF1F0344249A01E897D7FF1F21
:108F9000238C0796014B6FF0AFD58947E310F4E4BB
:108FA000854717D7FF1F2301F7966FF04FD417D6C9
:108FB000FF1F0346569797D5FF1F83C5C596179584
:108FC00001001305E54C97700100E780E0A06FF009
:108FD0000FD26380F50693071002E399F5F497D555
:108FE000FF1F83C56594179501001305654C9770A5
:108FF0000100E780609E97D7FF1F23AB97C897D7E4
:10900000FF1F9387A7B7944383D7470017D7FF1F46
:10901000034727B717D6FF1F2326D6901D4497D6A0
:10902000FF1F2393F69097D7FF1F2380E7906FF0E1
:109030002FCC97D5FF1F83C5258F179501001305EA
:10904000A54897700100E780209997D7FF1F238DCF
:10905000078A97D7FF1F2397078C6FF02FF92547B3
:10906000638FE7C89946378700406394D70223008F
:109070008702B7E700E0B706400023A0D718010039
:109080000100130600FC2301C70223A0D7106FF0D4
:109090008FB99306100A639FD70023008702B7E7B2
:1090A00000E0B706400023A0D71801000100130616
:1090B00080FCD1BF9306A009E381D7FE9306400A46
:1090C000E38DD7FC93062002639DD700B7E700E04D
:1090D000B706400023A0D718010001002300870233
:1090E000F9B78546E384D7FE93070008E300FBFE4B
:1090F000B7E700E0B706400023A0D7180100010041
:10910000130620FC23008702BDBF17D7FF1F0347AC
:1091100037A66302F71E63E7E70295476300F7107F
:109120009947630AF704B786004023800602B7E731
:1091300000E03707400023A0E718010001001306F4
:10914000A0FC75B99307F005630AF700930750096F
:109150006306F70093071002E317F7FCB7E700E098
:109160003707400023A0E71801000100B786004040
:10917000130620FC69B117DBFF1F034B6B9F93079E
:1091800000045A8D63F46701130D000497D7FF1F85
:10919000938707B083AC07001374FD0F2286E68522
:1091A000268597600100E780C077B3078B406694FF
:1091B00017D7FF1F230EF79A97D7FF1F23AA87AC55
:1091C000B7870040630C0B022380A703B7E600E0DB
:1091D0003706400023A0C6180100010003C727027C
:1091E000134707042381E70203C727021377C70F3A
:1091F0002381E70223A0C6106FF0EFA223800702AD
:1092000037E700E0B70640002320D718010001002F
:10921000130620FC2381C7026FF0AFB937870040E7
:109220008347370097D6FF1F83C6169693F7070824
:10923000D58FA301F700B7064000B7E700E023A0F1
:10924000D718010001001306A0FC35BD97D7FF1FFA
:10925000938747A5CA9783C7070093F7F70FC1CF36
:1092600097D7FF1F83C727A6D9E717D7FF1F034745
:109270003790930700026310F70883AD040017CD01
:10928000FF1F034D6D6A97CCFF1F83CCFC6917CB82
:10929000FF1F034B8B69E6876A87DA866E8697C560
:1092A000FF1F83C565661795010013056523976049
:1092B0000100E780607297D7FF1F23A1B78D97D772
:1092C000FF1F238FA78B97D7FF1FA38B978B97D752
:1092D000FF1F2388678B97C7FF1FA3868762B7E7A7
:1092E00000E03707400023A0E71801000100B7861F
:1092F00000406FF04FA2B7E700E03707400023A01F
:10930000E71801000100B786004015BD97D6FF1F82
:1093100083C6669B0547639CE60429472381E702D1
:1093200009472383E7022385E70297D7FF1FA38B13
:10933000078497D7FF1FA3880798B7870040A381AA
:10934000070017D7FF1FA301078405472383E70002
:10935000B640264496440649F259625AD25A425BB4
:10936000B25B225C925C025DF24D616182802947B2
:109370002381E70209472383E7022385E702238746
:10938000E7022389E70255B717C7FF1FA30DF7565A
:109390006FE01FFF854717C7FF1F2305F76417C737
:1093A000FF1F2303F77017C7FF1F2301F77C17C7A1
:1093B000FF1F230EF77A6FE0BFFE854717C7FF1F19
:1093C0002302F76217C7FF1F2300F76E17C7FF1F9F
:1093D000230EF77817C7FF1F230BF77817C7FF1F58
:1093E000A302076017C7FF1FA300076C17C7FF1F63
:1093F000A30E077697C7FF1FA38B077682804111C4
:1094000006C697000000E78080FBB78700402380F6
:109410000700130740FC2386E7001307C004A38658
:10942000E70017C7FF1F1307E74F2398E70017C789
:10943000FF1F13072753239AE70017C7FF1F1307C0
:10944000A75E239CE70017C7FF1F1307276A239E09
:10945000E70029472381E70209472383E7022385A1
:10946000E7022387E7022389E702A3810700930627
:1094700000F8A380D700930690022380D700FD5602
:109480002383D7002381E7009306000537E700E038
:10949000230BD740B70640002320D71003C717007F
:1094A00013671700A380E700B24097C7FF1F239DF3
:1094B000076C41018280411106C697000000E780D9
:1094C00000F0B787004023800700130700FC2386C5
:1094D000E7003147A386E70017C7FF1F130787443C
:1094E0002398E70017C7FF1F1307C747239AE70012
:1094F00017C7FF1F13074753239CE7002947238102
:10950000E70209472383E7022385E702A3810700D7
:10951000930600F8A380D700930690022380D7001B
:10952000FD562383D7002381E7009306000537E724
:1095300000E0230BD740B70640002320D71003C715
:10954000170013671700A380E700B24097C7FF1FFB
:10955000239C076241018280F1679387072017C728
:10956000FF1F232DF760854717C7FF1F231AF760DA
:10957000A14717C7FF1F2306F76097C7FF1FA382E6
:10958000076097C7FF1F238F075E97C7FF1F238DB5
:10959000073697C7FF1FA3880736814717C5FF1FE8
:1095A0001305C536FD5517C6FF1F1306E6362947B6
:1095B000B306F5002380B600B306F600238006004C
:1095C0008507E397E7FE97C7FF1FA384075A97C74E
:1095D000FF1FA382075A97C7FF1F238D075897C7FE
:1095E000FF1F2388075897C7FF1F2387075897C770
:1095F000FF1FA381075897C7FF1F238E0756814778
:1096000017C6FF1F130606694147B306F6002380FD
:1096100006008507E39BE7FE828017C7FF1F03470D
:10962000876A85476316F700170300006700E3E8C1
:10963000170300006700E3DC411122C406C617C708
:10964000FF1F0347476885472E8613F4F50FAA8549
:109650006317F70417C5FF1F130505419760010045
:10966000E780202C97C7FF1F23800744B78700405F
:1096700023848702B7E600E03706400023A0C6181F
:109680000100010003C7A7021377C70F2385E70274
:10969000B240224423A0C61001454101828017C573
:1096A000FF1F1305253097600100E780802797C7CB
:1096B000FF1F23890732B787004023828702B7E65E
:1096C00000E03706400023A0C6180100010003C7D0
:1096D00067021377C70F2383E7025DBF411106C6F8
:1096E00097000000E78080E7B240410117030000C7
:1096F0006700E3F2411106C697F0FFFFE78080BFE5
:1097000097C7FF1F83C7172EA1CB97C5FF1F83C520
:10971000852D89C917C5FF1F1305052D97E0FFFF8C
:10972000E780E06497C7FF1FA38E072A97C7FF1F34
:10973000238A074437E700E0B70640002320D71804
:1097400001000100378600408347660293F7370F18
:109750002303F6022320D710B2404101828041C981
:10976000D9C597C7FF1F83C72742D1C3011122CC98
:109770004AC84EC656C25AC006CE26CA52C42E8900
:10978000AA890144930A0004371B0300637724036A
:10979000B3078940C207C183BE8463F4FA0093040F
:1097A0000004C204C180130A1BD497C7FF1F83C7DC
:1097B00067239DE37D1A631C0A00F2406244D24491
:1097C0004249B249224A924A024B0561828097F08F
:1097D000FFFFE78020B2D1BF338589002694A6859C
:1097E000420497000000E78060E5418045B7828031
:1097F00097C7FF1F9387875F18429C4383D6450016
:109800000345070083C5C700035646006396A500BD
:1098100083D5E700638DD502011106CE2386A7000C
:109820002397D700B705CF00DC4B9385757D0507DF
:109830007D162EC2230001003AC42316C10023174F
:10984000D10099C30A858297F240056182808280A7
:10985000411122C417A4FF1F130484BA5C4C06C62E
:1098600091CBC84B01C9B7E70400BC5782975C4C49
:1098700023AA0700B240224441018280DC4DDC4B28
:1098800081CFB7E70400904503A38705914517C52D
:10989000FF1F0345E55502838280B7E7040003A359
:1098A0000705A14517C5FF1F0345855402836D7148
:1098B0003C083EC6B707E500232291103EC8AA84A3
:1098C0003C083285232611103ECA23248110232010
:1098D00021112E8997300000E780605A2A849795DD
:1098E0000100938565C3177501001305E56E976048
:1098F0000100E780600EA28517950100130585CE53
:1099000097600100E780400D294597600100E780DE
:109910008011B705CB009385757D68009710000016
:10992000E780E05FA285680097300000E78080470D
:10993000014781467000CA85268597200000E78090
:10994000608305CD2A84979501009385E5BC177542
:1099500001001305656897600100E780E007A285B4
:10996000179501001305C5C897600100E780C00680
:10997000294597600100E780000B8320C110032474
:10998000811083244110032901105161828097C7FF
:10999000FF1F9387A74518429C43797122D406D6AE
:1099A0000348070083C807012A8483D6450003556E
:1099B00046006396080183D82701638DD802238867
:1099C000070105072399D7003708CC00DC4B1308A3
:1099D000787D3ACC1307F5FF42CA23080100231E05
:1099E000E100231FD10099C7080832C62EC4829710
:1099F0003246A245228597000000E78080EBB250F6
:109A000022544561828079713146977501009385B2
:109A1000654D280006D697600100E78080F097A783
:109A2000FF1F83D7E79D231B0100231C0100231D7B
:109A30000100231E0100231F010099E3C167FD17E8
:109A4000231AF10097A7FF1F83D7A79B91EB97C716
:109A5000FF1F9387A7399C439C43DC4783D70700AC
:109A600097A6FF1F9386C699231BF100D84E83D774
:109A70004600231CF1005C4B91CB97A7FF1F83C7C7
:109A8000979881EB97000000E780C0DCB2504561F9
:109A90008280FD1717A6FF1FA307F696035607013E
:109AA00083C706014C472800230FF10097300000C0
:109AB000E780602C97C7FF1F938747339C4301477C
:109AC000979601009386C6AE884330004C089710E5
:109AD0000000E780206A5DD975B799C9B7E704002F
:109AE00003A30705A14517C5FF1F03456530028382
:109AF00082805C4EDC4BB9CFB1CD411122C41775C9
:109B000001001305654D2E8497950100938505A6E8
:109B100006C697600100E78020ECA285179501003A
:109B2000130505A797600100E78000EB29459760C2
:109B30000100E78040EFB7E704002244B24003A3EE
:109B4000870517C5FF1F0345A52A13064006914543
:109B5000410102838280411122C417A4FF1F130414
:109B6000E4871C4C06C689C7DC4399C34C488297DE
:109B7000584CB7E70400BC57484B82975C4CB24046
:109B8000224423AA07004101828017A7FF1F130761
:109B9000E786834707009306F00B850793F7F70FD7
:109BA00063E9F60097A6FF1F238AF68403450700A2
:109BB0008280930700F8FDB78357450099E37D55F0
:109BC0008280011122CC17A4FF1F130464835C4C14
:109BD0004AC84EC6DC4B52C406CE26CA56C2B2890B
:109BE0002E8A2A898DC7B7E70400FC5F829797C742
:109BF000FF1F9387A71D9C431307301FB307F54032
:109C000071556375F70697000000E780A0C49307BD
:109C1000D00D7D5563EC3705B7E4040093878900C8
:109C2000B858832AC401139507014181029723AADA
:109C3000AA00484C584921E7979501009385059162
:109C4000177501001305453997600100E780C0D8FA
:109C5000179501001305859C97600100E780C0D728
:109C6000294597600100E78000DC5D55F2406244C1
:109C7000D2444249B249224A924A056182801387FE
:109C80004900B705CF002319E5009385757D31059F
:109C900097100000E780A028484C834569003105F3
:109CA00097300000E7800010484C4E86D285310581
:109CB00097300000E780200C7146CA851795FF1F7A
:109CC0001305057497600100E780A0C5FC5C8297CE
:109CD0000326C90097C7FF1F23AAA70E11CABC4CB1
:109CE000854517C5FF1F0345A51082970145BDBFD8
:109CF00097000000E78060D1D5BF411106C622C49D
:109D000026C217C4FF1F1304A40E97000000E780AB
:109D100060B4B7E40400FC4C034504008545829719
:109D200003450400224403A3C405B2409244A14564
:109D300041010283411126C297C4FF1F9384040B83
:109D40009C4006C622C44AC0D5C3DC43C5C35CC11F
:109D50002300B5002A84978501009385657A1775DD
:109D600001001305652797600100E780E0C62945DB
:109D700097600100E78020CB9C4023A4070023A22A
:109D800007009797FF1F93876765DC4FDC4B91C7F0
:109D9000295597000000E78040DC9797FF1F9387C5
:109DA0002766DC4FDC4B89C797000000E78020F571
:109DB00037E904008327C905894517C5FF1F0345F7
:109DC000250382978327C905914517C5FF1F0345C2
:109DD000250282979C4003A3470163090300228563
:109DE0002244B2409244024941010283B2402244DB
:109DF00092440249410182800111328506CE22CC73
:109E000026CA2E8497300000E7806007AA849785D1
:109E1000010093852572177501001305E51B9760F6
:109E20000100E78060BB030784000356640083558C
:109E30004400A68617850100130505789760010088
:109E4000E78080B9294597600100E780C0BD9797FA
:109E5000FF1F83C70759639D9700014597000000C6
:109E6000E780A0CF81450A8597000000E780C0EC1D
:109E7000F2406244D244056182806D7123248110D6
:109E8000232611102322911093F745002E84638717
:109E900007143C083EC0B707E5003EC23C083EC47C
:109EA000231701002318010023190100231A0100C0
:109EB000231B01009797FF1F83D7475299E3C16780
:109EC000FD172316F1009797FF1F83D7475191EB9A
:109ED00097C7FF1F938787F19C439C43DC4783D739
:109EE00007001797FF1F1307674F2317F100544F01
:109EF000835747002318F100DC4AA1E7978501004A
:109F000093858567177501001305050D976001009E
:109F1000E78080AC178501001305C57697600100C6
:109F2000E78080AB294597600100E780C0AF13450B
:109F300044008320C1100324811083244110516107
:109F400082809797FF1F83C7D7492555D9C3FD172F
:109F50001796FF1FA307F64803D60601834707019C
:109F6000CC460A85230BF10097300000E780A0E083
:109F700097C7FF1F938787E79C431797FF1F130718
:109F8000E745978601009386266088430A866C0021
:109F900097100000E780001EAA8451D99785010020
:109FA0009385855D17750100130505039760010012
:109FB000E78080A2A685178501001305656D97606F
:109FC0000100E78060A1294597600100E780A0A516
:109FD000268597000000E78040B891BF93F72500E1
:109FE0009DC7B7E70400BC474146814528088297D2
:109FF000255597000000E78040B628089305F00F2C
:10A0000097000000E78040D3134524001DB793F765
:10A01000150081CB97000000E780209F13451400B6
:10A0200009BF93F78500014589D71797FF1F03479D
:10A03000973D9797FF1F9387A73C0DC3D84F584B69
:10A0400011CF37E70400384F9047854517C5FF1FEC
:10A05000034505DA029713458400E1BD97F0FFFF41
:10A06000E780407FCDBF5C4D411106C688C317C74E
:10A07000FF1F232DF7D6B7E7040083A707081705AE
:10A0800000001305C5DF8297B24097C7FF1F2381E9
:10A09000A7D601454101828001113335A000A307F5
:10A0A000A100B7E7040083A7471706CE1306F10007
:10A0B0008545130550308297F24005618280828089
:10A0C000411122C406C697A7FF1F83C7771805440E
:10A0D00089EF97B7FF1F83C7E757014499E717A494
:10A0E000FF1F0344E4161344140022859700000068
:10A0F000E780C0FA178501001305456009E417855C
:10A1000001001305A5602244B2404101176301001C
:10A110006700838C797122D4A30F010037E4040017
:10A120008327841726D24AD006D6AA842E891305FF
:10A1300050309305F10132C6829732468347F101D0
:10A1400093150601C18185CB01452EC697000000FD
:10A15000E780C0F483274417B2454A862685829754
:10A16000054597000000E78060F3B25022549254F6
:10A17000025945618280832744174A862685829743
:10A18000EDB741119397050122C406C626C2C187C7
:10A190002E8463D40702B7E40400FC541795FF1F14
:10A1A00003450529829719C1BC5482972165218DE9
:10A1B000B240224492444101828093F715008DC73A
:10A1C000B7E7040083A7471A1796FF1F1306462513
:10A1D00097C5FF1F938585C21795FF1F034545252A
:10A1E000829713451400E9B793F725000145E9D399
:10A1F00097C7FF1F83C707C285E7B7E7040003A817
:10A20000871A1307401F9797FF1F83C7672281464E
:10A2100013064006994517C5FF1F035525BF029831
:10A220001345240071B797C7FF1F83D727BE6398D4
:10A23000A70217C7FF1F231CB7BC17C7FF1F23198F
:10A24000C7BC17C7FF1F2316D7BC2E861785010072
:10A2500013054552BE85175301006700E377178544
:10A2600001001305A552176301006700C38E035751
:10A27000450097C7FF1F83D767B96318F702C16707
:10A28000F91717C7FF1F2323F7B897C7FF1F23A18D
:10A2900007B897C7FF1F238907B697C7FF1F238BF0
:10A2A00007B6170300006700E3E1178501001305F7
:10A2B000E54D176301006700038A7D15954763E24A
:10A2C000A71C178701001307E7410A053A951C41AF
:10A2D000011122CC06CEBA972E8482871785010001
:10A2E0001305454B97600100E780E086A1A203C7F4
:10A2F000250099476311F7022E8597000000E7803B
:10A3000040F783456400178501001305A549975060
:10A310000100E780606C97A7FF1F238B07F217856A
:10A3200001001305E5497DBF03C725009547631963
:10A33000F702C16717C7FF1F035747ADF91703D5CA
:10A34000A5006309F702B7E7040083A7C717829740
:10A35000178501001305C54797500100E780A07FCE
:10A36000854717A7FF1F2305F7EE17850100130583
:10A37000A5488DBF97C7FF1F239AA7A883D7E500DD
:10A3800097C6FF1F2395F6A883D7050197C6FF1F21
:10A390002390F6A883D7250197C6FF1F239BF6A617
:10A3A00097C7FF1F238207A6631BE502B7E70400D8
:10A3B000BC4F09661306069089451795FF1F034594
:10A3C000250782970356E4008355A40017850100F2
:10A3D0001305454197500100E780006051B793078E
:10A3E000700F2316F100B7E7040083A7870D1796B7
:10A3F000FF1F0346E6036C0082974DF9854717C798
:10A40000FF1F2303F7A05DB7178501001305853FE4
:10A41000D1BD83C5250091476392F50217850100E0
:10A420001305C53F97500100E780E07297000000D8
:10A43000E78040C9F2406244056182809947639297
:10A44000F502228597000000E780A0E283456400C2
:10A45000178501001305053597500100E780C057A7
:10A46000D1BF9547639AF50083471400E1F3178540
:10A4700001001305E53CBDB5178501001305C53C7A
:10A48000E1BF82803757315F9797FF1F938787FB24
:10A49000130777D598C39356C50017870100130794
:10A4A000272ABA9683C5060093568500BD8ABA96B8
:10A4B00003C6060093564500BD8A3D89BA962A9781
:10A4C00083C6060003470700238407002383D700C1
:10A4D000A383E7002382B700A382C7009797FF1FDB
:10A4E000938747F72383B700A383C7002384D7004C
:10A4F000A384E7008280411106C697000000E78030
:10A50000A0F8B7E7040083A787141796FF1F130668
:10A5100066F3D54501458297B2404D469795FF1F9A
:10A52000938545F313057030410117030000670060
:10A53000A3BE61712324811A37E404008327040831
:10A540002326111A2322911A2320211B232E31198D
:10A5500017050000130525C382971799FF1F1309DC
:10A5600029ED994785442300A900231CF100978514
:10A5700001009385E51B930740061775010013053D
:10A58000A5A5231CF1082308910097B9FF1F938903
:10A59000C91C97500100E780204483D50900178526
:10A5A00001001305E51797500100E780E0422945B7
:10A5B00097500100E780204703D50900970000006D
:10A5C000E78080EC83274417100885451305503039
:10A5D0008297832744171796FF1F1306A6E7CD45DA
:10A5E000130570308297832744171796FF1F1306B1
:10A5F00066E4B54513056030829783274417300819
:10A6000089451305103182978327441730098945FE
:10A61000130520318297832744159305000A0D45C1
:10A620008297832744159305000A11458297A30555
:10A6300091002306910002CD23080100230C0100A4
:10A64000832784163009914513057040829783272C
:10A6500084161306B10085451305004082978327B1
:10A660008416700085451305104082978327841651
:10A6700030088545130520408297832784161008EB
:10A680008545130550408297832704157D55829791
:10A69000832744137D5582977D559790FFFFE78070
:10A6A000C0FE8327440C82979790FFFFE78020DA53
:10A6B000832784141796FF1F1306C6D8D545014576
:10A6C000829789471306700F814528092306F100F8
:10A6D0009780FFFFE780A0A38D4713060008814500
:10A6E0002808230CF1089780FFFFE78040A29147DC
:10A6F000230CF100976701009387877F984383C7F6
:10A7000047003AC8230AF10097C0FFFFE78020FE08
:10A710007000854505459790FFFFE78020FE3009D2
:10A720009305700F09459790FFFFE78020FD3008E3
:10A73000930500080D459790FFFFE78020FC100867
:10A74000954511459790FFFFE78040FBC16717B71C
:10A75000FF1F1307A76BF9171CC3232207001795C8
:10A76000FF1F1305A5CC9790FFFFE78000F8832714
:10A77000C41D17B5FF1F1305E56782973C480345C5
:10A780000900854582978320C11A0324811A8324F6
:10A79000411A0329011A8329C1195D618280C167A9
:10A7A00017B8FF1F03588866F9176301F8083DCDF5
:10A7B000B5CD011126CAB7E4040083A7841222CCC8
:10A7C0002E862315B10006CE2A8401478146ED4529
:10A7D000428582972AC611ED17850100130585F77A
:10A7E00097500100E7802037F2406244D24405616F
:10A7F0008280FC440356A100A28582972C0017B5E5
:10A80000FF1F0355A5609790FFFFE780C0FA69DD41
:10A8100017850100130545F597500100E780A03327
:10A8200083A7C412ED45280082977DBF82800DC5A5
:10A8300085471797FF1FA304F7C09797FF1F238132
:10A8400007C035469795FF1F9385C5BE1305603039
:10A85000170300006700438C9797FF1FA38107BE73
:10A86000E9BF97B7FF1F83C7E75AA9EFC16717B7BB
:10A87000FF1F0357A759F9176306F70441118547CE
:10A8800022C417B7FF1F2307F75837E404007C4C96
:10A8900006C689451795FF1F034585B9829703238F
:10A8A000841A2244B2409797FF1F83C767B817B531
:10A8B000FF1F0355A5551307401F81463146994593
:10A8C0004101028382806D7123248110232611109F
:10A8D00023229110328401CD8947630AF502832037
:10A8E000C110032481108324411051618280178597
:10A8F0000100130525F6AE8497500100E780A025DE
:10A90000A285268597B0FFFFE78020E5C9BFB7E79E
:10A910000400FC472800829717850100130545F4C1
:10A9200097500100E78020238347810039C4130733
:10A93000000B6380E7021387A7051377F70F8D4697
:10A9400063EDE602A285280097B0FFFFE780205B59
:10A9500079B78547E3F587F88345910017750100BE
:10A960001305859AB335B0009797FF1F238EB772F2
:10A9700097500100E78040069DB703479100A2076A
:10A98000B966D98F1387E6556384E70C636DF704C6
:10A990002D671307B755638FE708636AF7002967C8
:10A9A0001307A755638FE708A2852800A1BF316769
:10A9B0001307C7556388E70635671307D755E3952F
:10A9C000E7FE8947E3FD87F097000000E780A0E9F4
:10A9D0009305E4FFC205C1811305A1009790FFFF15
:10A9E000E7800080EDBD3D671306F7556389C70614
:10A9F000636DF6009386E665E398D7FAA285280092
:10AA000097C0FFFFE7800093D9BD9306F766638D7B
:10AA1000D7041307F777E399E7F897C0FFFFE780BC
:10AA2000A0BE75BD0146A285280097B0FFFFE78054
:10AA3000A07875B5A285280097C0FFFFE780C08386
:10AA400079BDA285280097C0FFFFE780A08441BDA3
:10AA5000A285280097C0FFFFE780C08449B597C052
:10AA6000FFFFE7804096A5BD97C0FFFFE780E09B12
:10AA7000BDB5C16717B5FF1F03554539F917630702
:10AA8000F500B7E7040003A3C7170283828017F31A
:10AA9000FFFF670023631773FFFFE702A3622A84A7
:10AAA00008452E89B28919C900C197150000938500
:10AAB000A586610597300100E780200581447D5A15
:10AAC00097100000E780E03963C7A4048144971021
:10AAD0000000E780003A63C8A40497B7FF1F93877C
:10AAE000A7339C43DC47B307F94091872302F40066
:10AAF000638309048327C900B307F4409587A30241
:10AB0000F4001C4C89C79C4799C322858297177310
:10AB1000FFFF6700635E5C44139714008504BA97D7
:10AB20002390470171BF1C48139714008504BA97FE
:10AB30002390070069BF832789000547B307F440C6
:10AB40009587A302F40083570400638EE7028DC348
:10AB500009476384E7040D47E395E7FA9787010007
:10AB60009387C7221CCC978701009387272311A8BE
:10AB700097870100938707E91CCC9787010093878B
:10AB800067E95CC8BDBF978701009387A7D41CCC39
:10AB900097870100938707D5EDB7978701009387C3
:10ABA000A7231CCC9787010093870724D9BF95E57D
:10ABB0001773FFFFE702A35200461844834794002F
:10ABC00075839D8B6317F70097100000E78060B4D2
:10ABD00048C41773FFFF6700C35282801773FFFFDB
:10ABE000E702434E13893500C16442094111AA8925
:10ABF0000144F11413590901054A2EC697100000AB
:10AC0000E7802026B2456348A4000145410117733F
:10AC1000FFFF6700634E83A7090013171400BA975C
:10AC200083D707006388B7006394970063742A0191
:10AC30000504E1B70545D9BF1773FFFFE702A34736
:10AC4000AA892E89328BB6843A8ABE8A97A00000E0
:10AC5000E780C0FE71C9268597200000E780C00C00
:10AC60008D4763E7A7007D551773FFFF67002348F3
:10AC700083DB440097100000E780A0242A8497100B
:10AC80000000E780402593077400314433058502B6
:10AC900063CDA70297100000E780A0229710000064
:10ACA000E78020222A8497100000E780C0229307C3
:10ACB000740031443305850263C3A7049710000074
:10ACC000E78020209307450029A897100000E7801F
:10ACD0008020330585021307F0179307C017E35F41
:10ACE000A7FA2D55E3C277F963040B02D686528684
:10ACF000A6854A8597200100E780C0BDB5B79710AB
:10AD00000000E780401D330585029307C5FFD1BFD2
:10AD1000832749001385C90083D5270097000000C9
:10AD2000E78000EC61F581B769553DBF97B7FF1F1C
:10AD30002396A70E97B7FF1F9387070E904381476F
:10AD40000C463307F500420741836393B7008280C6
:10AD50005446139847008507C2962390E600D5B75E
:10AD600097B7FF1F9387470B9C4303C587008280DB
:10AD700017B5FF1F0355850A82801773FFFFE7028F
:10AD80000336C1671387D7FF630BE502636AA70029
:10AD9000F1176300F50201451773FFFF6700633683
:10ADA0001387E7FF6302E502FD171D8D13351500BC
:10ADB000E5B797500000E780602A7D15C5BF975022
:10ADC0000000E780E0FED5BF97500000E78000FD5F
:10ADD000EDB71773FFFFE70283304111AA840144E6
:10ADE0002EC697100000E780C008B2456348A40053
:10ADF000014541011773FFFF6700A3309C481315FD
:10AE000014003E9583570500E385B7FE0504C9BFCE
:10AE100003485500814693F7F60F63E50701814724
:10AE20003E858280584593975600BA9703D72700EE
:10AE30006316B70003D70700E304C7FE8506E1BF2A
:10AE40008346450001479377F70F63E4D7008147B6
:10AE500011A81C45131657000507B29703D6070023
:10AE6000E313B6FE3E8582801773FFFFE70283255A
:10AE700093170501C18797BAFF1F938AEAF9635BAD
:10AE8000F00883A70A00C0479C4703570400198DA8
:10AE9000420541816368F500014422851773FFFF75
:10AEA0006700832512052A94CDBFDC47139449001F
:10AEB000014A3E94834744006341FA02014A8347B2
:10AEC00054006349FA028509C20993D9090183A78D
:10AED0000A009847E3EBE9FCC1B71C4413195A0078
:10AEE000A6853E994A8597000000E780C0EE05E1FF
:10AEF000050AC9B75C4413195A00A6853E994A85CC
:10AF000097000000E78020ED19E1050A4DBFE30C32
:10AF100009FA61B7AA8481495DBF1773FFFFE70291
:10AF2000031C1C452A8481E79307C5001CC51C44EB
:10AF3000231204001CC09307F00F63EDB70093F5D4
:10AF4000F50F228597200000E780C0E51773FFFF0B
:10AF50006700231B93940501C167C18063F9F50065
:10AF6000A685228597200000E780E0E8C5B7C1816B
:10AF700093F5F50F228597200000E780A0E2A685D3
:10AF8000228597200000E780E0E3C9B797B7FF1F4D
:10AF9000938787E8884382801C4599C797B7FF1F2E
:10AFA00023ACA7E6014582807D55828097B7FF1FBD
:10AFB000938787E6984383474500484792073E9525
:10AFC00082801773FFFFE7028311617100451C182F
:10AFD0003EC6B70780013EC81C183ECA83574400CE
:10AFE00002CE02D002CC231EF100834784002A89BE
:10AFF00002D22301F1023C083ED402D697000000A1
:10B00000E78000FB835705002316F10297500000EC
:10B01000E78000C82307A1025C4003556400F18368
:10B0200013F717008347F10252055181F99BD98F1D
:10B03000A307F10297100100E780207939CDAA8497
:10B040000355050097A00000E78020C083D70400C7
:10B050002AD26800231CF10083D72400231DF100AD
:10B060001C4803D647008C4397200000E780A0D0FF
:10B070008347B400CA86177601001306267F81171E
:10B08000A305F4006C00481097200100E78080843D
:10B090005D611773FFFF6700C3062155D5BF1C45CF
:10B0A000B1CF03C5A700894613576500630BD702CC
:10B0B0008D46630ED70285466300D702130740060C
:10B0C0003305E50203C7B700418B15CB83C7B70033
:10B0D000BD8B3355F54082801375F5031307803E11
:10B0E000C5B709671375F50313070771D1BF372774
:10B0F00009001375F5031307077CD9B70145828052
:10B100001773FFFFE702A3FD03A98500630C090481
:10B110008347B900AE8493F7070E85C303459900B2
:10B12000930520030D810505B305B502884461052B
:10B1300097300100E78080AD35A02E859700000094
:10B14000E78020F62A8419CD97000000E780605C34
:10B150008325C900B307B54063FA87002E94B30571
:10B16000A440E9F51773FFFF6700A3F985457DBF8C
:10B170001773FFFFE702A3F62A8403D50500011128
:10B1800032C636C43AC22EC002CA02CC02CE97A042
:10B190000000E78080AB82452ACA22852ECC97002A
:10B1A0000000E780E0E003570500231EE100975010
:10B1B0000000E780E0ADA24632469247230FA1008F
:10B1C00036874C08B2862285014697000000E7804A
:10B1D000E0A605611773FFFF6700A3F21773FFFF77
:10B1E000E702E3EF61711C183EC6B70780013EC855
:10B1F0001C183ECA3C0800453ED4AA8402CC02CEAC
:10B2000002D002D202D697000000E78060DA8357AE
:10B21000050035592316F10297500000E78040A73A
:10B220002307A10209C48357440081EB21594A85B1
:10B230005D611773FFFF6700C3EC0355640052059F
:10B24000518197100100E78040582A8965D18347D2
:10B25000B40093F7070E99C71305840197300100D6
:10B26000E780009D83574400231EF100834784003C
:10B270002301F1025C4003550900D98313F7070845
:10B2800083471102231CA10093F7F707D98FA3006E
:10B29000F10283572900231DF1005C40F18313F76D
:10B2A00017008347F102F99BD98FA307F10297A0FA
:10B2B0000000E78080992AD235D98347940068003E
:10B2C000139757008347B400FD8BD98FA305F40073
:10B2D0001C4803D647008C4397200000E780A0A9B4
:10B2E000A6871777010013076758740005464C10AE
:10B2F000268597000000E78060942A890DD983474E
:10B30000B400A685FD8BA305F40097000000E7803C
:10B3100060DF31BF1773FFFFE70263DC832485FE24
:10B320002A844111268597000000E78080D7834753
:10B3300034FF93F7070E8DCB2AC6268597000000B1
:10B34000E78060C809CD834734FFB245FD8BA30970
:10B35000F4FE91C5228597300100E780208B4101E2
:10B360001773FFFF6700E3D97DD98327C4FF2685C4
:10B37000829775F5834734FF93F7070E91C72285AF
:10B3800097300100E780C08A032584FE9700000003
:10B39000E78000E5E9B71773FFFFE70243D19C415F
:10B3A00041112A8903C7070089472E8493566700F5
:10B3B0006380F6040D466388C6049307F0076304B0
:10B3C000F7022E8597200000E78060ABAA848149B0
:10B3D000C16B130C490097B7FF1F9387E7A39C43EA
:10B3E000984763E4E90441011773FFFF6700E3CF67
:10B3F00003D745008547E3F8E7FE2E859720000038
:10B40000E78040ADE1B703D74500E3FEE7FC2E85BA
:10B4100097200000E780A0A6AA842285972000003C
:10B42000E78000A8C204C98C5DB7DC470355A900BA
:10B43000139A49003E9A93170501C187635DF00096
:10B4400083570A006397A70263E774038327CA0040
:10B45000034D5A002DA0A1672167A98F1307F7EFAD
:10B46000E374F7FE6397090097000000E7802091DE
:10B4700061FD85098DB783278A00034D4A00835DEE
:10B48000A90003576900216A138BC7003AC6814A95
:10B4900033CA4D01631E5D0197B7FF1F938747981D
:10B4A0009C43E1DBA2866286814526858297D1B7DF
:10B4B000A1679387F7EF930C4BFF63F24703B24505
:10B4C0005A8597F0FFFFE780A0710DC103278B001D
:10B4D000104709CE10436382C4023107D5BFEE8501
:10B4E000668597000000E780008F71F993861A0047
:10B4F00093FAF60F130B0B0271BF835644005C43A3
:10B50000E3E9F6F622853AC697200000E78020811D
:10B51000A1679387D7042A8A035D4400324763E812
:10B5200097008347D90093E707F8A306F9001C4763
:10B5300066852286E2858297C1670844FD17337AC3
:10B54000FA00529508C02312A40125B797B7FF1F30
:10B550009387878C9843814715C31447814763FFBE
:10B56000D500939745004C47BE9519C903C75500B0
:10B5700081476375E600DC451606B2973E858280FA
:10B5800003C745008147E37BE6FE16069C45F5B7F9
:10B590001773FFFFE70203B3AA892E8A814497BA83
:10B5A000FF1F938A6A8783A70A00984763E6E4002F
:10B5B0001773FFFF670043B4DC471394440001494D
:10B5C0003E9413BB140083474400634BF9000149C8
:10B5D00013BB140083475400634FF9008504E1B79F
:10B5E0000844931759005287DA860146A2853E9592
:10B5F00082990509C9BF4844931759005287DA86D2
:10B600000546A2853E9582990509E9B71773FFFFA4
:10B61000E702E3AC814517F5FFFF1305054897A73F
:10B62000FF1F239D077E97000000E780A0F6177399
:10B63000FFFF670003AD97A7FF1F9387E77D9C433C
:10B6400095C31773FFFFE70283A9814517F5FFFF35
:10B650001305A54497000000E780C0F31773FFFFB0
:10B66000670023AA82801773FFFFE702A3A537E4D0
:10B6700004008327841241112315E100AE89328929
:10B68000368A3A8681460147ED45AA8482972AC6C2
:10B6900021C90356A100D28597400100E7806028A8
:10B6A0008327C413CE8526858297058905C98327FC
:10B6B000440D2314210101462C00268582972A84FB
:10B6C00001C9B7E7040083A7C712ED452800829798
:10B6D000228541011773FFFF670003A24944D5B7D4
:10B6E0006554FDB75C41FD175CC182801773FFFF95
:10B6F000E702E39EB7E70400FC5F829795473305B6
:10B70000F50281450D811773FFFF6700839F177353
:10B71000FFFFE702C39CB7E70400FC5F82979547F1
:10B720003305F5020D811773FFFF6700839D1773C3
:10B73000FFFFE702C39AB7E7040083A7870B03550F
:10B74000050082971773FFFF6700A39B1773FFFF26
:10B75000E702E398035505003287AE861786FF1F80
:10B76000035666D597A5FF1F9385C56B970000000C
:10B77000E780A0EF1773FFFF6700A3981773FFFF21
:10B78000E702E395B7E7040083A7C717829717730B
:10B79000FFFF670003971773FFFFE7024394B7E7C4
:10B7A000040083A7871397A5FF1F9385A56782973A
:10B7B00001451773FFFF6700C3941773FFFFE7028C
:10B7C0000392B7E7040083A7C71F81451785FF1FB2
:10B7D000035565CA82971773FFFF6700839217733B
:10B7E000FFFFE702C38FB7E7040083A7871397A57E
:10B7F000FF1F93852564829701451773FFFF67003C
:10B8000043901773FFFFE702838DB7E7040083A718
:10B81000C71F81451785FF1F0355E5CB8297177317
:10B82000FFFF6700038E1773FFFFE702438B2E8530
:10B8300097800000E78080B397800000E78080F069
:10B840001773FFFF6700E38B1773FFFFE70223897E
:10B8500097800000E78080FA1773FFFF6700638A14
:10B860005C49E1175CC95CC583572501A107231911
:10B87000F50083570501A1072318F5008280F147E1
:10B880003305F50297A7FF1F9387C75C9C433E953E
:10B8900082808D476315F60803D74600854763F01D
:10B8A000E7081773FFFFE7028383368536842E8906
:10B8B00097100000E780A05C29C9835744009314C7
:10B8C0000501C18063E39704228597100000E7809B
:10B8D000005BFD14231294009307A0026300F5029D
:10B8E0009307B0026307F50293079002631FF50008
:10B8F000228597000100E780608901A80146CA857A
:10B90000228597A00000E78000B41763FFFF67005F
:10B91000437F228597100000E7806007FDB7828093
:10B9200097A6FF1F938646539C42014599CF9843A3
:10B93000D44217A6FF1F2321E6526396D70097A68D
:10B94000FF1F23ADE6501385C7FE82801763FFFFFC
:10B95000E702E37897000000E780A04B71443305CD
:10B960008502914597900000E780C0EC11E5655590
:10B970001763FFFF6700E37897A7FF1F23AAA74C71
:10B9800097000000E780E0483305850291459790D5
:10B990000000E78020EA61DD97A7FF1F23ACA74ADC
:10B9A00097000000E780E04697A7FF1F239CA74869
:10B9B00097000000E780E04597A7FF1F2395A74861
:10B9C000977701009387C7EF17A7FF1F2320F7483A
:10B9D00097070000938707E917A7FF1F2326F7465D
:10B9E000014579B71763FFFFE702636FAA8517A5C3
:10B9F000FF1F1305254597100000E780605F176360
:10BA0000FFFF670003701763FFFFE702436D9700B6
:10BA10000000E78060FD97100000E780E05E97A7D8
:10BA2000FF1F938767439C4391CF1387C7FE19CBB2
:10BA300083D5C7FF17A5FF1F130585429720010077
:10BA4000E780C01C1763FFFF6700A36B1763FFFF4E
:10BA5000E702E36897000000E780C0EC09CD834768
:10BA600085002A8493F7070499EB0355E5009700B6
:10BA70000000E78080F91763FFFF67008368834752
:10BA8000C5009304450117A9FF1F1309E93C85E38D
:10BA9000832709005CC997A7FF1F23AF973A832725
:10BAA0004900F1FB97A7FF1F23AA973AE9B7FD17B3
:10BAB0002306F500610597800000E78060DA8307C0
:10BAC000840063CB07048347840093E707F82304CB
:10BAD000F400B7E704009C5F82974205A9474181C3
:10BAE0003375F5028347840093F707FCC98F23045D
:10BAF000F4008347D4003E951C402318A40089CF4E
:10BB0000984319CB8347C4005040814585073305CE
:10BB1000F502420541810297832709005CC897A777
:10BB2000FF1F23AB97328327490089E797A7FF1FA1
:10BB300023A697328347C4009DDF8355040117A5D0
:10BB4000FF1F1305E53197200100E780200C25B782
:10BB50001763FFFFE702A35897A7FF1F9387875537
:10BB60009C4701448583858B85E3AE84B2853A8604
:10BB700097100000E780204F2A8419C59710000015
:10BB8000E7806045829408CC22851763FFFF670039
:10BB900043571763FFFFE702E35241112E8932C674
:10BBA000AA8997000000E780C031324713060502DA
:10BBB000CA86970500009385C5CC17A5FF1F1305FE
:10BBC000652897000000E780E0F82A8425C99304DF
:10BBD000C50097000000E780E0411946AA85268548
:10BBE00097100000E78020198545268597100000F2
:10BBF000E780001517750100130545CA4E9583456A
:10BC00000500268597100000E780C0195C48314682
:10BC10008145A1075CC85CC483572401E11723193F
:10BC2000F40083570401E1172318F4001C4C3E85EF
:10BC30009760FFFFE780A04DA30425012285410105
:10BC40001763FFFF6700434B1763FFFFE7022349BA
:10BC50004111AA842EC632C497100000E780003A32
:10BC6000004DB2452246834784000CC050C093F774
:10BC7000F70393E707042304F40023180400268540
:10BC800097100000E780203583479400A9462317CA
:10BC9000A40013D7370005073307D7029D8B85070C
:10BCA0002306F400A306E40083C70401D8488507EF
:10BCB000230FF7FE17A7FF1F1307071A5843232A5E
:10BCC00004009307440129E317A7FF1F2328F7184F
:10BCD00017A7FF1F2322F71817A4FF1F13044418E8
:10BCE000228597200100E780A0E41C44858B5D8DB0
:10BCF00019E58145228597200100E78020F1410167
:10BD00001763FFFF6700E33F1CC317A7FF1F23272D
:10BD1000F714D9B71763FFFFE702633C97050000EC
:10BD2000938565B7014597000000E78000B00145A5
:10BD30001763FFFF6700E33C1763FFFFE702233A47
:10BD400097000000E78080B01763FFFF6700633B48
:10BD50008347C500A5E31763FFFFE70243382A8442
:10BD60000355E50097000000E78000C821C1834724
:10BD7000840093F7F7FB2304F4001C4091C7DC43D5
:10BD800081C74C400145829797000000E78080B949
:10BD900017A5FF1F1305C50C97200100E78040E998
:10BDA0000355E40097000000E78020C61763FFFFFB
:10BDB0006700233582801763FFFFE702433297A7AE
:10BDC000FF1F9387670997050000938565C817A52E
:10BDD000FF1F1305E50823A0070023A207009720F3
:10BDE0000100E78080D21763FFFF670083311C4D9D
:10BDF00091CFDC4381CF1763FFFFE702432E8345DA
:10BE0000070082971763FFFF6700A32F828097A721
:10BE1000FF1F938727079C4303C50700828097A7CE
:10BE2000FF1F938727069C4303C51700828097A7AF
:10BE3000FF1F938727059C4303C52700828097A790
:10BE4000FF1F938727049C4303C54700828097A761
:10BE5000FF1F938727039C4303C53700828097A762
:10BE6000FF1F938727029C4303C55700828097A733
:10BE7000FF1F938727019C4303C56700828097A714
:10BE8000FF1F938727009C4303C57700828097A7F5
:10BE9000FF1F938727FF9C4303C58700828097A7D6
:10BEA000FF1F938727FE9C4303C59700828097A7B7
:10BEB000FF1F938727FD9C4303C5A700828097A798
:10BEC000FF1F938727FC9C4303C5B70011E11D4565
:10BED000828097A7FF1F9387E7FA9C4303C5C7009B
:10BEE000828097A7FF1F9387E7F99C4303C5D7007C
:10BEF000828097A7FF1F9387E7F89C4303C5E7005D
:10BF0000828097A7FF1F9387E7F79C4303D507011C
:10BF1000828097A7FF1F9387E7F69C4303C52701FD
:10BF2000828097A7FF1F9387E7F59C4303D54701BE
:10BF3000828097A7FF1F9387E7F49C4303D567018F
:10BF4000828097A7FF1F9387E7F39C4303D5870160
:10BF5000828097A7FF1F9387E7F29C4303C5A70141
:10BF6000828097A7FF1F9387E7F19C4303C5B70122
:10BF7000828097A7FF1F9387E7F09C4303C5C70103
:10BF8000828097A7FF1F9387E7EF9C4303C5D701E4
:10BF9000828097A7FF1F9387E7EE9C438857828094
:10BFA00097A7FF1F938707EE9C4303D5C7028280A4
:10BFB00097A7FF1F938707ED9C4303D5E70219E17D
:10BFC0001305800C828097A7FF1F9387A7EB9C43E4
:10BFD00003C50703828097A7FF1F9387A7EA9C43A7
:10BFE000C85B828097A7FF1F938747E988438280B9
:10BFF00097A7FF1F9387C7E88843828019E17D5583
:10C000008280F5DE984265DFFDD917A7FF1F130771
:10C01000670A1847AA877155058B631D072403C556
:10C0200007001547E37DA7FC03C737001305F0059C
:10C030007D171377F70FE364E5FC03C35700E300B4
:10C0400003FC83C86700E38C08FA03C777004945FF
:10C0500079171377F70FE364E5FA03C7A7001148D0
:10C060001305F7FF1375F50FE36BA8F803CE9700E0
:10C070000D481305FEFF1375F50FE362A8F803C81A
:10C08000B7006309080065181378F80F1305600DF1
:10C09000E36705F703C5C700794879151375F50FF0
:10C0A000E36FA8F403C8D7000D457D181378F80F87
:10C0B000E36705F503D80701930E401751184208AE
:10C0C00013580801E3ED0EF303C8E7007D18137859
:10C0D000F80FE36605F303C827017D181378F80FFE
:10C0E000E36F05F103C88700C54E75181378F80F84
:10C0F000E3E70EF103D86701856E938EBEE06D18FD
:10C10000420813580801E3EC0EEF03D847016D18FD
:10C11000420813580801E3E40EEF03D887017918A9
:10C12000420813580801E36C05ED03C8A7017D1808
:10C130001378F80FE36505ED03C5B7011D487D15BC
:10C140001375F50FE36DA8EA03C5D701714879159A
:10C150001375F50FE365A8EA03D5E7011308E00FAF
:10C160007D1542054181E36CA8E803C507024948F3
:10C1700079151375F50FE364A8E8C85301C937C8EA
:10C1800034005915130858BFE36BA8E603A88702CB
:10C1900037C53400130555BF5918E36205E717A5E5
:10C1A000FF1F232FC5CC03C6050117A5FF1F232B97
:10C1B000F5CC0545E375C5E403D82501D0493376B0
:10C1C0000603E31E06E203C61501E30A06E217A60C
:10C1D000FF1F2325B6CA83C5270001466387A50034
:10C1E00003C61700F1453306B60283C7070393055C
:10C1F000C00272971A071307C70516031A97960805
:10C200004697B387B70241553E973297420741831D
:10C210006362E8061763FFFFE70263EC36859780E9
:10C220000000E780406C97000100E780C04B2A8443
:10C2300097A00000E780205E2A9497F00000E78036
:10C24000002A2A9497900000E78040852A9497F06E
:10C25000FFFFE780E06F2A9497400000E780009797
:10C260002A9497700000E78040A022951763FFFF93
:10C27000670023E982801763FFFFE70243E641116D
:10C28000A307A10097A00000E78040C99305F10033
:10C29000170500001305E5B597F0FFFFE780802F35
:10C2A000014541011763FFFF6700A3E51763FFFF27
:10C2B000E70263E017A4FF1F1304C4DF0328840010
:10C2C00079599368180097A4FF1F23A914DF1378E6
:10C2D000180063100802BA84BE89368B328A2E8910
:10C2E000AA8A97F0FFFFE780E0A77D15269519E55C
:10C2F00031594A851763FFFF670063DF97F0FFFF3F
:10C30000E78040A67D152695A167E353F5FE97A724
:10C31000FF1F9387271198433E8C814B01CB01452A
:10C3200097F00000E780C047933B15004A85DA8606
:10C330005686D28597900000E78060512A8911CDFA
:10C340001C44F99B17A7FF1F232AF7D683270C004D
:10C35000CDD3E3800BFA829769BF268597A7FF1F8D
:10C3600023AC07D497F0FFFFE780809C4146CE8541
:10C3700017A5FF1F130585DD97300100E780605A80
:10C3800097D00000E780E09C0325040B97D00000C5
:10C39000E780A0A0054597D00000E780A0A705454D
:10C3A00097000000E78060EDA9B797A7FF1F93876C
:10C3B00067D09C47858BEDC71763FFFFE70223D249
:10C3C00017A5FF1F1305C5D697A7FF1F23A407CEE8
:10C3D00097A7FF1F23A207CE97A7FF1F23A007CE73
:10C3E00097200100E780C08497500000E78080F923
:10C3F00097100100E780405097100100E7804056F9
:10C4000097A7FF1F938787C99C4391C705459780CE
:10C410000000E780E02397A7FF1F9387E7B19C43C5
:10C4200099C741657D1597700000E780E0A597F0FA
:10C430000000E780804197D00000E780209397A715
:10C44000FF1F938727DC9C43139717016356070050
:10C4500097F00000E780A0B097A7FF1F23A807CEA2
:10C4600097A7FF1F23A607CE97A7FF1F23A407CEDA
:10C4700097A7FF1F23A207CE97000000E780008C3C
:10C4800097000000E780A07597F0FFFFE780401855
:10C4900097F00000E780E0D91763FFFF670063C6ED
:10C4A000828097A7FF1F9387E7C08843828097A762
:10C4B000FF1F938727C0C8438280B7E7B0009387E8
:10C4C000075063E1A70297A7FF1F9387A7BED84332
:10C4D000FD576367E50097A7FF1F23AFA7BC814700
:10C4E0003E858280B957EDBF1763FFFFE70223BF88
:10C4F00097800000E780607597800000E780C07734
:10C500001763FFFF6700E3BF1763FFFFE70283BB0B
:10C510002A849304140201112E85B289A68521462E
:10C5200036C63A8997300100E780403D0DE9B246B2
:10C5300038082686CE851305940497500000E780BE
:10C54000604121462C084A8597300100E780003B76
:10C550001335150005611763FFFF6700E3B9014557
:10C56000D5BF1763FFFFE70283B79305450617A5FD
:10C57000FF1F1305659197100100E780206917637D
:10C58000FFFF670003B81763FFFFE70243B54111E0
:10C590002EC697F0FFFFE780C017B24588C1410162
:10C5A0001763FFFF6700E3B51763FFFFE70283B17F
:10C5B000AA842E8497800000E780006CAA898545B4
:10C5C000228597000000E780E07D83C7E40113899E
:10C5D000940899E313890403CE852285970000000F
:10C5E000E780407C214693051902228597000000D0
:10C5F000E780607897A7FF1F9387C7AB8C4322859E
:10C6000097100000E780C08221469385840222852E
:10C6100097000000E78020761763FFFF6700C3AD37
:10C620001763FFFFE70223A9397197F00000E78045
:10C63000E0B49305400661E997800000E780006060
:10C640006302051497A7FF1F83C7C78513B7170099
:10C6500097A6FF1F2388E684014499CFC16417A9D8
:10C66000FF1F130929A59309400EFD149700000030
:10C67000E78020836342A40A97F0FFFFE780600908
:10C680004169B7290900096AFD7A2A8B81447D191D
:10C690009389F97B130A0A71938A8AC7970000006D
:10C6A000E780208063D7A4041304400EB38784027C
:10C6B00017A7FF1F130707A00324070B3E948357F8
:10C6C000C4016382270B18403307EB4063EAE9009B
:10C6D000834744008507B3874703D6976365F70808
:10C6E00001468145094597F0FFFFE780C04AAA8BC4
:10C6F00029E597400000E780808385476317F506AA
:10C700008965938505711795FF1F1305E5779710C8
:10C710000100E780A04F95A0B30734030327090B5E
:10C72000BA9703D7C7016308970003C75700A382CE
:10C7300007002382E700050415BF9305C500228585
:10C7400097000000E78080E65E85228697650100FD
:10C750009385051697F0FFFFE780404F5E859710A1
:10C760000000E780608A850415BF97A7FF1F9387A5
:10C7700067949C478D83858BC1F721611763FFFF09
:10C780006700E39601468545094502D002D202D4EE
:10C7900002D697F0FFFFE7800040AA8479DD97F08A
:10C7A0000000E780E09C1389C4002A8481454A8503
:10C7B00097000000E780005F0C4041464A859700E3
:10C7C0000000E780405B832944006385090C4E85A7
:10C7D00002D802DA02DC02DE97300100E780E0389E
:10C7E0002ACE141005462C0808184ECC975000008D
:10C7F000E780E00A1375F50F51ED8355840093E54A
:10C8000025004A8597000000E780E05E11460C1085
:10C810004A8597000000E7800056014697650100B1
:10C8200093858509268597F0FFFFE78020422685BE
:10C8300097000000E780407D5C40A1D3014685451C
:10C840000D4597F0FFFFE7800035AA841DD54840CD
:10C850001389C40097300100E78020312AC64A8539
:10C8600097000000E780404C3246636FC5004C40A3
:10C870004A8597000000E7800050014681452685E3
:10C8800097F0FFFFE780803C268597000000E78057
:10C89000A077E5B583558400ADB71763FFFFE702C6
:10C8A000038497A7FF1F9387E7809C471DC193E7E9
:10C8B00087001795FF1F1305255D1797FF1F232F6F
:10C8C000F77E97100100E78040321763FFFF670093
:10C8D0004383DD9B1797FF1F2322F77E97300000CD
:10C8E000E780E0647DF11795FF1F1305E559971068
:10C8F0000100E780E033D1BF1753FFFFE702A37BBE
:10C900004169AA892E8AB28A368BBA8B8144179CD8
:10C91000FF1F130C2C7A930C400E7D1997F0FFFF2C
:10C92000E780205863C4A40001443DA033849403ED
:10C9300083270C0B3E948357C401638627055A87CF
:10C94000D6865286CE851305040397000000E78043
:10C95000E0BB01C923800B0022851753FFFF67004E
:10C9600003798347F40185C35A87D6865286CE85DC
:10C970001305940897000000E78040B909C5854772
:10C980002380FB00D1BF850451BF835745006380DE
:10C99000071E1753FFFFE702E37201112A84970075
:10C9A0000000E780C04D09C985476309F5060561A8
:10C9B0001753FFFF6700437497E00000E780007C97
:10C9C0007DF5835744004947ED9BE392E7FEC1455F
:10C9D000228597000000E7804033AA8422859700D3
:10C9E0000000E780204F0357440002CE91472A8978
:10C9F000631AF700228597000000E780A0513C08E9
:10CA00002ACC3ECE97E00000E78080765C55C5D307
:10CA100074084A86A6850545829751BF035744008E
:10CA2000D147E3F6E7F8032A0400C1690149979A60
:10CA3000FF1F938A2A68130B400EFD1997F0FFFF22
:10CA4000E7802046634FA90E2285032A0400970041
:10CA50000000E780C042A1452A8922859700000096
:10CA6000E780A02AAA84228597000000E780804AF8
:10CA700014402A86AA8978082685CA85970000006E
:10CA8000E780C0E7AA8405D503C7F4018947631589
:10CA9000F7008347C10181DF5546D28513856400C5
:10CAA00097300100E780E0E7014597800000E780CC
:10CAB000C01901C583D7C401A5E79797FF1F9387C6
:10CAC000675F9C4793551900858913D73700058BFD
:10CAD00001CF8983858B6399B70001452EC69700E6
:10CAE0000000E780C0DBB2454E8597800000E780FC
:10CAF000601F0346C1012A8493751900268597900B
:10CB00000000E780E03935C1268597800000E78086
:10CB1000E018268511C0014597800000E780004C91
:10CB200097300000E780A0408547E312F5E883C70F
:10CB300054001307F00FE38CE7E68507A382F400A7
:10CB4000BDB5B304690383A70A0BBE9483D7C401A0
:10CB5000638B37015546D2851385640097300100F9
:10CB6000E780C0D955DD0509D1BD5DD86DB782809C
:10CB70001753FFFFE702035597800000E780000C82
:10CB800005C1C16401441799FF1F1309A9529309F4
:10CB9000400EFD1497F0FFFFE780A030634EA40025
:10CBA0001795FF1F1305452E97100100E780E0033E
:10CBB0001753FFFF67004354330534038327090BE2
:10CBC0003E958357C501638897002312050097801F
:10CBD0000000E780A00C050475BF9797FF1F93879F
:10CBE000674D9C478D83858B8DE31753FFFFE702CD
:10CBF000034F1795FF1F1305252997100100E780A4
:10CC000020031753FFFF6700C34F82801753FFFFB6
:10CC1000E702E34C970500009385C5A01795FF1F19
:10CC20001305852697100100E78020EE1753FFFFBC
:10CC30006700234D1753FFFFE702634A8841B7E7B8
:10CC40000400BC5B050542054181829709C5854703
:10CC50002300F50005051753FFFF6700834A83C7CC
:10CC6000F5FF2E858507A38FF5FE828083C7F5FF2C
:10CC7000FD1793F7F70FA38FF5FE99EF1753FFFFFB
:10CC8000E702E345B7E70400BC571385F5FF829739
:10CC90001753FFFF6700E34682801C41035745009E
:10CCA0008D8FBA951CC12312B5003E85828093D723
:10CCB0008500A2051441DD8D835745001387E6FFEB
:10CCC00018C189072312F50013D685004111238F5F
:10CCD000B6FEA38FC6FE4101828018419307F7FF7D
:10CCE0001CC18357450085072312F500A30FB7FE2B
:10CCF0008280835745008D8F2312F5001C41BE951D
:10CD00000CC12E858280AA8703D7470008410D8F6A
:10CD1000AA952392E7008CC3828018410845330509
:10CD2000A740828083574500035765001D8F1C4133
:10CD300008453385A7403305A74082801753FFFF7E
:10CD4000E702E33941112EC62A8497000000E780EC
:10CD5000A0FDB2456373B50001A0835744000840AD
:10CD6000BE952312B4003E9541011753FFFF6700A3
:10CD700043391753FFFFE702833641112E84B285F2
:10CD800032C697000000E780A0FB3246A2859730AC
:10CD90000100E78000B941011753FFFF67006336C8
:10CDA0001753FFFFE702A3332E8485459700000049
:10CDB000E78000F9230085001753FFFF6700633405
:10CDC0001753FFFFE702A33141112317B100894533
:10CDD00097000000E780C0F68347E1002300F500DC
:10CDE0008347F100A300F50041011753FFFF6700DF
:10CDF00043311753FFFFE702832E93D78500A20527
:10CE00004111DD8D2317B100894597000000E780AF
:10CE100020F38347E1002300F5008347F100A300DE
:10CE2000F50041011753FFFF6700A32D1753FFFFC4
:10CE3000E702E32A1397850193D78501C16693869C
:10CE400006F0D98F13D78500758FD98FA2053707C4
:10CE5000FF00F98D4111DD8D2EC691459700000030
:10CE6000E78000EE6C00114697300100E78060AB70
:10CE700041011753FFFF6700C3281753FFFFE70265
:10CE800003261C41854503C4070097000000E78086
:10CE900080E622851753FFFF6700A3261753FFFF85
:10CEA000E702E3231C414111894503C7070083C7FB
:10CEB00017002307E100A307F10097000000E780B7
:10CEC00080E30355E10041011753FFFF670063232F
:10CED0001753FFFFE702A3201C414111894503C7F7
:10CEE000070083C717002307E100A307F10097009D
:10CEF0000000E78040E08357E100410113D587003F
:10CF0000A2075D8D420541811753FFFF6700631F34
:10CF10001753FFFFE702A31C0C4141112A8411465D
:10CF2000680097300100E780C09F914522859700F7
:10CF30000000E78040DCB247C166938606F0139795
:10CF4000870113D58701598D13D78700758F598DA8
:10CF5000A2073707FF00F98F5D8D41011753FFFFCF
:10CF60006700231A1C45BE950CC18280AE8794438E
:10CF700091E6584101EF0CC15CC1828003C75700A4
:10CF800013671700A382E700B687D5B70CC3EDB7C8
:10CF9000AA87084119CD1841D44398C36313D5001B
:10CFA000D8C32A87034657009376160081E62320CC
:10CFB00007008280944381CA8C4203A847008CC337
:10CFC00063930601CCC3799A14C3A302C7003687C2
:10CFD000D1BF1C45DC471D8DB777DBB6938777DB68
:10CFE00009853305F502420541818280F147B38509
:10CFF000F50248452E958280834745008507230228
:10D00000F50082801753FFFFE702630D2A8409E4CD
:10D010001753FFFF6700E30E83474400F5DBFD175E
:10D0200093F7F70F2302F400E5F71C4403D727001A
:10D0300005072391E700DC4399C3228582974C487A
:10D0400089CD83475400898B99E71C4422859C47EE
:10D050009C439C478297232A04000040232004001D
:10D060007DB71753FFFFE702830783572500411160
:10D070002EC681EB0144228541011753FFFF670053
:10D080004308035705008147F146E305F7FEB385E2
:10D09000D702404585072E948345440008C4F5F522
:10D0A000B247AA8481E7232A040009A81C456C0022
:10D0B00022859C439C43829748C84DDD85472312B7
:10D0C000F400B24723200400231804002319F400BD
:10D0D0005C485CC483D72400FD172391F40061BF32
:10D0E0001753FFFFE702A3FF9797FF1F9387C7DB45
:10D0F00088432326050023240500410597100100DD
:10D10000E78000B31753FFFF6700A3FF1753FFFF2C
:10D11000E702E3FC1794FF1F130404D91C404111DC
:10D1200099CF9C472300B5002AC65CC19700000038
:10D13000E78040FB1C40DC4399C3324582974101A4
:10D140001753FFFF6700E3FB0347450029E3584DF2
:10D15000AA877D551DCF1753FFFFE70243F81CC375
:10D16000DC479796FF1F23A1E6D4F156130507016C
:10D170002390D700970500009385050297100100C2
:10D18000E780A09801451753FFFF670083F77D559F
:10D19000828082801753FFFFE70263F4011161462A
:10D1A000814528009750FFFFE78060F69797FF1FA3
:10D1B000938787CF9C4328009305F00FDC473EC63A
:10D1C00097000000E780C0F405611753FFFF670078
:10D1D00043F39797FF1F938727CD9C43D847A167B9
:10D1E0009387C702631EF70A397106DE22DC26DA4E
:10D1F00080004AD84ED652D456D23285B284970097
:10D200000000E780C0C7AA89268597000000E78054
:10D2100020C92318A4FC268597000000E78040C899
:10D220002319A4FC268597000000E78060C783D7F8
:10D2300044000A8A231AA4FC858393F7F70F230E70
:10D24000F4FC8607BD0793F7073F3301F1408A8A54
:10D2500001498347C4FD6367F902CE85130584FC49
:10D26000232C54FD97000000E78080EA52811301CF
:10D2700004FCF2506254D2544259B259225A925A82
:10D2800021618280268597000000E78060C19317A6
:10D290001900D69705092390A7001379F90F55BFF8
:10D2A00082809797FF1F938727C09C43D847A16729
:10D2B0009387A702631AF70A397106DE22DC26DAA1
:10D2C00080004AD84ED652D456D23285B2849700C6
:10D2D0000000E780C0BAAA89268597000000E78091
:10D2E00020BCFD572318A4FC26852319F4FC9700C5
:10D2F0000000E780E0BA83D744000A8A231AA4FC1E
:10D30000858393F7F70F230EF4FC8607BD0793F789
:10D31000073F3301F1408A8A01498347C4FD6367AF
:10D32000F902CE85130584FC232C54FD97000000E0
:10D33000E78000DE5281130104FCF2506254D254A3
:10D340004259B259225A925A216182802685970009
:10D350000000E780E0B493171900D69705092390E1
:10D36000A7001379F90F55BF82809797FF1F938706
:10D37000A7B39C43D847A16789076310F70A39719F
:10D3800006DE22DC26DA80004AD84ED652D456D2A7
:10D390003285328997000000E78060AEAA894A850D
:10D3A00097000000E780C0AF835749000A8A23181E
:10D3B000A4FC858393F7F70F230CF4FC8607BD07C5
:10D3C00093F7073F3301F1408A8A8144834784FD04
:10D3D00063E7F402CE85130584FC232A54FD9700ED
:10D3E0000000E780E0D25281130104FCF250625445
:10D3F000D2544259B259225A925A216182804A85A6
:10D4000097000000E780C0A993971400D697850481
:10D410002390A70093F4F40F55BF82809797FF1FC6
:10D42000938787A89C43D847A1679387E704631E27
:10D43000F70A397106DE22DC26DA80004AD84ED699
:10D4400052D456D23285B28497000000E78020A3E0
:10D45000AA89268597000000E78080A42318A4FCF1
:10D46000268597000000E780A0A3231AA4FC268548
:10D4700097000000E780C0A283D744000A8A2319DE
:10D48000A4FC858393F7F70F230EF4FC8607BD07F2
:10D4900093F7073F3301F1408A8A01498347C4FD6E
:10D4A0006367F902CE85130584FC232C54FD970095
:10D4B0000000E780E0C55281130104FCF250625481
:10D4C000D2544259B259225A925A216182802685F9
:10D4D00097000000E780C09C93171900D6970509B4
:10D4E0002390A7001379F90F55BF82809797FF1FEC
:10D4F0009387879B9C43D847A1679387C704631A88
:10D50000F70A397106DE22DC26DA80004AD84ED6C8
:10D5100052D456D23285B28497000000E78020961C
:10D52000AA89268597000000E7808097FD57231879
:10D53000A4FC2685231AF4FC97000000E78040969F
:10D5400083D744000A8A2319A4FC858393F7F70F35
:10D55000230EF4FC8607BD0793F7073F3301F14024
:10D560008A8A01498347C4FD6367F902CE851305A2
:10D5700084FC232C54FD97000000E78060B95281A1
:10D58000130104FCF2506254D2544259B259225A47
:10D59000925A21618280268597000000E7804090A2
:10D5A00093171900D69705092390A7001379F90F4F
:10D5B00055BF82809797FF1F9387078F9C43D8475B
:10D5C000A167DD076317F7041753FFFFE70223B1D5
:10D5D00079713285328497000000E780408A2AC63C
:10D5E000228597000000E780A08B2311A1022285ED
:10D5F00097000000E780A088B2452300A102280818
:10D6000097000000E780C0B045611753FFFF670037
:10D6100043AF82809797FF1F938707899C43D84722
:10D62000A167938787046317F7041753FFFFE70287
:10D6300003AB79713285328497000000E780208443
:10D640002AC6228597000000E78080852311A10269
:10D65000228597000000E7808082B2452300A10266
:10D66000280897000000E780A0AA45611753FFFF34
:10D67000670023A982809797FF1F9387E7829C43C7
:10D68000D847A1679387A7046312F7021753FFFFD8
:10D69000E702E3A401112800814597000000E7801C
:10D6A00020A705611753FFFF6700A3A58280978716
:10D6B000FF1F9387677F9C43D847A16793875702D3
:10D6C0006319F7021753FFFFE70263A101113285C7
:10D6D00097F0FFFFE780A07A2308A100814528008A
:10D6E00097000000E780C0A205611753FFFF6700A5
:10D6F00043A182809787FF1F9387077B9C43D8476E
:10D70000A1679387E702631BF7041753FFFFE70244
:10D71000039D01113285328497F0FFFFE780407846
:10D72000AA84228597F0FFFFE7808077854709E983
:10D73000228597F0FFFFE78080744205B337A00091
:10D7400028008145231891003ECA97000000E78019
:10D75000209C05611753FFFF6700A39A828097877B
:10D76000FF1F938767749C43D84799476313F70853
:10D770001753FFFFE702A39679713285328497F041
:10D78000FFFFE780C06F2AC6228597F0FFFFE78082
:10D7900020712310A102228597F0FFFFE780206E01
:10D7A0002301A102228597F0FFFFE780406DA301CE
:10D7B000A102228597F0FFFFE780606C2302A1029F
:10D7C000228597F0FFFFE780806B2313A10222855B
:10D7D00097F0FFFFE780A06AB2452314A102280852
:10D7E00097000000E780C09245611753FFFF670074
:10D7F000439182809787FF1F9387076B9C43D8478D
:10D80000A1679387C7036313F7081753FFFFE70266
:10D81000038D79713285328497F0FFFFE7802066AF
:10D820002AC6228597F0FFFFE78080672310A102B8
:10D83000228597F0FFFFE780A0662311A1022285D1
:10D8400097F0FFFFE780A0632302A102228597F0F3
:10D85000FFFFE780C062A302A102228597F0FFFFCD
:10D86000E780E0612303A102228597F0FFFFE780B4
:10D870000061B245A303A102280897000000E780D9
:10D88000208945611753FFFF6700A38782801753E4
:10D89000FFFFE702C38401112A8497F0FFFFE780AE
:10D8A000005EAA84228597F0FFFFE780605F2285F3
:10D8B00097F0FFFFE780C05E035744008D4763F792
:10D8C000E700228597F0FFFFE780805D228597F0D3
:10D8D000FFFFE780E05C2800A68597000000E78056
:10D8E000208305611753FFFF6700A3819787FF1F00
:10D8F0009387875B9C43D847A167FD07631FF700A9
:10D900001743FFFFE702A37D328597000000E78001
:10D9100040F81743FFFF6700C37E82809787FF1F91
:10D92000938787589C43D847A167E5076315F70895
:10D930001743FFFFE702A37A79713285328497F0AB
:10D94000FFFFE780C0532AC6228597F0FFFFE780DC
:10D950002055228597F0FFFFE78080542310A10215
:10D96000228597F0FFFFE780A053520551812311D4
:10D97000A10222852302010297F0FFFFE7802050D9
:10D98000A302A102228597F0FFFFE780404F230307
:10D99000A102228597F0FFFFE780604EB245A30306
:10D9A000A102280897F0FFFFE780807645611743C2
:10D9B000FFFF6700037582809787FF1F9387C74E1D
:10D9C0009C43D847A1679387E703631FF70017437A
:10D9D000FFFFE702C370328597000000E78060EB2D
:10D9E0001743FFFF6700E37182809787FF1F9387CC
:10D9F000A74B9C43D847A16793874704631EF70250
:10DA00001743FFFFE702A36D79713285328497F0E7
:10DA1000FFFFE780C0462AC6228597F0FFFFE78018
:10DA20002048B245280897F0FFFFE780606E456107
:10DA30001743FFFF6700E36C82809787FF1F938780
:10DA4000A7469C43D847A167938787026310F704D2
:10DA50001743FFFFE702A36879713285328497F09C
:10DA6000FFFFE780C0412AC6228597F0FFFFE780CD
:10DA70000041B2452300A102280897F0FFFFE7808C
:10DA8000206945611743FFFF6700A3678280174342
:10DA9000FFFFE702C364011197F0FFFFE780203E1C
:10DAA000AA85280097F0FFFFE7808066056117438D
:10DAB000FFFF670003659787FF1F9387E73E9C433F
:10DAC000D847A167D107631FF7001743FFFFE7029D
:10DAD0000361328597000000E780A0FB1743FFFF3A
:10DAE0006700236282809787FF1F9387E73B9C43F1
:10DAF000D847A167C507631FF7001743FFFFE70279
:10DB0000035E328597000000E780A0F81743FFFF0F
:10DB10006700235F82809787FF1F9387E7389C43C6
:10DB2000D847A167B907631FF7001743FFFFE70254
:10DB3000035B328597000000E780A0F51743FFFFE5
:10DB40006700235C82809787FF1F9387E7359C439C
:10DB5000D847A167AD07631FF7001743FFFFE70230
:10DB60000358328597000000E780A0F21743FFFFBB
:10DB70006700235982809787FF1F9387E7329C4372
:10DB8000D84789476318F7021743FFFFE702235579
:10DB90000111328532C897F0FFFFE780402EAA8539
:10DBA000280097F0FFFFE780A05605611743FFFFAD
:10DBB0006700235582809787FF1F9387E72E9C433A
:10DBC000D847A1678D076311F7041743FFFFE702EA
:10DBD000035101113285328497F0FFFFE780202A3C
:10DBE00013066100AA844C00228597300000E7806C
:10DBF000C0232800A68597F0FFFFE78060510561EC
:10DC00001743FFFF6700E34F82809787FF1F9387CB
:10DC1000E7299C4381CFDC4391CB1743FFFFE70209
:10DC2000034C82971743FFFF6700A34D8280174381
:10DC3000FFFFE702C34A79713C08AE843ED2A1657A
:10DC4000B7070A002A843ED448103C08DD053ED6BA
:10DC500036C432C63AC297D0FFFFE780402C124745
:10DC60004810BA8597F0FFFFE780C013324648108E
:10DC7000B28597F0FFFFE780E014A2464810B68512
:10DC800097F0FFFFE7800012501001478146A685FC
:10DC9000228597D0FFFFE780E04D45611743FFFFE6
:10DCA000670023461743FFFFE702634301117C002F
:10DCB0000329C501AE843ECAA165B70707002A84BF
:10DCC0003ECC48087C00C5053ECE97D0FFFFE780DC
:10DCD00000258345D900480897F0FFFFE780800CB6
:10DCE000500801478146A685228597D0FFFFE7802F
:10DCF000604805611743FFFF6700A3401743FFFF1C
:10DD0000E702E33D83C7950093F7F707A384F50087
:10DD100097000000E78040F91743FFFF6700633E6C
:10DD20001743FFFFE702A33B79713C08AE843ED264
:10DD3000A165B70709002A843ED448103C089385A2
:10DD400045043ED632C636C497D0FFFFE780201D7B
:10DD5000A2464810B68597F0FFFFE780A004324640
:10DD60004810B28597F0FFFFE780C00550100147CB
:10DD70008146A685228597D0FFFFE780A03F4561B9
:10DD80001743FFFF6700E3371743FFFFE702233521
:10DD900083C7950041112A8493F7F707A384F50000
:10DDA00032852EC697F0FFFFE780800F85672AC473
:10DDB0006370F50297700000E78020E92246B245C3
:10DDC00009ED11478146228597000000E78060E653
:10DDD00041011743FFFF6700C33201478346F50146
:10DDE000DDB71743FFFFE702E32D01113C003ECAF8
:10DDF000B7070A003ECC3C003ECE83C79500AA89F7
:10DE0000328593F7F707A384F5002E8497F0FFFF80
:10DE1000E78000098567637DF504A165AA84938581
:10DE20008504480897D0FFFFE780600F268597702C
:10DE30000000E78080E12A8929E19145480897F0B0
:10DE4000FFFFE78020F6A685480897F0FFFFE780F0
:10DE500060F7CA85480897F0FFFFE780A0F4014704
:10DE600081465008A2854E8597D0FFFFE78080301D
:10DE700005611743FFFF670023288145480897F095
:10DE8000FFFFE78020F20349090275BF1743FFFF38
:10DE9000E702432379711C103ECAB7070F003ECC3E
:10DEA000404D1C10AA84AE894808994532C636896F
:10DEB0003ECE97D0FFFFE780800632464808B28505
:10DEC00097F0FFFFE78000EE630C0902A5454808C4
:10DED00097F0FFFFE780C0E62546CA85972001003E
:10DEE000E78020A4500801478146CE85268597D03B
:10DEF000FFFFE780202845611743FFFF6700C31F2E
:10DF00008355C402480897F0FFFFE780A0EB035554
:10DF1000E402814505C5854785456301F502C16772
:10DF2000FD179305F00F630BF5007D15977000004A
:10DF3000E780208E9305150093F5F50F480897F0BC
:10DF4000FFFFE78020E683450403480897F0FFFFC2
:10DF5000E78040E583451403480897F0FFFFE7801A
:10DF600060E483552403480897F0FFFFE78080E5CD
:10DF700083554403480897F0FFFFE780A0E49DB76E
:10DF80001743FFFFE702A31583C7950081460146AB
:10DF900093F7F707A384F50097000000E78040EFB0
:10DFA0001743FFFF6700E3151743FFFFE702231343
:10DFB00079713E841C103ECA2E89B7070F00A165F7
:10DFC0003ECCFD051C10AA84480842C03AC23ECE91
:10DFD00036C432C697D0FFFFE78060F43246480867
:10DFE000B28597F0FFFFE780E0DBA2464808B685E0
:10DFF00097F0FFFFE78000DD12474808BA8597F0E9
:10E00000FFFFE78020DC0248630C080291454808C6
:10E0100097F0FFFFE780C0D21146A285972001004C
:10E02000E7802090500801478146CA85268597D011
:10E03000FFFFE780201445611743FFFF6700630C73
:10E040008945480897F0FFFFE78080CF83470400A9
:10E050002300F50083471400A300F500E1B7174340
:10E06000FFFFE702230683C7950001112A8A93F771
:10E07000F707A384F5003285AE8432C697F0FFFF20
:10E08000E78000E232462A89328597F0FFFFE78079
:10E0900000DF85676373F902AA894A8597700000DB
:10E0A000E780A0BA2A8419ED114781464A86A685E1
:10E0B000528597000000E780C0B705611743FFFF56
:10E0C000670083039387E9FF93F7F70F0547E3663C
:10E0D000F7FE8347F50195EB8947E380F9FE834618
:10E0E000F401528501474A86A68597000000E78023
:10E0F00040B4A167D90748083ECC230A010002CEEC
:10E1000097000000E780A0B04DBF639EE7008947FD
:10E11000639EF90093071020231FF50097700000FD
:10E12000E780C0B76DBF0947E39BE7FA8D47E398E7
:10E13000F9FA228597700000E78080DF9787FF1F3C
:10E140009387C7F59C4399E79787FF1F9387C7DE9F
:10E150009C4399C703D5040097800000E780A0CEB8
:10E16000231F040022855DBF1743FFFFE70223F74B
:10E1700001113C003ECAB7070B003ECC3C003ECE2E
:10E1800083C795002A89328593F7F707A384F500A2
:10E19000AE8497F0FFFFE780A0D093170501C187F9
:10E1A000635AF006A1652A849385E502480897D052
:10E1B000FFFFE780C0D6A285480897F0FFFFE78001
:10E1C00060C09787FF1F938727D79C43A9EB014423
:10E1D0009375F40F480897F0FFFFE780A0BC9355B4
:10E1E000844093F5F50F480897F0FFFFE78080BB68
:10E1F0009355044193F5F50F480897F0FFFFE7802A
:10E2000060BA014781465008A6854A8597D0FFFF2E
:10E21000E78040F605611743FFFF670083EE416525
:10E2200085460546A2857D1597500000E78060BDB4
:10E2300059DD510597000100E780808F13044006E7
:10E240003344850271B71743FFFFE70243E9011129
:10E25000B70706003EC683C7950021642A8993F755
:10E26000F707A384F500AE8428009305A4040AC42C
:10E270000AC897D0FFFFE78080CA30000147814677
:10E28000A6854A8597D0FFFFE780C0EE97E0FFFFA5
:10E29000E780E01113049404480822CC230A01000B
:10E2A00002CE97000000E780809605611743FFFFCC
:10E2B000670023E51743FFFFE702C3E0C1642A8933
:10E2C00001449789FF1F9389E9DE130A8002FD1438
:10E2D00097E0FFFFE780E0BD6347A40001451743D7
:10E2E000FFFF670063E1B307440303A7C90ABA97B6
:10E2F00003D707006306970083D7270063842701AD
:10E300000504F9B70545E1BF1743FFFFE70283DBCB
:10E310002A8A2E8999C123A0050081498144978AC0
:10E32000FF1F938AEAB8614B97E0FFFFE780A0BE2A
:10E3300063C7A4004E851743FFFF6700E3DB338408
:10E34000640383A70A003E948357040099E763049B
:10E350000900232089008504C1BF4146D2851305E9
:10E36000440097100100E780605975F5A289E5B770
:10E370001743FFFFE70203D539717C083ED4B70786
:10E380000A003ED67C083ED883C795002A8A32858B
:10E3900093F7F707A384F5002E8932C697F0FFFFA5
:10E3A000E78000B085676373F5083246AA8432853A
:10E3B00097F0FFFFE780A0AC8547AA8963E8A7062E
:10E3C000A16593858504281097D0FFFFE78020B5CD
:10E3D000268597700000E78040872A8429ED9145C3
:10E3E000281097F0FFFFE780E09BA685281097F0A4
:10E3F000FFFFE780209DCE85281097F0FFFFE78084
:10E40000609A014781463010CA85528597D0FFFF38
:10E41000E78040D6A1679387770448183EDC230A3B
:10E42000010202DE97F0FFFFE780607E2161174363
:10E43000FFFF670063CC8145281097F0FFFFE7805E
:10E440006096A685281097F0FFFFE780A097978732
:10E45000FF1F9387E7FC9C4381CB228563890900DA
:10E4600097D00000E78040248345040271B797D01D
:10E470000000E780C022CDBF1743FFFFE70283C43F
:10E4800083C795004111AA8993F7F707A384F50084
:10E490003285AE84328A97F0FFFFE78060A08567FF
:10E4A000637FF5022A8997600000E780007A2A845A
:10E4B000914631C58347F50105476387E70291C758
:10E4C0000D476366F704AD461DA8930505030325B4
:10E4D0000A00414697100100E78040420DE94101E2
:10E4E0001743FFFF670043C19305950803250A0002
:10E4F000414697100100E7806040814669F54A86F1
:10E50000A6854E8597000000E780C081C9BF83259E
:10E510000A001305940897700000E780A02919C12C
:10E52000C146F1BF9787FF1F938747B79C4399E781
:10E530009787FF1F938747A09C4399C722859780A1
:10E540000000E780208A69FD8547A30FF40022853B
:10E5500097B00000E7806084228597600000E78024
:10E56000E0734E8581464A86A68597F0FFFFE780D7
:10E57000607BA1679387570448003EC423020100D3
:10E5800002C697F0FFFFE780806891BF1743FFFF47
:10E59000E70263B283C795004111AA8993F7F70791
:10E5A000A384F50032852E89B28A97F0FFFFE780B9
:10E5B000208F85676374F50EAA8497600000E7805A
:10E5C000C0682A840DED416B014A978BFF1F938B26
:10E5D0006BAE130C400E7D1B19A833048A0383A76E
:10E5E0000B0B3E948357C40163836705050A97E0CC
:10E5F000FFFFE780008BE342AAFE95460DA08357FC
:10E60000C501639697029305050303A50A004146D9
:10E6100097100100E780802E994611E181462686F9
:10E62000CA854E8597F0FFFFE780C06F85A883A558
:10E630000A001305040397700000E780A017C14685
:10E6400079FD2285231E940097A00000E780E074E6
:10E65000228597600000E78060649787FF1F93879B
:10E6600027DC9C43A9C323000402228597D0000025
:10E67000E78040F04E8581462686CA8597F0FFFFE9
:10E68000E780406AA1679387070448003EC42302DD
:10E69000010002C697F0FFFFE78060574101174372
:10E6A000FFFF6700C3A489472300F402E1B7397173
:10E6B00006DE22DC4AD8800052D456D25AD026DA5E
:10E6C0004ED65ECE2E8A32892A8B97D0FFFFE78006
:10E6D000407A0605710541998A8A3301A1402322B7
:10E6E00024FC231404FC97D0FFFFE7808078834745
:10E6F0009A000605350593F7F7072315A4FCA30434
:10E70000FA004A85232624FC97E0FFFFE780407942
:10E7100093170501C1876340F0025681130104FC81
:10E72000F2506254D2544259B259225A925A025B60
:10E73000F24B21618280AA844A8597E0FFFFE7803F
:10E740002076AA894A8597E0FFFFE7806075A1657A
:10E750009385C5022A89130544FC97C0FFFFE78013
:10E76000007C268597C0FFFFE7804070854511C972
:10E770004A86CE8597C0FFFFE780C069AA8B21E952
:10E780008945130544FC97E0FFFFE780A061A6855B
:10E79000130544FC97E0FFFFE780C062CE851305B8
:10E7A00044FC97E0FFFFE780E061CA85130544FC65
:10E7B00097E0FFFFE780006101478146130644FCB4
:10E7C000D2855A8597D0FFFFE780C09AB9B78145B7
:10E7D000130544FC97E0FFFFE780C05CA6851305A6
:10E7E00044FC97E0FFFFE780E05DCE85130544FC25
:10E7F00097E0FFFFE780005DCA85130544FC97E0C2
:10E80000FFFFE780205C814497D0FFFFE7806066D0
:10E81000E3D4A4FA83A70B0113971400BA9783D506
:10E82000070099C5130544FC97E0FFFFE780805976
:10E830008504D9BF797106D622D44AD000184ECEAD
:10E8400052CC56CA26D25AC8AE893289AA8A97D0E3
:10E85000FFFFE78000620605690541990A8A3301D6
:10E86000A140232A24FC231C04FC97D0FFFFE7804F
:10E87000406083C7990006052D0593F7F707231D10
:10E88000A4FCA384F9004A85232E24FC97E0FFFF13
:10E89000E780006193170501C187634FF000528143
:10E8A000130104FDB250225492540259F249624AB3
:10E8B000D24A424B45618280AA844A8597E0FFFF95
:10E8C000E780005EA1659385A5022A89130544FDB2
:10E8D00097C0FFFFE780A064268597C0FFFFE78011
:10E8E000E058854509C9CA8597C0FFFFE780805574
:10E8F0002A8B29E18945130544FD97E0FFFFE78056
:10E90000604AA685130544FD97E0FFFFE780804B32
:10E91000CA85130544FD97E0FFFFE780A04A014741
:10E920008146130644FDCE85568597D0FFFFE780CC
:10E930006084B5B78145130544FD97E0FFFFE7808C
:10E940006046A685130544FD97E0FFFFE7808047FA
:10E95000CA85130544FD97E0FFFFE780A046814488
:10E9600097D0FFFFE780E050E3DBA4FA83270B0199
:10E9700013971400BA9783D5070099C5130544FD72
:10E9800097E0FFFFE78000448504D9BF1733FFFFFE
:10E99000E702E37483474500404DD5EFFD575DC462
:10E9A0008346940009476363D70A0346B40085464B
:10E9B00063EEC6088306E40063CA06085C45F956A0
:10E9C0002390D7009777FF1F83C7C74E99E3A3040F
:10E9D000E4009777FF1F938727569C4381E7894779
:10E9E000A306F4009787FF1F938787A39C4381E7C3
:10E9F00089472306F4009705000093854506AA84FD
:10EA00001305040197F00000E7802010FD57231A3A
:10EA1000F40281471CDC01489777FF1F23A8874831
:10EA20009777FF1F9387C748232E040304C08043B2
:10EA300097D0FFFFE780204E61463306C50281452F
:10EA400022859730FFFFE780806C81473E85173332
:10EA5000FFFF6700036BFD57D5BF1733FFFFE702CA
:10EA600003682A840355450297600000E780E01D93
:10EA700019E5231E04001733FFFF670083688357DF
:10EA8000E401F5DB930504FF174501001305851C20
:10EA900097E00000E780E014F9BF1733FFFFE702BB
:10EAA00003642E89A16541119385E5032A8436C448
:10EAB00032C6BE843AC297C0FFFFE7804046124785
:10EAC0002285BA8597E0FFFFE780C02D3246228578
:10EAD000B28597E0FFFFE780E02EA2462285B6854B
:10EAE00097E0FFFFE780002E63030902914522852E
:10EAF00097E0FFFFE780C0241146A685971001002C
:10EB0000E78020E241011733FFFF6700835F8945FB
:10EB1000228597E0FFFFE780A02283C7040023003F
:10EB2000F50083C71400A300F500E9BF1733FFFF0A
:10EB3000E702E35A83C79500444D054793F7F7076B
:10EB4000A384F5001C42411183C707006367F706E1
:10EB50002E842A89B1C003C7D400630FF702177748
:10EB6000FF1F1307673D184305C3A386F40097A052
:10EB70000000E780404A83C7D40099E741657D15CE
:10EB800097400000E780403083D72403918B89C7EA
:10EB900097E00000E780C0134A85A28597F0FFFF49
:10EBA000E7808010A167C10748003EC4230201002E
:10EBB00002C697F0FFFFE780800541011733FFFF92
:10EBC000670023541733FFFFE702635103D7450063
:10EBD0008D47AA8441112E8432892E8563E3E70292
:10EBE00097E0FFFFE780C02BAA8523000900268558
:10EBF00097C0FFFFE780002541011733FFFF670043
:10EC0000435097E0FFFFE780A0292AC6228597E0BE
:10EC1000FFFFE780E028B24585472A862300F900F8
:10EC2000268597C0FFFFE780E01EF9B7397106DE41
:10EC300022DC26DA80004ED652D456D24AD85AD098
:10EC40005ECEAE89B284AA8A97D0FFFFE7806021AA
:10EC500006051305250241990A8A3301A1402322A2
:10EC600024FC231404FC97D0FFFFE780801F83C798
:10EC7000990006054D0593F7F7072315A4FCA38417
:10EC8000F9002685232624FC97E0FFFFE78040213A
:10EC900093170501C1876340F0025281130104FC00
:10ECA000F2506254D2544259B259225A925A025BDB
:10ECB000F24B21618280AA8B03AB040097C0FFFF57
:10ECC000E780C01A51E583D7440001498544F11714
:10ECD00093B71700A301F4FC834734FCA165C9C7AF
:10ECE0009385E504130544FC97C0FFFFE7802023CC
:10ECF000A685130544FC97E0FFFFE780A00ADE85A8
:10ED0000130544FC97E0FFFFE780C00B834734FC0A
:10ED1000114691E30946DA85130544FC97E0FFFFAD
:10ED2000E78060058144630A0900416B7D1B97D031
:10ED3000FFFFE780001363CCA4020147814613065E
:10ED400044FCCE85568597C0FFFFE780A042B1B74F
:10ED5000A685130634FC97000000E780E0E69334B4
:10ED600015002A8986048DBF9385C504A5BF832716
:10ED7000C90013971400BA9783D50700638865010B
:10ED8000130544FC97E0FFFFE780C003850445B707
:10ED90001733FFFFE702233279711C103EC4B70717
:10EDA0000F003EC61C103EC883C79500AA8A328554
:10EDB00093F7F707A384F500AE89328497E0FFFF4D
:10EDC000E780000E93170501C187635AF0062A8A6F
:10EDD000228597E0FFFFE780A00C2A895285032B4C
:10EDE000040097C0FFFFE780600839ED83574400B7
:10EDF00081440544F11793B71700A303F10083453D
:10EE00007100DA872287CA865286280097000000A0
:10EE1000E780E0C8014781463000CE85568597C01F
:10EE2000FFFFE7802035A1679387D70348083ECCD2
:10EE3000230A810026CE97F0FFFFE78040DD456181
:10EE40001733FFFF6700A32AA285130671009700FE
:10EE50000000E78060D7AA84094455D13544E30017
:10EE600055FB4A8597F0FFFFE78000450D4441D9E7
:10EE7000014497D0FFFFE780C0FE634DA400C16B43
:10EE80000144FD1B97D0FFFFE780A0FD634EA40067
:10EE90001544B5B7DC4413171400BA9783D707009D
:10EEA000638327030504F1B7D84493171400BA9776
:10EEB00003D70700631B770123902701268597A0BE
:10EEC0000000E78080DB01441DBF050465BF1733E8
:10EED000FFFFE702231F83C7950041112A8A93F79A
:10EEE000F707A384F50032852E89328497E0FFFF6F
:10EEF000E78000FB93170501C1876353F006AA89D9
:10EF0000228597E0FFFFE780A0F92311A1004E853D
:10EF1000832A040097C0FFFFE78040F539E5835757
:10EF2000440085440144F11793B71700A300F10092
:10EF30000348110003572100D6875285CE862686C6
:10EF4000CA8597F0FFFFE7806006A167F1074800D8
:10EF50003EC42302910022C697F0FFFFE78020CB3A
:10EF600041011733FFFF67002319A2851306110023
:10EF700097000000E78040C52A84894455D983570B
:10EF8000210011678544BA97C2071167C18313072F
:10EF9000F7EFE36FF7F89777FF1F938727109C43EE
:10EFA00081CB85451305210097500000E78020752F
:10EFB000835521002285814497C0FFFFE780A0E1AF
:10EFC00025D923100500228597A00000E78040CDB9
:10EFD00085B71733FFFFE702030E83C79500411182
:10EFE0002A8B93F7F707A384F50032852E8A3284A3
:10EFF00097E0FFFFE780C0EA93170501C1876351DF
:10F00000F006AA8A228597E0FFFFE78060E92A8957
:10F010005685832B040097C0FFFFE78020E531E58C
:10F020008357440081440544F11793B71700A301A7
:10F03000F10003483100DE875A854A87D68622864A
:10F04000D28597F0FFFFE78060F6A167ED074800E3
:10F050003EC42302810026C697F0FFFFE78020BB55
:10F0600041011733FFFF67008308A28513063100B3
:10F0700097000000E78040B5AA8409445DD99167F4
:10F08000CA97C2071167C1831307F7EF0544E3620C
:10F09000F7FACA8597C0FFFFE780E0D3014451F932
:10F0A000814997D0FFFFE780C0DC63DBA900984867
:10F0B00093971900BA9703D7070005EF239027010C
:10F0C00097D0FFFFE780E0DA1544E384A9F62685B0
:10F0D00097A00000E780C0BC9777FF1F938707FCCD
:10F0E0009C430144B9D74A8597500000E780C05837
:10F0F00089B785097DB71733FFFFE702A3FC797154
:10F100003E847C083EC82E8AB7071400A1653ECA1B
:10F11000E5057C08AA89080836C4428932C6BA8A3D
:10F12000C6843ECC97C0FFFFE78060DFCA85080831
:10F1300097E0FFFFE78000C732460808B28597E0F6
:10F14000FFFFE78020C8A246630A09049D4508081E
:10F1500097E0FFFFE780C0BE1D4681459730FFFF67
:10F16000E780E0FA63890A089145080897E0FFFF05
:10F17000E78000BD1146A68597000100E780607A10
:10F18000100801478146D2854E8597C0FFFFE78072
:10F1900060FE45611733FFFF670003F6B685080878
:10F1A00097E0FFFFE78000C21C400808D843935552
:10F1B000C701858912075183B205D98D97E0FFFFFA
:10F1C000E78040C01C40080883C5870097E0FFFF28
:10F1D000E78040BD1C40080883C5A70097E0FFFFFB
:10F1E000E78040BC1C40080883C5970097E0FFFFFC
:10F1F000E78040BB85BF8945080897E0FFFFE780AF
:10F2000020B483C704002300F50083C71400A300C3
:10F21000F500BDB71733FFFFE702C3EA83C79500C8
:10F220004111AA8993F7F707A384F5003285AE84CC
:10F23000328497E0FFFFE780A0C693170501C187DE
:10F24000635DF0042A89032A040097C0FFFFE7806A
:10F25000E0C119E9835744000548F11793B7170037
:10F26000A307F100814631A81306F100A28597009B
:10F270000000E78060951DC51C459DC783D64700EB
:10F2800001480347F10093078500D2884A86A68586
:10F290004E8597000000E78040E641011733FFFFED
:10F2A000670083E509487DBF1D486DBF1733FFFF29
:10F2B000E70243E165715C083EC4B7077B013EC6C7
:10F2C0005C083EC883C795002A8A328593F7F70702
:10F2D000A384F500AE8997E0FFFFE78040BA83572B
:10F2E000E100E1C78945280097C0FFFFE78020C300
:10F2F0008145280097E0FFFFE780C0AA97C0FFFF85
:10F30000E78000C99777FF1F938787119C43177485
:10F31000FF1F034424BAAA843334800099C31364C2
:10F3200024009777FF1F938727C19C4399C31364D9
:10F3300044009777FF1F938767D69C4399C3136454
:10F34000840083D504002800014997E0FFFFE7808F
:10F3500060A783D52400280097E0FFFFE78080A600
:10F3600083D54400280097E0FFFFE780A0A597D051
:10F37000FFFFE78000AB93150501C181280097E0EE
:10F38000FFFFE78020A4A285280097E0FFFFE78029
:10F3900060A39C446360F902014781463000CE853A
:10F3A000528597C0FFFFE780E0DC59611733FFFF0C
:10F3B000670083D4DC441314490028003E9497E08E
:10F3C000FFFFE780609683474400034754008907A6
:10F3D0000607BA978607E36AF5FC835524002800E0
:10F3E000814A97E0FFFFE780E09D834544002800C5
:10F3F00097E0FFFFE780009B83455400280097E0DB
:10F40000FFFFE780209A8347440063C9FA00814ADE
:10F410008347540063C1FA020509A5BF1C44139732
:10F420005A002800BA9783D50700850A97E0FFFFA6
:10F43000E7804099C9BF032BC40093975A00280066
:10F440003E9B83552B00850A97E0FFFFE78080975E
:10F4500083550B00280097E0FFFFE780A0964DBF83
:10F460001733FFFFE702A3C75C4993E717005CC9A6
:10F4700097A00000E78020B61733FFFF670063C83E
:10F480001733FFFFE702A3C52E84814597F0FFFFE6
:10F49000E780C0E705C583570500FD172310F50079
:10F4A00009C4835725002310F40097000000E7806B
:10F4B00060FB01451733FFFF6700A3C431457DD8CA
:10F4C00023100400C5BF1733FFFFE702A3BF83C7A4
:10F4D000950041112A8A93F7F707A384F500328536
:10F4E0002E89328497E0FFFFE780809B9317050108
:10F4F000C1876356F006AA89C145228597E0FFFFC0
:10F50000E780A0802A8B4E85832A040097C0FFFFE6
:10F51000E780C09531E98357440023110100054479
:10F52000F11793B71700A300F100814403481100BD
:10F5300003572100D6875285CE862286CA8597F04A
:10F54000FFFFE780A0A6A1679387170248003EC48B
:10F550002302810026C697E0FFFFE780406B410150
:10F560001733FFFF670043B913061100A28597F018
:10F57000FFFFE7806065AA8409E5231101000944C3
:10F5800075B7930521005A8597000000E78080EF4A
:10F59000835721002A84D9DB9777FF1F938707B011
:10F5A0009C4381CB85451305210097500000E780DF
:10F5B0000015835521002685314497C0FFFFE78061
:10F5C00080812DD523100500268597900000E780C7
:10F5D000206D0144A1BF1733FFFFE70243B0411183
:10F5E0002E896C00AA8402C697F0FFFFE78000D244
:10F5F0000DC10357050005072310E5009700000023
:10F60000E78040E681473E8541011733FFFF6700F1
:10F6100043AF3247954765DBCA85268597300000A2
:10F62000E780400DC147E34005FE3244854741462F
:10F630002310F40083570900A68513054400231105
:10F64000F40097000100E780C02D228545BF1733E5
:10F65000FFFFE70223A783C795004111AA8A93F70A
:10F66000F707A384F5003285AE89328497E0FFFF67
:10F67000E780008393170501C1876356F0062A8A45
:10F68000C145228597D0FFFFE7802068AA84528574
:10F69000032B040097B0FFFFE780407D31E98357DB
:10F6A0004400231101008544F11793B71700A3000C
:10F6B000F10001440348110003572100DA87568501
:10F6C000D2862686CE8597F0FFFFE780208EA16741
:10F6D0009387070248003EC42302910022C697E0A8
:10F6E000FFFFE780C05241011733FFFF6700C3A04F
:10F6F000A2851306110097F0FFFFE780E04C2A84F3
:10F7000009E523110100894475B726859305210079
:10F7100097000000E78060ECAA8449FD8355210032
:10F72000228597B0FFFFE780006B49F5014997C03C
:10F73000FFFFE7800074635DA90018489317190064
:10F74000BA9703D707000DEF035721002390E70076
:10F7500097C0FFFFE780E071630625039777FF1FDF
:10F760009387C7939C4399C7035521009750000086
:10F77000E78080F0228597900000E78060521DBFEF
:10F78000050975B795443DB705C19307F00F630FA1
:10F79000F500C547630CF5009307F5FF05453315E4
:10F7A000F5004205418182800145828041657D15D9
:10F7B0008280B9E91733FFFFE7026392034506032E
:10F7C000328497000000E78060FC9305803EB3051B
:10F7D000B502C205C18181CD0357E402854763F8B4
:10F7E000E7001305040197E00000E78020428357FB
:10F7F000E40241677D176385E700FD172317F402D4
:10F800001733FFFF6700E38F82801733FFFFE702A4
:10F81000838A004283C79500444D0349140093F73F
:10F82000F707A384F50083470400220911673369B1
:10F83000F900A167B347F90041112A8BAE8A63EC46
:10F84000E70E834724001307C00EB91793F7F70F8D
:10F850006373F71003473400C14763EEE70E834735
:10F8600044001307E00793C707086371F70C834947
:10F87000840083477400A209B3E9F900856763F740
:10F88000F90A034A6400834754004E85220A336A0A
:10F89000FA0097500000E780403B61C123962403A3
:10F8A000834B3400137AFA00239A340323887403B9
:10F8B0002399440393890401631C090023A60402CD
:10F8C000239804024E8597E00000E78060363DA053
:10F8D000034924004A8597000000E78020EB239726
:10F8E000A402834744004E85A388F402E38D0BFCF9
:10F8F000E30B09FC97E00000E780202F97900000C1
:10F90000E780007381460146D6855A8597E0FFFF60
:10F91000E7800058A167938797033EC42302010044
:10F92000480002C697E0FFFFE780602E41011723E1
:10F93000FFFF6700C37B8544A2862686D6855A854D
:10F9400097E0FFFFE780C054A167938797033EC409
:10F9500023029100F1B7BD44C5B79144F1BF17230D
:10F96000FFFFE702237601111C08404D3EC2B70796
:10F970000F003EC41C083EC62A89AE8997C0FFFF0F
:10F98000E78000D7585C1C5C6346B70E6394E500C3
:10F9900063E2A70E3385A740B3B7A700B305B7400E
:10F9A0001306803E81469D8D97000100E78080B759
:10F9B00093140501C180A1659385C503480097B0E4
:10F9C000FFFFE780C0558145480097D0FFFFE780E3
:10F9D000603D83550404480097D0FFFFE780803ED8
:10F9E00083552404480097D0FFFFE780A03D814560
:10F9F00089CCC167FD179305F00F6388F400268555
:10FA000097500000E780E0E0AA85480097D0FFFF0C
:10FA1000E780403903554404814501CDC167FD1796
:10FA20009305F00F6307F50097500000E78060DE54
:10FA3000AA85480097D0FFFFE780C036834564045D
:10FA4000480097D0FFFFE780E03583457404480005
:10FA500097D0FFFFE7800035500001478146CE85F3
:10FA60004A8597B0FFFFE780E07005611723FFFF2D
:10FA700067008368814481B71723FFFFE70223668D
:10FA800083C7950093F7F707A384F500970000005C
:10FA9000E78020ED1723FFFF6700A3661723FFFF12
:10FAA000E702436283C795004111404D93F7F70782
:10FAB000A384F5002A8A3285B284AE8997D0FFFFED
:10FAC000E780003E2A8B268597D0FFFFE780403DE8
:10FAD0002A89268597D0FFFFE780603A93170B01AC
:10FAE00063CA0702E177CA97C207C183116763E35C
:10FAF000E70293070910C207C1831307B00F637BA6
:10FB0000F70093170901C187AA8A634AF000C54725
:10FB100063FE570141011723FFFF6700E35D97B0C4
:10FB2000FFFFE7802025E31725FFD5B763080B0209
:10FB300063060902814463890A02B7077F00231024
:10FB40006405231124057CC0568597000000E780DA
:10FB5000E0C39304803EB304950239A0B7077F0049
:10FB6000232004047CC081440355240497E0000052
:10FB7000E780A0A3A1C497C0FFFFE78060B72695E8
:10FB800093D7F44133379500AE97BA9708DC5CDC25
:10FB9000CE85528597000000E780A0DC99E0232203
:10FBA0000404A1679387B70348003EC42302010001
:10FBB00002C697E0FFFFE7808005A9BF81470148A3
:10FBC0001CDC232E0403E9B71723FFFFE7022351B0
:10FBD00097C0FFFFE7802034E1473305F5029145E8
:10FBE00097500000E78000C5E55711C59767FF1FD4
:10FBF00023A0A72C81473E851723FFFF6700635092
:10FC000085471767FF1F2307F72A82801723FFFF07
:10FC1000E702E34C9767FF1F9387472980433DC066
:10FC2000835704046390A70683572404639CB70496
:10FC30003689B28497C0FFFFE78080AB5C5C63C30A
:10FC4000B7046395B7001C5C63EEA70283476404A6
:10FC500063F3F400A6872303F4048347740463F377
:10FC60009700A687A303F4048357440441677D17D4
:10FC70006385E70085072312F4043C4481C7CA85E5
:10FC8000268582971723FFFF6700A3479767FF1F0B
:10FC90009387C7219C43014599C303C58700828090
:10FCA0001723FFFFE702A3430111B70707003EC672
:10FCB00083C79500584D0AC493F7F7070AC8A38471
:10FCC000F5002A89AE8411CB1C4283C707002304A8
:10FCD000F70097900000E7800034216493055402F8
:10FCE000280097B0FFFFE780802397000000E7809F
:10FCF00020FAAA85280097D0FFFFE780A00A3000ED
:10FD000001478146A6854A8597B0FFFFE780804678
:10FD100013044402480822CC230A010002CE97E0D3
:10FD2000FFFFE780C0EE05611723FFFF6700633D1B
:10FD30001723FFFFE702A33A01117C003ECAB70771
:10FD400007003ECC7C003ECE83C795002E84AA845B
:10FD500093F7F707A384F500A1659385550248083A
:10FD600097B0FFFFE780A01B97000000E78040F2FC
:10FD7000AA85480897D0FFFFE780C00250080147D6
:10FD80008146A285268597B0FFFFE780A03E0561EA
:10FD90001723FFFF6700E3369767FF1F938707115D
:10FDA0009C43094599C303C5970082809767FF1F4D
:10FDB0009387C70F9C43094599C303C5D700828029
:10FDC0009767FF1F9387870E9C43014599C303C51F
:10FDD000A70082801723FFFFE702C32E0111B70798
:10FDE00008003EC683C79500404D0AC493F7F70745
:10FDF0000AC8A384F5002A89AE8429C41442854721
:10FE000003C7060063E0E70A834794000946814977
:10FE10006380C702B307F740A304E400B339F000DE
:10FE200083C716002305F40097900000E780A01E0A
:10FE300003572403058B19C76386090097D0000078
:10FE4000E78000E9216493058402280097B0FFFF52
:10FE5000E780E00C97000000E78040F4AA852800C6
:10FE600097D0FFFFE78000F497000000E78080F55F
:10FE7000AA85280097D0FFFFE780C0F2014781469E
:10FE80003000A6854A8597B0FFFFE780A02E1304B7
:10FE90007402480822CC230A010002CE97E0FFFF3B
:10FEA000E780E0D605611723FFFF6700E3241723EF
:10FEB000FFFFE702C32201117C003ECAB70708001A
:10FEC0003ECC7C003ECE83C795002E84AA8493F757
:10FED000F707A384F500A16593858502480897B0CC
:10FEE000FFFFE780C00397000000E78020EBAA85B2
:10FEF000480897D0FFFFE780E0EA97000000E7801E
:10FF000060ECAA85480897D0FFFFE780A0E9500879
:10FF100001478146A285268597B0FFFFE7808025AF
:10FF200005611723FFFF6700C31D9767FF1F9387B6
:10FF3000E7F79C43014599C303C5B70082801723A7
:10FF4000FFFFE702C3190111B70707003EC683C7C9
:10FF50009500404D0AC493F7F7070AC8A384F5003B
:10FF60002A89AE8405C81C42054783C70700636819
:10FF7000F7060347B400630FF700A305F40097905A
:10FF80000000E78040098347B400B9CF97D0FFFF56
:10FF9000E78040BE21649305B400280097B0FFFFBE
:10FFA000E780E0F797000000E78060F8AA85280066
:10FFB00097D0FFFFE78000DF014781463000A6852C
:10FFC0004A8597B0FFFFE780E01A2904480822CC51
:10FFD000230A010002CE97E0FFFFE78040C30561DE
:10FFE0001723FFFF6700E31197D0FFFFE78020BFD3
:10FFF00055B71723FFFFE702830E01117C003ECAAD
:020000040001F9
:10000000B70707003ECC7C003ECE83C795002E8408
:10001000AA8493F7F707A384F500A165AD05480806
:1000200097B0FFFFE780A0EF97000000E78020F087
:10003000AA85480897D0FFFFE780C0D6500801473F
:100040008146A285268597B0FFFFE780A012056153
:100050001723FFFF6700E30A9767FF1F938707E5F2
:100060009C43094599C303C5C70082801723FFFF3E
:10007000E702E30601117C00AE843ECAA165B70722
:1000800007002A843ECCD1057C0048083ECE97B0BC
:10009000FFFFE780C0E897000000E78020FCAA850A
:1000A000480897D0FFFFE780E0CF5008014781461E
:1000B000A685228597B0FFFFE780C00B0561172357
:1000C000FFFF670003041723FFFFE702430183C715
:1000D000950093F7F707A384F50097000000E780E9
:1000E00020F91723FFFF6700C3011723FFFFE70273
:1000F00063FD83C795000329C501411193F7F707F5
:10010000A384F5001C4283C90700854763E63707CF
:100110009767FF1F9387C7309C432E84AA8485CF9F
:1001200097000000E78080F389476306F5026304C7
:1001300009028347C900638037032306390197907A
:100140000000E78040ED83572903898B89C797D04A
:100150000000E780E0B72685A28597000000E780D1
:1001600020F1A167CD0748003EC42302010002C66A
:1001700097E0FFFFE780A0A941011723FFFF670079
:10018000A3F79767FF1F938767D29C431D4599C3C9
:1001900003C5E70082801723FFFFE70243F4011144
:1001A000B70707003EC683C79500584D0AC493F7AA
:1001B000F7070AC8A384F5002A89AE8415C71C4234
:1001C00083C7070093968701E18663C406068546C8
:1001D0006381D7068346E7006388F6002307F700AC
:1001E00097900000E78020E321649305E400280055
:1001F00097B0FFFFE780A0D297000000E780A0F84B
:10020000AA85280097D0FFFFE780C0B90147814643
:100210003000A6854A8597B0FFFFE780A0F535043A
:10022000480822CC230A010002CE97E0FFFFE780B6
:10023000009E05611723FFFF6700A3EC1723FFFF54
:10024000E702E3E901117C003ECAB70707003ECC94
:100250007C003ECE83C795002E84AA8493F7F707CF
:10026000A384F500A165B905480897B0FFFFE780B2
:1002700000CB97000000E78000F1AA85480897D0DE
:10028000FFFFE78020B2500801478146A2852685FE
:1002900097B0FFFFE78000EE05611723FFFF6700BF
:1002A00043E61723FFFFE702E3E1AA84014417694D
:1002B000FF1F1309E9BFE14997C0FFFFE780A0C511
:1002C0006344A400014519A83305340383270900BA
:1002D0003E95835725006397970011051723FFFF6D
:1002E000670083E10504C9BF032E8500630A0E126F
:1002F0001763FF1F130383DA03230300631503004F
:1003000029436390061203234E01631503001D4326
:10031000639907101723FFFFE702E3D9C689428AD2
:100320003E89BA8AB684328BAE8B2A84B5E10355F6
:100330004E0019E501431A851723FFFF670023DBF1
:10034000A167A98F116763FBE70097000000E780B2
:1003500080F5814597F0FFFFE780C0120844B7079A
:1003600000E05841F98F18455CC1B707001FF98FAD
:100370001CC55C4991C7610597E00000E780408B90
:10038000E38A09FA228597900000E78060C65DB78E
:10039000328597C00000E78040430D4349DD1C448F
:1003A000116703D54700A167A98F63FBE70097009A
:1003B0000000E78040EF814597F0FFFFE780800C69
:1003C0000323840093164B01D1828347B300035665
:1003D00063008588FD8BA305F300FD777D8E558E28
:1003E000FD76FD16B204F18E83274301C58E2312DC
:1003F00073012313D3002304530123052301A30412
:100400004301BDDF228597B0FFFFE78080C9AA8541
:100410000844B5D1610597D00000E780207F8DB7F3
:100420001D431A8582801723FFFFE702A3C90569D0
:10043000AA84AE89328A0144FD5A7D1997C0FFFF14
:10044000E78020A26347A40001451723FFFF670050
:10045000A3CAD84493171400BA9703D70700631FA1
:1004600037032390570163070A0026859790000001
:10047000E780A0809C449DC383D76700B3F7270122
:10048000639E3701D2880148814701478146014672
:100490008145268597000000E78040E5050479BF87
:1004A0001723FFFFE70203C279711C103EC4B70790
:1004B0000F003EC61C103EC883C79500AA8A32852D
:1004C00093F7F707A384F5002E89328497D0FFFFB6
:1004D000E780009D93170501C187635AF006AA893A
:1004E000228597D0FFFFE780A09B2A8A4E85032BA9
:1004F000040097B0FFFFE780609739ED8357440011
:1005000081440544F11793B71700A303F100834515
:100510007100DA872287D2864E86280097E0FFFF97
:10052000E780E057014781463000CA85568597B07D
:10053000FFFFE78020C4A1679387F70348083ECCFC
:10054000230A810026CE97D0FFFFE780406C4561EB
:100550001723FFFF670043BAA2851306710097E0D7
:10056000FFFFE7806066AA84094455D1528597E071
:10057000FFFFE78060D40D4459D90546D285268512
:1005800097000000E78060EA2A8451B71723FFFF35
:10059000E702E3B4835507000346270041112A848C
:1005A0002E8532C62EC497E0FFFFE780E0D001C958
:1005B0003246A245228597000000E78000E741010E
:1005C0001723FFFF6700E3B31723FFFFE702A3AE84
:1005D00083C795004111AA8A93F7F707A384F50012
:1005E0003285AE89328497D0FFFFE780608B931706
:1005F0000501C1876357F00AC1452A8A228597C041
:10060000FFFFE78080702A8D228597D0FFFFE7806B
:1006100020892A89228597D0FFFFE78040869307AB
:1006200005F893F7F70F1307E007AA8B637BF7062C
:10063000228597D0FFFFE78080842A8C228597D07F
:10064000FFFFE780C083AA8C5285032B040097B07C
:10065000FFFFE780A08139E983574400231101009F
:100660008144F11793B71700A300F1000544034735
:10067000110083562100938784005685DA882288EA
:100680005286CE8597F0FFFFE78020A7A167E90794
:1006900048003EC42302810026C697D0FFFFE780B2
:1006A000005741011723FFFF670063A413061100E1
:1006B000A28597E0FFFFE7802051AA8409E5231176
:1006C000010009446DB7930521006A8597F0FFFF8B
:1006D000E780A0F02A8441FD835521009356C9008C
:1006E0001316490185486688E2875E87858A5182AC
:1006F000268597000000E78060BF2A848DBF1723FE
:10070000FFFFE702439B83C7950041112A8B93F7B4
:10071000F707A384F5003285AE89328497C0FFFFC6
:10072000E780007893170501C1876352F00A2A8A8F
:10073000228597C0FFFFE780A076AA8A228597C00E
:10074000FFFFE780E0752A89228597C0FFFFE780D9
:100750000073930705F893F7F70F1307E0072A8C48
:100760006377F706228597C0FFFFE7804071AA8C68
:10077000228597C0FFFFE78080702A8D5285832BEA
:10078000040097A0FFFFE780606E39E583574400BF
:1007900085440144F11793B71700A301F100034703
:1007A0003100930784005A85DE882688D6865286D3
:1007B000CE8597F0FFFFE78040948D4748003EC408
:1007C0002302910022C697D0FFFFE78040444101F9
:1007D0001723FFFF6700A391A2851306310097E05E
:1007E000FFFFE780603E2A84894455D99356C900AB
:1007F0001316490185486A88E6876287858A51828F
:10080000D68597000000E78060AEAA8449BF172311
:10081000FFFFE702238B2A8981440144617A916AB0
:10082000176BFF1F130B8B8797B0FFFFE780606488
:1008300063C7A40022851723FFFF6700E38B83278C
:10084000090093991400CE9703D50700330745019B
:10085000420741836364570305C103270B0019C78F
:1008600085453E8597400000E78060E983270900C1
:100870000504CE972390070085047DB797000000FC
:10088000E78060A2832709000504CE972390070024
:1008900065D5814597F0FFFFE780C0BEF1BF172304
:1008A000FFFFE702238283C7950041112A8A93F74D
:1008B000F707A384F50032852E89328497C0FFFFA5
:1008C000E780005E93170501C187635AF004AA8987
:1008D000832A040097A0FFFFE780405931E5835742
:1008E000440085440144F11793B71700A301F100B8
:1008F00003483100D68752850147CE862686CA85B1
:1009000097D0FFFFE780806AA167F50748003EC4E3
:100910002302910022C697D0FFFFE780402F4101BC
:100920001713FFFF6700437DA2851306310097E090
:10093000FFFFE78060292A8489445DD99757FF1F0C
:100940009387C7759C4381CF044997B0FFFFE78029
:100950004052AA85268597400000E78040DA1305BB
:10096000040197000000E780C0EA2285978000001C
:10097000E78000338144ADBF1713FFFFE702A37385
:1009800083C795004111AA8A93F7F707A384F5005E
:100990003285AE8932842311010097C0FFFFE780C2
:1009A000205093170501C1876354F0062A8AC14578
:1009B000228597C0FFFFE7804035AA8B5285032B25
:1009C000040097A0FFFFE780604A21E983574400B5
:1009D00085440144F11793B71700A300F1000348C1
:1009E000110003572100DA875685D2862686CE85E8
:1009F00097D0FFFFE780805BA167938727024800BD
:100A00003EC42302910022C697D0FFFFE78020203A
:100A100041011713FFFF6700836DA28513061100C4
:100A200097E0FFFFE780401A2A8489444DD9975701
:100A3000FF1F9387A76698433E8901CF044997B06B
:100A4000FFFFE7800043AA85268597400000E780E6
:100A500000CB1305040197000000E78080DB97B00E
:100A6000FFFFE780004195443DD9930521005E8555
:100A700097F0FFFFE78060B6AA8435F11C48035762
:100A8000210022852390E70097800000E780402125
:100A900083270900A9D70355210097400000E7806C
:100AA000A0BD35BF1713FFFFE702E36083C79500C2
:100AB0004111AA8A93F7F707A384F5003285AE891E
:100AC000328497C0FFFFE780A03D93170501C187DF
:100AD0006351F0062A8A228597C0FFFFE780403CD9
:100AE0002A895285032B040097A0FFFFE780003876
:100AF00031E58357440085440144F11793B717004B
:100B0000A301F10003483100DA8756854A87D2866F
:100B10002686CE8597D0FFFFE7804049A167F90779
:100B200048003EC42302910022C697D0FFFFE78011
:100B3000000E41011713FFFF6700635BA2851306D8
:100B4000310097E0FFFFE78020082A8489445DD9BF
:100B50009167CA97C2071167C1831307F7EF8544EE
:100B6000E362F7FA9757FF1F938747539843BE8B6B
:100B700001CF044997B0FFFFE780A02FAA85268503
:100B800097400000E780A0B713050401970000001C
:100B9000E78020C897B0FFFFE780A02D95443DD1A6
:100BA0001C48228581442390270197800000E7801C
:100BB000200F83A70B00B9D74A8597400000E78034
:100BC000A0AB89B71713FFFFE70263512A844105E1
:100BD000B28497000000E780C0C311C522859780CA
:100BE0000000E780E00B81460146A68522859780BC
:100BF0000000E780C04E1C4C89C7DC4799C32285A2
:100C000082971713FFFF6700C34F9757FF1F938704
:100C1000E7299C43014599C31385070182809757B3
:100C2000FF1F9387A728884382801713FFFFE702DF
:100C3000034B9317C600DD8DC2054111C1812A8483
:100C400032C697C0FFFFE780E01732462285118247
:100C50009375F60F97C0FFFFE780C014410117138B
:100C6000FFFF6700034A1713FFFFE702A3457971EF
:100C70003C083ED2B7070C003ED43C083ED683C7A2
:100C80009500AE842A8993F7F707A384F500A16540
:100C900093853504481097A0FFFFE7804028C16581
:100CA000FD150144175AFF1F130ACA40930A400E4C
:100CB000AE892E8B2EC697B0FFFFE780801E4205BF
:100CC000931704014181C183B24563E9A702C1675B
:100CD000FD176387F500481097C0FFFFE780800E7F
:100CE000501001478146A6854A8597A0FFFFE780FF
:100CF000604845611713FFFF670003403307540343
:100D000083270A0BBA9703D6C701630A3601638AA1
:100D10003501481097000000E78060F1DA8505048E
:100D200051BFB285EDBF1713FFFFE702C3387971DA
:100D30007C083EC8B70711003ECA7C083ECC83C77A
:100D40009500AA89328593F7F707A384F5002E89C9
:100D500097C0FFFFE780C01485676378F504A1653D
:100D6000AA848905080897A0FFFFE780401B268515
:100D700097400000E78060ED133415000A04A28557
:100D8000080897C0FFFFE780E001A685080897C024
:100D9000FFFFE780200325CC014781461008CA8564
:100DA0004E8597A0FFFFE780E03C45611713FFFFEA
:100DB0006700E333B30754030327CA0ABA9703D77C
:100DC0000700631C970003D62700638065050808A9
:100DD00097000000E780A0E5DE8505042EC697B0E9
:100DE000FFFFE780000D4205931704014181C18395
:100DF000B245E3E1A7FCC167FD17E38FF5F80808EA
:100E000097C0FFFFE78000FC41BFB285F9B7C1651D
:100E1000FD150144175AFF1F130ACA29930A8002BD
:100E20002E8BAE8B65BF1713FFFFE702432B1841D4
:100E30008347170083460700A207D58FD207D183C7
:100E40002390F50083472700034717008D45A2072D
:100E5000D98F91832310F60097C0FFFFE780A0E9A8
:100E60001713FFFF6700E3291713FFFFE70283252E
:100E7000C16401441759FF1F1309C9239309800254
:100E8000FD1497B0FFFFE780C0026347A40001454F
:100E90001713FFFF67004326330534038327C90A6E
:100EA0003E9583570500E38597FE0504D9BF1713C8
:100EB000FFFFE70223212A8AAE89B284B68A9740CF
:100EC0000000E78080D819E591473E851713FFFFA2
:100ED000670083222A894E8597C00000E780E08E54
:100EE0002A84638E0A048D476DD103570500C547D8
:100EF000E31D47FD0347F9018546AD47E317D7FCDE
:100F00008347450081CF4146A6855D0597F00000E7
:100F1000E780C09E814755D9AD4745BF130965019C
:100F20002302E500CA85268597100000E7806062ED
:100F300031C1A547E38B0AF82302040079B705C144
:100F400083570500E39247F94146A685190597F0B6
:100F50000000E780A09A81472DD99947BDB74E85FB
:100F600097000000E78080F02A84954739DD130957
:100F700055004DBF4146A68523104401231134017D
:100F80001305190097F00000E780A099228597804B
:100F90000000E780A0EA81470DBF1713FFFFE702BB
:100FA000031479717C003ECCB7070A003ECE7C006A
:100FB0003ED083C79500B2842E8493F7F707A384AD
:100FC000F5001306A1002A892C0026859700000051
:100FD000E780A0E5A16528088D0597A0FFFFE780C1
:100FE00000F490408355A100035581008546970089
:100FF0000000E78000ECAA84AA85280897C0FFFFBC
:10100000E78040DA0356A100835581002808970045
:101010000000E780C0C1300801478146A2854A85AB
:1010200097A0FFFFE7800015854748103ED42302B4
:10103000910202D697D0FFFFE78060BD456117138C
:10104000FFFF6700030C1713FFFFE70243097971E5
:101050007C003ECCB7070A003ECE7C003ED083C762
:101060009500B2842E8493F7F707A384F500130646
:10107000A1002A892C00268597000000E780E0DA8D
:10108000A16528088D0597A0FFFFE78040E9904003
:101090008355A10003558100814697000000E78039
:1010A00040E1AA84AA85280897C0FFFFE78080CF87
:1010B0000356A10083558100280897000000E780AF
:1010C00000B7300801478146A2854A8597A0FFFFF7
:1010D000E780400A48102302910202D402D697D03A
:1010E000FFFFE780C0B245611713FFFF6700630190
:1010F0001713FFFFE702A3FE97000000E78060DB05
:101100001713FFFF6700E3FF9757FF1F938747DA27
:10111000884382801713FFFFE70263FC8357250093
:101120004111AE842A842307B10017F5FFFF130590
:1011300025466C002316F10097A0FFFFE78080454D
:1011400091C4228597800000E780E0D6FD572310E8
:10115000F400130620028145130554009710FFFF89
:10116000E780E0FA41011713FFFF670083F91713C7
:10117000FFFFE70223F579717C003ECCB7070A0038
:101180003ECE7C003ED083C79500AA89AE8493F7FB
:10119000F7073285A384F5001306A1002C00970001
:1011A0000000E78080C8035581001144974000008B
:1011B000E780A0A915C50355A100014497B0000020
:1011C000E780A06011CD0357050083578100454497
:1011D0006318F700854597000000E780E0F30144BD
:1011E000216993053900280897A0FFFFE78020D3E5
:1011F000A285280897C0FFFFE780C0BA0356A10068
:1012000083558100280897000000E78040A230083D
:1012100001478146A6854E8597A0FFFFE78080F5B0
:1012200048104AD42302810202D697D0FFFFE780FC
:10123000009E45611713FFFF670003EC1713FFFFC4
:10124000E70243E89757FF1F938747C62A848843DE
:101250002E8915C5035745038357C4016311F7024F
:101260002326050223180502410597D00000E780D8
:10127000209C6306090097800000E78060DB8144C2
:101280009759FF1F938909E3130A800297B0FFFF64
:10129000E78020C263C4A4049757FF1F9387C7C980
:1012A0009C4399C70355C40197200000E780C0BD47
:1012B00063070900228597800000E780C0A013061D
:1012C000400E814522859710FFFFE78040E4FD57DF
:1012D000231EF4001713FFFF670003E23385440366
:1012E00083A7C90A3E95035705008357C4016317B6
:1012F000F700CA8597000000E78000E2850479B70F
:101300001713FFFFE70203DC83C795004111AA8989
:1013100093F7F707A384F5003285AE8497C0FFFFEB
:10132000E78000B885676378F5042A899740000054
:10133000E780A091014401CD83D704003144638844
:101340002701854597000000E78080EF01444E8526
:10135000A2864A86A68597D0FFFFE780A09CA1675A
:101360009387170448003EC42302810002C697D029
:10137000FFFFE780C08941011713FFFF6700C3D754
:101380001713FFFFE70203D49757FF1F938707B296
:10139000804329C4014597C00000E78000218147B0
:1013A0000148C1641CDC232E0403232004041759C4
:1013B000FF1F130929D001449309400EFD1497B073
:1013C000FFFFE78000AE634FA400814517F5FFFFE4
:1013D0001305857F97A0FFFFE780C01B1713FFFF52
:1013E000670083D1330534038327090B3E95835768
:1013F000C50163879700854597000000E78040E4BA
:10140000050475BF9357050113D78700A380F50026
:1014100093170501C183A1832380E5002381F50093
:10142000A381A50082801713FFFFE70243CB2300AF
:10143000050083C71500A300F50083C7250023011D
:10144000F50083C73500A301F50083C745002302DB
:10145000F50083C75500A302F50083C76500930517
:101460009500A30305002303F5002304050032853E
:1014700097000000E78040F91713FFFF670063C87B
:101480001713FFFFE70203C44111E9540DCD85CDC9
:1014900093F9C5FF2E842A89AA84338AA900B7EA62
:1014A000040063189A020D88854411CCB7E7040044
:1014B0009C5F82972AC622866C003305390197E02B
:1014C0000000E7800046268541011713FFFF6700F3
:1014D000A3C283A78A039104829793170501C1834E
:1014E000A183A38EF4FE93570501238FF4FEA183FD
:1014F000238EA4FEA38FF4FE6DB763E6D502171307
:10150000FFFFE702C3BDB28741113686BE8536C6EE
:1015100097E00000E780E040B246410136851713AE
:10152000FFFF670003BE8146368582808387050002
:101530001387F5003D05FD8793F77708834607007D
:101540007D158606B58FA300F5006307B7007D17EC
:10155000834717009D83DDB782801713FFFFE702E3
:1015600003B8B7E7040083A7070932872A863A85BC
:101570008297133515001713FFFF670083B815C155
:1015800081478DC11713FFFFE70263B5414697E01E
:101590000000E780003985473E851713FFFF67008D
:1015A00043B681473E8582801DCD1713FFFFE702BA
:1015B00003B3414681452A849710FFFFE78020B599
:1015C00041468145130504039710FFFFE78020B4CF
:1015D0000147C1672322040438C87CC80545171396
:1015E000FFFF670003B20145828081473DCDB5CD45
:1015F0001713FFFFE702A3AEB2842E8913068005FE
:1016000081452A849710FFFFE78060B0CA8524C413
:10161000268597000000E780C0F641468145228577
:101620009710FFFFE780A0AE3044A2852285970087
:101630000000E780C0F293040401A285268597008C
:101640000000E780E0EEA685130504029700000085
:10165000E78000EE228597000000E78020F58547AF
:101660003E851713FFFF6700C3A93E8582801713CD
:10167000FFFFE70223A54111E9540DCD85CD93F974
:10168000C5FF2E842A89AA84338AA900B7EA0400F8
:10169000639844030D88814411CCB7E704009C5F34
:1016A00082972AC622866C003305390197E0000034
:1016B000E7802027268541011713FFFF6700C3A39A
:1016C00083A78A039104829793170501C183A1839D
:1016D000A38EF4FE93570501238FF4FEA183238E7E
:1016E000A4FEA38FF4FE6DB765CD1713FFFFE702CD
:1016F000639DB28411E605451713FFFF6700C39F82
:101700002A842E890145EDD93C487848B3E6E700A4
:10171000E5D69386F7FFB3B7F6007D17032A440496
:10172000BA9734C87CC863050A06C14913050A0381
:10173000B38949412295637D3601B2862E86A685FE
:1017400097000000E780A0DB7C40BE9464C065B7D2
:10175000CE862E86CE8597000000E78040DAC11441
:10176000D2944E9923220404A2879306040103C74E
:10177000070003C607038507318FA38FE7FEE398B1
:10178000F6FE3044A285228597000000E78020DD28
:101790002699C1493306994063EC9900A9DCA686D5
:1017A000A6851305040397000000E78040D579BFA4
:1017B0008147B306F4003307F6000347070083C5EB
:1017C000060085072D8F2380E600E39437FF304421
:1017D000A285228597000000E78060D8C1145DBF14
:1017E000014582800DC11713FFFFE702438F1306E7
:1017F000800581459710FFFFE7806091054517132D
:10180000FFFF6700039001458280814749C5C1C53C
:101810001713FFFFE702A38CFC4141462E84AA84E4
:101820006399C70413860501A2878146C14503C792
:10183000070003C507038507298F3305D600034535
:1018400005008506298FA38FE7FEE392B6FE30449C
:10185000A285268597000000E78060D0228597004A
:101860000000E78060F885473E851713FFFF67009B
:101870004389138507031D8E814522959710FFFF2D
:10188000E780E0887C40130700F813060402A29763
:101890002388E70251BF3E8582801713FFFFE702CE
:1018A00003846D712E84B284AA8590102800368935
:1018B00097000000E780A0D309EDD55725A0504040
:1018C0000C40280097000000E78040E27DD5FD1421
:1018D0002104F5F42C004A8597000000E78020F3EE
:1018E000814761DD3E8551611713FFFF670063810A
:1018F0001703FFFFE702A37E41112EC432C62C005E
:10190000054697000000E78080F941011703FFFFBB
:101910006700237F1703FFFFE702637C01112A841E
:101920002EC602C802CA02CC02CE97E00000E780B1
:10193000C023B2462A86A285080897000000E780E7
:1019400060FB1375F50F05611703FFFF6700637BED
:101950001703FFFFE702A3787971B2872A84214633
:101960002308B10013051101BE853AC436C697E0BD
:101970000000E78000FBB246930591013685970091
:101980000000E78060A82285141035460C089700F7
:101990000000E78020F62A84224701E921460C1046
:1019A0003A8597E00000E780C0F72285456117037C
:1019B000FFFF670003751703FFFFE70243727171B2
:1019C000AE84AA850A85328497000000E78060BB58
:1019D00011C90A86A685228597000000E78020B8F5
:1019E000814711E1C5473E854D611703FFFF670041
:1019F00043711703FFFFE702836B1D712A8AB289C7
:101A0000BE8435468547130511012E8CB68A3A8B64
:101A1000C28C468D2308F10097E00000E78060F05B
:101A200010100C085285231F010097000000E7806A
:101A3000C0F82A843DEDA1476313FD089307900584
:101A400091E0E5473546E2851305110113990A0136
:101A50002308F1001359090197E00000E78060ECCA
:101A60001357890093978A00D98F90080C085285E4
:101A7000231FF10097000000E78020F42A8415E975
:101A8000A1E49387FA0091831379F9003EC66313AA
:101A900009004149668B8144C14B854DB247639F24
:101AA000970C6A868C0033855C0197E00000E78024
:101AB00040E7228525611703FFFF67000363930753
:101AC0009004C9F0A547BDBF834701050947C14B35
:101AD0002308F10083471105A58FA308F100938720
:101AE0002400814463E1FB04014714083386E600C7
:101AF0008C08B386E400BA95DA9683C6060083C5DF
:101B000005000507AD8E2300D600E390E7FE4147B0
:101B1000639CE70490080C08528597000000E7805A
:101B2000C0E925D181A0B3069B00BA871008B30590
:101B3000F60090083E9603C506000346060085079A
:101B40008506298E2380C500E39277FF998F900840
:101B50000C085285BE9497000000E78000E6894794
:101B6000014749D12A84B1B790083E960346060042
:101B70001408BE962380C600850759BFB247850466
:101B80006387971481471808B306F70098083E97B3
:101B90003386F90003470700034606008507318FA7
:101BA0002380E600E39177FF90080C0852859700A8
:101BB0000000E78080E05DF53546E2851305110100
:101BC0002308B10197E00000E780A0D51397040136
:101BD0004183939784002183D98F10180C08528574
:101BE000231FF10097000000E78020DD25FD8147DD
:101BF00010183387F9003E96034707000346060096
:101C0000B306FB008507318F2380E600E39277FF60
:101C100065A81808B306F70098083E973386F900C0
:101C200003470700034606008507318F2380E6003F
:101C3000E3E127FFCA87639E770990080C08528565
:101C400097000000E78060D711FD81479800B30638
:101C5000F700900818103E973E960347070003468A
:101C600006008507318F2380E600E39177FF354634
:101C7000E285130511012308B10197E00000E78018
:101C800040CA139704014183939784002183D98F1D
:101C900010180C085285231FF10097000000E78000
:101CA000C0D1E31105EC814710183387F9003E9647
:101CB0000347070003460600B306FB008507318F84
:101CC0002380E600E3E227FFC109410BC1BB814746
:101CD00085B79408BE9683C6060018083E97230071
:101CE000D700850789BF638006321703FFFFE7022D
:101CF000033C59712A84BE89B28B8547354613054A
:101D000011022E8B468C4289BA8A368A2300F10250
:101D100097E00000E780E0C010180C102285231720
:101D2000010297000000E78040C963180512A1472F
:101D3000631FFC069307900563930900E54735464A
:101D4000DA851305110293140A012300F102C18000
:101D500097E00000E780E0BC93178A0013D7840067
:101D6000D98F90080C1022852317F10297000000EC
:101D7000E780A0C47DE1639209049307FA00BD885F
:101D8000918391E0C144C207C183DE8C814A3EC683
:101D9000414DB24763E2FA0E6286B3854B0188106B
:101DA00097E00000E78080B54DC93D557DA09307C1
:101DB0009004E39609F8A54759B7834701050947F9
:101DC000C14C2300F10283471105B3C7F900A300FA
:101DD000F10293872900814963E1FC0481461810D0
:101DE0003306D7008C083387D900B695569703473A
:101DF000070083C5050085062D8F2300E600E390CC
:101E0000D7FE41476390E70690080C1022859700A3
:101E10000000E78080BA35D189A0B3863A01BA873D
:101E20001010B305F60090083E9603C50600034661
:101E3000060085078506298E2380C500E39297FF5B
:101E40003387EC4090080C102285BA999700000067
:101E5000E780A0B68947014741D165611703FFFFBD
:101E60006700A32890083E96034606001410BE960D
:101E70002380C600850779B7B247850A93990A017E
:101E8000939D8A0093D909016391570F8547354681
:101E9000DA85130511022300F10293D9890097E036
:101EA0000000E78000A8B3ED3D0190000C102285F2
:101EB0002317B10397000000E78020B059FD814748
:101EC000A68963EA970626860C084A8597E00000F3
:101ED000E78020A581471810B306F700100898087E
:101EE0003E973E9603470700034606008507318F5D
:101EF0002380E600E3E197FE639FA90590080C109C
:101F0000228597000000E78040AB21F981479810B7
:101F1000B306F700900818183E973E96034707004F
:101F2000034606008507318F2380E600E391A7FF73
:101F30004109C10CB9BD18089000B306F7003E96E0
:101F40003387FC0003470700034606008507318FEF
:101F50002380E600B5B798084E97034707001C108A
:101F6000CE972380E700850941BF85473546DA854E
:101F7000130511022300F10293D9890097E00000B4
:101F8000E780209AB3ED3D0190000C1022852317C5
:101F9000B10397000000E78040A2E31005EC814701
:101FA00018089000B306F7003E963387FC000347FD
:101FB0000700034606008507318F2380E600E39182
:101FC000A7FF41460C084A8597E00000E78060952E
:101FD00081471810B306F700100898083E973E9600
:101FE00003470700034606008507318F2380E6007C
:101FF000E391A7FF90080C10228597000000E7806E
:10200000C09B1DD599BD7D5582801703FFFFE70258
:10201000030D01112A842E8593055100328902C0D7
:1020200002C202C402C69304740097F0FFFFE78067
:10203000A03D1D46A6851305910097E00000E780AE
:10204000408E10088A854A8597000000E780E09658
:1020500019ED93071400180883C60700034607000C
:1020600085070507B18EA38FD7FEE397F4FE0561C0
:102070001703FFFF6700E3081703FFFFE70283046E
:102080002E848C414111AA8983871500328991449D
:1020900063D30700A1449747FF1F938767389C438A
:1020A000A1C7C1CA8D472310F10083C725004A8507
:1020B0002301F10083C73500A301F10083C7450068
:1020C0002302F10083C75500A302F10083C7650016
:1020D00093059100A30301002303F10023040100F1
:1020E00097F0FFFFE78040320C404A860A8597F060
:1020F000FFFFE78080330328040083564400A6884E
:102100001D0881470147E51642868A854E8597005E
:102110000000E780408E2A8919E5A685228597B0C0
:10212000FFFFE780E0C14A8541011703FFFF670019
:10213000A3FC4A860A8597F0FFFFE780002F6DB762
:102140001703FFFFE70203F82E848C414111AA898F
:10215000838715003289914463D30700A1449747D0
:10216000FF1F9387E72B9C43A1C7C1C68D47231050
:10217000F10083C725004A852301F10083C735009C
:10218000A301F10083C745002302F10083C7550076
:10219000A302F10083C7650093059100A30301002A
:1021A0002303F1002304010097F0FFFFE780C0251F
:1021B0000C404A860A8597F0FFFFE7800027835688
:1021C0004400032804008A85858EC2061D08C1824A
:1021D0002312D400A68881470147E51642864E8522
:1021E00097000000E78060B041011703FFFF670020
:1021F000A3F04A860A8597F0FFFFE78000234DBFD2
:102200001703FFFFE702A3EDB335B0000111850509
:102210002A891315F601336515012308B1009305CA
:10222000110136843AC632C03EC442C297F0FFFF65
:10223000E780801DA2471248425593D68700230BA2
:10224000F1009305910193578800A30AD100A30BD5
:10225000F100230C010197F0FFFFE780E01A3247FD
:10226000024603280400B337E00083564400920777
:10227000914411C2A1444A85A68842860C0897F071
:10228000FFFFE78040772A8919E5A685228597B068
:10229000FFFFE780E0AA4A8505611703FFFF67009B
:1022A00043E61703FFFFE702E3E101113EC686475D
:1022B000B335B0008505AA891315F6015D8D230895
:1022C000B1009305110136843A89B28442C446C2F2
:1022D00097F0FFFFE7804013224892481645935736
:1022E0008800A30AF1009305910193D78800230B7E
:1022F0000101A30BF100230C110197F0FFFFE78010
:10230000A0103247104083564400B337E0009207D4
:1023100003280900914891C0A1480C084E859700F8
:102320000000E780809CAA8401E9835544004A8527
:1023300097B0FFFFE780C0A0268505611703FFFF68
:10234000670083DBAA959307F00F171701001307A7
:10235000E7936317B50013C5F7FF1375F50F828078
:1023600005058346F5FFB58FBA9783C70700D5B734
:102370000357450014419307F00F17160100130689
:10238000E690369742074183139506014181631B0E
:10239000E500AD8FB29703C50700130515F313359C
:1023A00015008280850603C5F6FFA98FB29783C703
:1023B0000700D9BF1703FFFFE70263D2B287368455
:1023C0002E86BA86AA853E85BA8497F0FFFFE780FD
:1023D0006052634F0500228597D00000E780E078C7
:1023E0002A86A686A285268597F0FFFFE780805083
:1023F0001703FFFF6700E3D01703FFFFE70283CC5B
:102400005D712A8BAE8A171501001305A5852C0076
:10241000B284368ABA893E8997F0FFFFE780C04FC1
:102420002A845DE134104146DA85280097F0FFFFE9
:10243000E780404C2A8449E98547A303F100A6C2FE
:10244000930771002408BEC4A68685470D462C1844
:10245000281002DC02DED6C0BEC697F0FFFFE78080
:1024600000442A8435E183477102A6860D4693F71E
:10247000F7072300FA00C1473EDE2C1889472810D1
:1024800026DCA303F10097F0FFFFE78040412A8498
:1024900005ED4146A6854E8597D00000E78060484F
:1024A0008D47A6860D462C182810A303F10097F03F
:1024B000FFFFE780C03E2A8401E94146A6854A85A0
:1024C00097D00000E780E045228561611703FFFF98
:1024D000670083C21703FFFFE70263C097F700009E
:1024E000938787A1984383C7470079712A89AE846F
:1024F00017050100130585770C083AC42306F1007F
:1025000097F0FFFFE78040412A8405ED1410414613
:10251000CA85080897F0FFFFE780C03D2A8415E1CF
:10252000140815462C00081097F0FFFFE780803C48
:102530002A8401E921462C08268597D00000E780EF
:10254000403E228545611703FFFF670083BB1703E9
:10255000FFFFE702C3B897F700009387E7999C470E
:102560007971AA842E84170501001305A5700C0843
:102570003EC697F0FFFFE780203A0DE91410414670
:10258000A685080897F0FFFFE780C03605E114082C
:1025900011466C00081097F0FFFFE780A03519E5A1
:1025A0008347F10193F7F7032300F4004561170314
:1025B000FFFF670003B51703FFFFE70243B236884A
:1025C000A14881470147E54697F0FFFFE780A04219
:1025D0001703FFFF6700E3B21703FFFFE70223B013
:1025E0003688A14881470147E54697F0FFFFE7801D
:1025F000C06F1703FFFF6700C3B01703FFFFE702B9
:1026000003AE01112A842E850C0832C697F0FFFF15
:10261000E780803009ED3247970601009386066413
:102620001008C145228597000000E780E0D80561C9
:102630001703FFFF6700E3AC1703FFFFE70223AABE
:102640004111C1472EC032C48A8509463EC23EC6EA
:1026500097F0FFFFE780A02441011703FFFF670009
:1026600043AA1703FFFFE70283A74111AE861306B3
:102670001009AA850A8502C002C202C402C697F0E8
:10268000FFFFE780202741011703FFFF670063A7D3
:102690001703FFFFE702A3A4328797060100938682
:1026A000E65D2E869305000297000000E780C0D00B
:1026B0001703FFFF6700E3A41703FFFFE70223A24E
:1026C0007971C1472ACC2ED032D42C080D4628006F
:1026D0003ECE3ED23ED602C402C602C802CA97F01F
:1026E000FFFFE780C01B45611703FFFF670063A181
:1026F0001703FFFFE702A39E0111AA842E8417058A
:102700000100130525588A8597F0FFFFE780C02058
:1027100015E514084146A6850A8597F0FFFFE78076
:10272000601D09ED8347E1010347F101A207D98F3D
:10273000CA07C9836177D98F2310F4000561170395
:10274000FFFF6700039C15CD1703FFFFE7022399E6
:102750009737FF1F9387477A90439735FF1F9385DD
:10276000E5791735FF1F1305257597D00000E78021
:1027700000C51735FF1F130525741703FFFF6700FA
:1027800043981735FF1F1305257382808DCD1703DE
:10279000FFFFE702C3949737FF1F9387E7759443C2
:1027A00001112E840A869735FF1F9385257597D0D2
:1027B0000000E78040C60A850294014505611703C1
:1027C000FFFF670003947D5582801703FFFFE70238
:1027D000039197D00000E78080D19737FF1F23AD8A
:1027E000A77017F5FFFF1305E5C997B00000E78054
:1027F000C0741703FFFF6700C3901737FF1F13074D
:10280000E7719317150008433E95FD572310F50017
:1028100082801703FFFFE702838C2A84084009E5C2
:102820001703FFFF6700E38D1C4158401CC0631372
:10283000E5005CC08347550023200500F99BA302F7
:10284000F50097A0FFFFE780207CC9BF1703FFFFBB
:10285000E70243879737FF1F9387476E98432A8481
:1028600011CB8347350093F7070289C7035505004D
:10287000894502971305440197B00000E780403B6B
:10288000835504000355E40097300000E780A00C56
:10289000485819C597A0FFFFE7800077232A040254
:1028A0001305840397000000E780E0F68144B149F6
:1028B0009790FFFFE780206A63CBA4028347340030
:1028C0002320040493F727FCA301F4000048979009
:1028D000FFFFE780406913161500814522859700A8
:1028E000FFFFE780C0821703FFFF6700E380B38725
:1028F00034030329040385043E994A8597000000A8
:10290000E78060F12304090065B78347350093F73A
:10291000070299E3014582808357E500E39CB7FEF7
:10292000C167FD176316F60005458280054599A825
:1029300017F3FEFFE702A37A93170601C187B2845B
:102940002A8401496359F002835705009DCB014554
:102950006367F600034584003E953325A600137592
:10296000F50F0DA01C4813171900BA9783D707005D
:10297000E38E97FA05099790FFFFE780C05EE34377
:10298000A9FE014517F3FEFF6700A37717F3FEFFCB
:10299000E7024373AE89AA849790FFFFE7806052F5
:1029A0002A8497D0FFFFE780A02EAA86014713064E
:1029B000840197050000938585E41735FF1F1305F3
:1029C00025569790FFFFE780E0182A8925C98C4497
:1029D0001304C50022859E0593F5050897A0FFFF07
:1029E000E780403CCC4083877400E18163DD0704CD
:1029F00093E50508228597A0FFFFE780A03A0D46E2
:102A000093854400228597A0FFFFE780C03683D5D9
:102A10000400228597A0FFFFE780E03D83D52400D6
:102A2000228597A0FFFFE780003D03D6490083A5DC
:102A30000900228597A0FFFFE780E0334A8517F35E
:102A4000FEFF6700636B93F5F5076DB717F3FEFFA5
:102A5000E702E36801112A84328532C697A0FFFF9E
:102A6000E780E0279780FFFFE780C03083570400AE
:102A70001737FF1F130707643246231BF100930724
:102A800000F8A30DF1001C471843231AA100898305
:102A9000858BB307F740B28548083ECE231C010062
:102AA000230D010097000000E78080EE056117F319
:102AB000FEFF6700036517F3FEFFE702A360004116
:102AC00001453DC49304C40026853289AE8997A090
:102AD000FFFFE780C02495452A8A2685035B040111
:102AE00097A0FFFFE7802021268597A0FFFFE780C2
:102AF000603E8D45AA8A268597A0FFFFE780A01F2C
:102B0000268597A0FFFFE780E03C5C48420A135A05
:102B10000A01D2975CC423186401814763983A0183
:102B200046054D81330625419337160013F5F70FFF
:102B300017F3FEFF6700435C17F3FEFFE702A3579E
:102B400089692A8BAE8B328AB68A81440144314C22
:102B5000FD199790FFFFE780004063CDA400979098
:102B6000FFFFE7804042018D33B5AA0017F3FEFF57
:102B70006700E3573389840383270B003E9963176B
:102B80000A008347890085043E94E1B703560A0092
:102B9000DE854A8533F6C90097000000E780E0F142
:102BA0006DD10545E1B717F3FEFFE702435301116D
:102BB0002A847C000355E5003ECAB70707003ECCD7
:102BC0007C003ECE97200000E78020082A898545BA
:102BD000480897A0FFFFE78020399945480897A04B
:102BE000FFFFE780E015AA844A8597200000E78070
:102BF000A0082380A4009737FF1F9387A74B9C430F
